
ConwayVGA.elf:     file format elf32-littlearm

Sections:
Idx Name          Size      VMA       LMA       File off  Algn
  0 .text         00001f78  00000000  00000000  00010000  2**2
                  CONTENTS, ALLOC, LOAD, READONLY, CODE
  1 .relocate     00000000  20000000  20000000  00011f78  2**0
                  CONTENTS
  2 .bss          000002bc  20000000  20000000  00020000  2**2
                  ALLOC
  3 .stack        00000404  200002bc  200002bc  00020000  2**0
                  ALLOC
  4 .ARM.attributes 00000028  00000000  00000000  00011f78  2**0
                  CONTENTS, READONLY
  5 .comment      00000059  00000000  00000000  00011fa0  2**0
                  CONTENTS, READONLY
  6 .debug_info   0002c21c  00000000  00000000  00011ff9  2**0
                  CONTENTS, READONLY, DEBUGGING
  7 .debug_abbrev 00002c3b  00000000  00000000  0003e215  2**0
                  CONTENTS, READONLY, DEBUGGING
  8 .debug_loc    000115e7  00000000  00000000  00040e50  2**0
                  CONTENTS, READONLY, DEBUGGING
  9 .debug_aranges 00000aa0  00000000  00000000  00052437  2**0
                  CONTENTS, READONLY, DEBUGGING
 10 .debug_ranges 00000cf0  00000000  00000000  00052ed7  2**0
                  CONTENTS, READONLY, DEBUGGING
 11 .debug_macro  000177e2  00000000  00000000  00053bc7  2**0
                  CONTENTS, READONLY, DEBUGGING
 12 .debug_line   0000db94  00000000  00000000  0006b3a9  2**0
                  CONTENTS, READONLY, DEBUGGING
 13 .debug_str    00082fba  00000000  00000000  00078f3d  2**0
                  CONTENTS, READONLY, DEBUGGING
 14 .debug_frame  00001c84  00000000  00000000  000fbef8  2**2
                  CONTENTS, READONLY, DEBUGGING

Disassembly of section .text:

00000000 <exception_table>:
       0:	c0 06 00 20 25 01 00 00 21 01 00 00 21 01 00 00     ... %...!...!...
	...
      2c:	21 01 00 00 00 00 00 00 00 00 00 00 21 01 00 00     !...........!...
      3c:	21 01 00 00 21 01 00 00 21 01 00 00 21 01 00 00     !...!...!...!...
      4c:	0d 0c 00 00 21 01 00 00 21 01 00 00 21 01 00 00     ....!...!...!...
      5c:	91 1d 00 00 21 01 00 00 21 01 00 00 21 01 00 00     ....!...!...!...
      6c:	21 01 00 00 21 01 00 00 00 00 00 00 00 00 00 00     !...!...........
      7c:	21 01 00 00 21 01 00 00 21 01 00 00 21 01 00 00     !...!...!...!...
      8c:	21 01 00 00 21 01 00 00 00 00 00 00 00 00 00 00     !...!...........
      9c:	21 01 00 00 21 01 00 00 21 01 00 00 21 01 00 00     !...!...!...!...
      ac:	21 01 00 00 00 00 00 00                             !.......

000000b4 <__do_global_dtors_aux>:
      b4:	b510      	push	{r4, lr}
      b6:	4c06      	ldr	r4, [pc, #24]	; (d0 <__do_global_dtors_aux+0x1c>)
      b8:	7823      	ldrb	r3, [r4, #0]
      ba:	2b00      	cmp	r3, #0
      bc:	d107      	bne.n	ce <__do_global_dtors_aux+0x1a>
      be:	4b05      	ldr	r3, [pc, #20]	; (d4 <__do_global_dtors_aux+0x20>)
      c0:	2b00      	cmp	r3, #0
      c2:	d002      	beq.n	ca <__do_global_dtors_aux+0x16>
      c4:	4804      	ldr	r0, [pc, #16]	; (d8 <__do_global_dtors_aux+0x24>)
      c6:	e000      	b.n	ca <__do_global_dtors_aux+0x16>
      c8:	bf00      	nop
      ca:	2301      	movs	r3, #1
      cc:	7023      	strb	r3, [r4, #0]
      ce:	bd10      	pop	{r4, pc}
      d0:	20000000 	.word	0x20000000
      d4:	00000000 	.word	0x00000000
      d8:	00001f78 	.word	0x00001f78

000000dc <frame_dummy>:
      dc:	4b08      	ldr	r3, [pc, #32]	; (100 <frame_dummy+0x24>)
      de:	b510      	push	{r4, lr}
      e0:	2b00      	cmp	r3, #0
      e2:	d003      	beq.n	ec <frame_dummy+0x10>
      e4:	4907      	ldr	r1, [pc, #28]	; (104 <frame_dummy+0x28>)
      e6:	4808      	ldr	r0, [pc, #32]	; (108 <frame_dummy+0x2c>)
      e8:	e000      	b.n	ec <frame_dummy+0x10>
      ea:	bf00      	nop
      ec:	4807      	ldr	r0, [pc, #28]	; (10c <frame_dummy+0x30>)
      ee:	6803      	ldr	r3, [r0, #0]
      f0:	2b00      	cmp	r3, #0
      f2:	d100      	bne.n	f6 <frame_dummy+0x1a>
      f4:	bd10      	pop	{r4, pc}
      f6:	4b06      	ldr	r3, [pc, #24]	; (110 <frame_dummy+0x34>)
      f8:	2b00      	cmp	r3, #0
      fa:	d0fb      	beq.n	f4 <frame_dummy+0x18>
      fc:	4798      	blx	r3
      fe:	e7f9      	b.n	f4 <frame_dummy+0x18>
     100:	00000000 	.word	0x00000000
     104:	20000004 	.word	0x20000004
     108:	00001f78 	.word	0x00001f78
     10c:	00001f78 	.word	0x00001f78
     110:	00000000 	.word	0x00000000

00000114 <atmel_start_init>:

/**
 * Initializes MCU, drivers and middleware in the project
 **/
void atmel_start_init(void)
{
     114:	b510      	push	{r4, lr}
	system_init();
     116:	4b01      	ldr	r3, [pc, #4]	; (11c <atmel_start_init+0x8>)
     118:	4798      	blx	r3
}
     11a:	bd10      	pop	{r4, pc}
     11c:	00000401 	.word	0x00000401

00000120 <Dummy_Handler>:

/**
 * \brief Default interrupt handler for unused IRQs.
 */
void Dummy_Handler(void)
{
     120:	e7fe      	b.n	120 <Dummy_Handler>
	...

00000124 <Reset_Handler>:
{
     124:	b5f8      	push	{r3, r4, r5, r6, r7, lr}
        if (pSrc != pDest) {
     126:	4a23      	ldr	r2, [pc, #140]	; (1b4 <Reset_Handler+0x90>)
     128:	4b23      	ldr	r3, [pc, #140]	; (1b8 <Reset_Handler+0x94>)
     12a:	429a      	cmp	r2, r3
     12c:	d009      	beq.n	142 <Reset_Handler+0x1e>
     12e:	4b22      	ldr	r3, [pc, #136]	; (1b8 <Reset_Handler+0x94>)
     130:	4a20      	ldr	r2, [pc, #128]	; (1b4 <Reset_Handler+0x90>)
     132:	e003      	b.n	13c <Reset_Handler+0x18>
                        *pDest++ = *pSrc++;
     134:	6811      	ldr	r1, [r2, #0]
     136:	6019      	str	r1, [r3, #0]
     138:	3304      	adds	r3, #4
     13a:	3204      	adds	r2, #4
                for (; pDest < &_erelocate;) {
     13c:	491f      	ldr	r1, [pc, #124]	; (1bc <Reset_Handler+0x98>)
     13e:	428b      	cmp	r3, r1
     140:	d3f8      	bcc.n	134 <Reset_Handler+0x10>
                        *pDest++ = *pSrc++;
     142:	4b1f      	ldr	r3, [pc, #124]	; (1c0 <Reset_Handler+0x9c>)
     144:	e002      	b.n	14c <Reset_Handler+0x28>
                *pDest++ = 0;
     146:	2200      	movs	r2, #0
     148:	601a      	str	r2, [r3, #0]
     14a:	3304      	adds	r3, #4
        for (pDest = &_szero; pDest < &_ezero;) {
     14c:	4a1d      	ldr	r2, [pc, #116]	; (1c4 <Reset_Handler+0xa0>)
     14e:	4293      	cmp	r3, r2
     150:	d3f9      	bcc.n	146 <Reset_Handler+0x22>
        SCB->VTOR = ((uint32_t) pSrc & SCB_VTOR_TBLOFF_Msk);
     152:	4a1d      	ldr	r2, [pc, #116]	; (1c8 <Reset_Handler+0xa4>)
     154:	21ff      	movs	r1, #255	; 0xff
     156:	4b1d      	ldr	r3, [pc, #116]	; (1cc <Reset_Handler+0xa8>)
     158:	438b      	bics	r3, r1
     15a:	6093      	str	r3, [r2, #8]
        SBMATRIX->SFR[SBMATRIX_SLAVE_HMCRAMC0].reg = 2;
     15c:	39fd      	subs	r1, #253	; 0xfd
     15e:	2390      	movs	r3, #144	; 0x90
     160:	005b      	lsls	r3, r3, #1
     162:	4a1b      	ldr	r2, [pc, #108]	; (1d0 <Reset_Handler+0xac>)
     164:	50d1      	str	r1, [r2, r3]
        USB->DEVICE.QOSCTRL.bit.CQOS = 2;
     166:	4a1b      	ldr	r2, [pc, #108]	; (1d4 <Reset_Handler+0xb0>)
     168:	78d3      	ldrb	r3, [r2, #3]
     16a:	2503      	movs	r5, #3
     16c:	43ab      	bics	r3, r5
     16e:	2402      	movs	r4, #2
     170:	4323      	orrs	r3, r4
     172:	70d3      	strb	r3, [r2, #3]
        USB->DEVICE.QOSCTRL.bit.DQOS = 2;
     174:	78d3      	ldrb	r3, [r2, #3]
     176:	270c      	movs	r7, #12
     178:	43bb      	bics	r3, r7
     17a:	2608      	movs	r6, #8
     17c:	4333      	orrs	r3, r6
     17e:	70d3      	strb	r3, [r2, #3]
        DMAC->QOSCTRL.bit.DQOS = 2;
     180:	4b15      	ldr	r3, [pc, #84]	; (1d8 <Reset_Handler+0xb4>)
     182:	7b98      	ldrb	r0, [r3, #14]
     184:	2230      	movs	r2, #48	; 0x30
     186:	4390      	bics	r0, r2
     188:	2220      	movs	r2, #32
     18a:	4310      	orrs	r0, r2
     18c:	7398      	strb	r0, [r3, #14]
        DMAC->QOSCTRL.bit.FQOS = 2;
     18e:	7b99      	ldrb	r1, [r3, #14]
     190:	43b9      	bics	r1, r7
     192:	4331      	orrs	r1, r6
     194:	7399      	strb	r1, [r3, #14]
        DMAC->QOSCTRL.bit.WRBQOS = 2;
     196:	7b9a      	ldrb	r2, [r3, #14]
     198:	43aa      	bics	r2, r5
     19a:	4322      	orrs	r2, r4
     19c:	739a      	strb	r2, [r3, #14]
        NVMCTRL->CTRLB.bit.MANW = 1;
     19e:	4a0f      	ldr	r2, [pc, #60]	; (1dc <Reset_Handler+0xb8>)
     1a0:	6851      	ldr	r1, [r2, #4]
     1a2:	2380      	movs	r3, #128	; 0x80
     1a4:	430b      	orrs	r3, r1
     1a6:	6053      	str	r3, [r2, #4]
        __libc_init_array();
     1a8:	4b0d      	ldr	r3, [pc, #52]	; (1e0 <Reset_Handler+0xbc>)
     1aa:	4798      	blx	r3
        main();
     1ac:	4b0d      	ldr	r3, [pc, #52]	; (1e4 <Reset_Handler+0xc0>)
     1ae:	4798      	blx	r3
     1b0:	e7fe      	b.n	1b0 <Reset_Handler+0x8c>
     1b2:	46c0      	nop			; (mov r8, r8)
     1b4:	00001f78 	.word	0x00001f78
     1b8:	20000000 	.word	0x20000000
     1bc:	20000000 	.word	0x20000000
     1c0:	20000000 	.word	0x20000000
     1c4:	200002bc 	.word	0x200002bc
     1c8:	e000ed00 	.word	0xe000ed00
     1cc:	00000000 	.word	0x00000000
     1d0:	41007000 	.word	0x41007000
     1d4:	41005000 	.word	0x41005000
     1d8:	41004800 	.word	0x41004800
     1dc:	41004000 	.word	0x41004000
     1e0:	00001dd5 	.word	0x00001dd5
     1e4:	00001d9d 	.word	0x00001d9d

000001e8 <TIMER_0_init>:
 * \brief Timer initialization function
 *
 * Enables Timer peripheral, clocks and initializes Timer driver
 */
static void TIMER_0_init(void)
{
     1e8:	b510      	push	{r4, lr}
			peripheral = (uint32_t)_pm_get_ahb_index(module);
			PM->AHBMASK.reg |= 1 << peripheral;
		}
		break;
	case PM_BUS_APBA:
		PM->APBAMASK.reg |= 1 << peripheral;
     1ea:	4a08      	ldr	r2, [pc, #32]	; (20c <TIMER_0_init+0x24>)
     1ec:	6993      	ldr	r3, [r2, #24]
     1ee:	2120      	movs	r1, #32
     1f0:	430b      	orrs	r3, r1
     1f2:	6193      	str	r3, [r2, #24]
}

static inline void hri_gclk_write_CLKCTRL_reg(const void *const hw, hri_gclk_clkctrl_reg_t data)
{
	GCLK_CRITICAL_SECTION_ENTER();
	((Gclk *)hw)->CLKCTRL.reg = data;
     1f4:	4a06      	ldr	r2, [pc, #24]	; (210 <TIMER_0_init+0x28>)
     1f6:	4b07      	ldr	r3, [pc, #28]	; (214 <TIMER_0_init+0x2c>)
     1f8:	805a      	strh	r2, [r3, #2]
	_pm_enable_bus_clock(PM_BUS_APBA, RTC);
	_gclk_enable_channel(RTC_GCLK_ID, CONF_GCLK_RTC_SRC);
	timer_init(&TIMER_0, RTC, _rtc_get_timer());
     1fa:	4b07      	ldr	r3, [pc, #28]	; (218 <TIMER_0_init+0x30>)
     1fc:	4798      	blx	r3
     1fe:	0002      	movs	r2, r0
     200:	4906      	ldr	r1, [pc, #24]	; (21c <TIMER_0_init+0x34>)
     202:	4807      	ldr	r0, [pc, #28]	; (220 <TIMER_0_init+0x38>)
     204:	4b07      	ldr	r3, [pc, #28]	; (224 <TIMER_0_init+0x3c>)
     206:	4798      	blx	r3
}
     208:	bd10      	pop	{r4, pc}
     20a:	46c0      	nop			; (mov r8, r8)
     20c:	40000400 	.word	0x40000400
     210:	00004004 	.word	0x00004004
     214:	40000c00 	.word	0x40000c00
     218:	00000c09 	.word	0x00000c09
     21c:	40001400 	.word	0x40001400
     220:	200002a0 	.word	0x200002a0
     224:	0000077d 	.word	0x0000077d

00000228 <SPI_0_PORT_init>:
{
     228:	b5f0      	push	{r4, r5, r6, r7, lr}
     22a:	46c6      	mov	lr, r8
     22c:	b500      	push	{lr}
	((Port *)hw)->Group[submodule_index].OUTCLR.reg = ~data;
}

static inline void hri_port_clear_OUT_reg(const void *const hw, uint8_t submodule_index, hri_port_out_reg_t mask)
{
	((Port *)hw)->Group[submodule_index].OUTCLR.reg = mask;
     22e:	22c0      	movs	r2, #192	; 0xc0
     230:	05d2      	lsls	r2, r2, #23
     232:	2310      	movs	r3, #16
     234:	6153      	str	r3, [r2, #20]
	((Port *)hw)->Group[submodule_index].DIRSET.reg = mask;
     236:	6093      	str	r3, [r2, #8]

static inline void hri_port_write_WRCONFIG_reg(const void *const hw, uint8_t submodule_index,
                                               hri_port_wrconfig_reg_t data)
{
	PORT_CRITICAL_SECTION_ENTER();
	((Port *)hw)->Group[submodule_index].WRCONFIG.reg = data;
     238:	4b25      	ldr	r3, [pc, #148]	; (2d0 <SPI_0_PORT_init+0xa8>)
     23a:	4926      	ldr	r1, [pc, #152]	; (2d4 <SPI_0_PORT_init+0xac>)
     23c:	6299      	str	r1, [r3, #40]	; 0x28
     23e:	21c0      	movs	r1, #192	; 0xc0
     240:	0609      	lsls	r1, r1, #24
     242:	468c      	mov	ip, r1
     244:	6299      	str	r1, [r3, #40]	; 0x28
	tmp = ((Port *)hw)->Group[submodule_index].PINCFG[index].reg;
     246:	2044      	movs	r0, #68	; 0x44
     248:	5c19      	ldrb	r1, [r3, r0]
	tmp &= ~PORT_PINCFG_PMUXEN;
     24a:	2701      	movs	r7, #1
     24c:	43b9      	bics	r1, r7
	tmp |= value << PORT_PINCFG_PMUXEN_Pos;
     24e:	2601      	movs	r6, #1
     250:	4331      	orrs	r1, r6
     252:	b2c9      	uxtb	r1, r1
	((Port *)hw)->Group[submodule_index].PINCFG[index].reg = tmp;
     254:	5419      	strb	r1, [r3, r0]
	tmp = ((Port *)hw)->Group[submodule_index].PMUX[index].reg;
     256:	2132      	movs	r1, #50	; 0x32
     258:	5c58      	ldrb	r0, [r3, r1]
	tmp &= ~PORT_PMUX_PMUXE_Msk;
     25a:	250f      	movs	r5, #15
     25c:	43a8      	bics	r0, r5
	tmp |= PORT_PMUX_PMUXE(data);
     25e:	2403      	movs	r4, #3
     260:	46a0      	mov	r8, r4
     262:	4644      	mov	r4, r8
     264:	4320      	orrs	r0, r4
     266:	b2c0      	uxtb	r0, r0
	((Port *)hw)->Group[submodule_index].PMUX[index].reg = tmp;
     268:	5458      	strb	r0, [r3, r1]
	((Port *)hw)->Group[submodule_index].OUTCLR.reg = mask;
     26a:	2020      	movs	r0, #32
     26c:	6150      	str	r0, [r2, #20]
	((Port *)hw)->Group[submodule_index].DIRSET.reg = mask;
     26e:	6090      	str	r0, [r2, #8]
	((Port *)hw)->Group[submodule_index].WRCONFIG.reg = data;
     270:	4819      	ldr	r0, [pc, #100]	; (2d8 <SPI_0_PORT_init+0xb0>)
     272:	6298      	str	r0, [r3, #40]	; 0x28
     274:	4660      	mov	r0, ip
     276:	6298      	str	r0, [r3, #40]	; 0x28
	tmp = ((Port *)hw)->Group[submodule_index].PINCFG[index].reg;
     278:	2045      	movs	r0, #69	; 0x45
     27a:	4684      	mov	ip, r0
     27c:	5c18      	ldrb	r0, [r3, r0]
	tmp &= ~PORT_PINCFG_PMUXEN;
     27e:	43b8      	bics	r0, r7
	tmp |= value << PORT_PINCFG_PMUXEN_Pos;
     280:	4330      	orrs	r0, r6
     282:	b2c0      	uxtb	r0, r0
	((Port *)hw)->Group[submodule_index].PINCFG[index].reg = tmp;
     284:	4664      	mov	r4, ip
     286:	5518      	strb	r0, [r3, r4]
	tmp = ((Port *)hw)->Group[submodule_index].PMUX[index].reg;
     288:	5c58      	ldrb	r0, [r3, r1]
	tmp &= ~PORT_PMUX_PMUXO_Msk;
     28a:	3c36      	subs	r4, #54	; 0x36
     28c:	4020      	ands	r0, r4
	tmp |= PORT_PMUX_PMUXO(data);
     28e:	2430      	movs	r4, #48	; 0x30
     290:	46a4      	mov	ip, r4
     292:	4664      	mov	r4, ip
     294:	4320      	orrs	r0, r4
     296:	b2c0      	uxtb	r0, r0
	((Port *)hw)->Group[submodule_index].PMUX[index].reg = tmp;
     298:	5458      	strb	r0, [r3, r1]
	((Port *)hw)->Group[submodule_index].DIRCLR.reg = mask;
     29a:	310e      	adds	r1, #14
     29c:	6051      	str	r1, [r2, #4]
	((Port *)hw)->Group[submodule_index].WRCONFIG.reg = data;
     29e:	4a0f      	ldr	r2, [pc, #60]	; (2dc <SPI_0_PORT_init+0xb4>)
     2a0:	629a      	str	r2, [r3, #40]	; 0x28
     2a2:	4a0f      	ldr	r2, [pc, #60]	; (2e0 <SPI_0_PORT_init+0xb8>)
     2a4:	629a      	str	r2, [r3, #40]	; 0x28
	((Port *)hw)->Group[submodule_index].PINCFG[index].reg &= ~PORT_PINCFG_PULLEN;
     2a6:	2246      	movs	r2, #70	; 0x46
     2a8:	5c99      	ldrb	r1, [r3, r2]
     2aa:	2004      	movs	r0, #4
     2ac:	4381      	bics	r1, r0
     2ae:	5499      	strb	r1, [r3, r2]
	tmp = ((Port *)hw)->Group[submodule_index].PINCFG[index].reg;
     2b0:	5c99      	ldrb	r1, [r3, r2]
	tmp &= ~PORT_PINCFG_PMUXEN;
     2b2:	43b9      	bics	r1, r7
	tmp |= value << PORT_PINCFG_PMUXEN_Pos;
     2b4:	4331      	orrs	r1, r6
     2b6:	b2c9      	uxtb	r1, r1
	((Port *)hw)->Group[submodule_index].PINCFG[index].reg = tmp;
     2b8:	5499      	strb	r1, [r3, r2]
	tmp = ((Port *)hw)->Group[submodule_index].PMUX[index].reg;
     2ba:	2133      	movs	r1, #51	; 0x33
     2bc:	5c5a      	ldrb	r2, [r3, r1]
	tmp &= ~PORT_PMUX_PMUXE_Msk;
     2be:	43aa      	bics	r2, r5
	tmp |= PORT_PMUX_PMUXE(data);
     2c0:	4640      	mov	r0, r8
     2c2:	4302      	orrs	r2, r0
     2c4:	b2d2      	uxtb	r2, r2
	((Port *)hw)->Group[submodule_index].PMUX[index].reg = tmp;
     2c6:	545a      	strb	r2, [r3, r1]
}
     2c8:	bc04      	pop	{r2}
     2ca:	4690      	mov	r8, r2
     2cc:	bdf0      	pop	{r4, r5, r6, r7, pc}
     2ce:	46c0      	nop			; (mov r8, r8)
     2d0:	41004400 	.word	0x41004400
     2d4:	40000010 	.word	0x40000010
     2d8:	40000020 	.word	0x40000020
     2dc:	40020040 	.word	0x40020040
     2e0:	c0020000 	.word	0xc0020000

000002e4 <SPI_0_CLOCK_init>:
			peripheral = (uint32_t)_pm_get_apbb_index(module);
			PM->APBBMASK.reg |= 1 << peripheral;
		}
		break;
	case PM_BUS_APBC:
		PM->APBCMASK.reg |= 1 << peripheral;
     2e4:	4a04      	ldr	r2, [pc, #16]	; (2f8 <SPI_0_CLOCK_init+0x14>)
     2e6:	6a13      	ldr	r3, [r2, #32]
     2e8:	2104      	movs	r1, #4
     2ea:	430b      	orrs	r3, r1
     2ec:	6213      	str	r3, [r2, #32]
     2ee:	4a03      	ldr	r2, [pc, #12]	; (2fc <SPI_0_CLOCK_init+0x18>)
     2f0:	4b03      	ldr	r3, [pc, #12]	; (300 <SPI_0_CLOCK_init+0x1c>)
     2f2:	805a      	strh	r2, [r3, #2]
}
     2f4:	4770      	bx	lr
     2f6:	46c0      	nop			; (mov r8, r8)
     2f8:	40000400 	.word	0x40000400
     2fc:	00004014 	.word	0x00004014
     300:	40000c00 	.word	0x40000c00

00000304 <SPI_0_init>:
{
     304:	b510      	push	{r4, lr}
	SPI_0_CLOCK_init();
     306:	4b04      	ldr	r3, [pc, #16]	; (318 <SPI_0_init+0x14>)
     308:	4798      	blx	r3
	spi_m_sync_init(&SPI_0, SERCOM0);
     30a:	4904      	ldr	r1, [pc, #16]	; (31c <SPI_0_init+0x18>)
     30c:	4804      	ldr	r0, [pc, #16]	; (320 <SPI_0_init+0x1c>)
     30e:	4b05      	ldr	r3, [pc, #20]	; (324 <SPI_0_init+0x20>)
     310:	4798      	blx	r3
	SPI_0_PORT_init();
     312:	4b05      	ldr	r3, [pc, #20]	; (328 <SPI_0_init+0x24>)
     314:	4798      	blx	r3
}
     316:	bd10      	pop	{r4, pc}
     318:	000002e5 	.word	0x000002e5
     31c:	42000800 	.word	0x42000800
     320:	20000288 	.word	0x20000288
     324:	000005a9 	.word	0x000005a9
     328:	00000229 	.word	0x00000229

0000032c <USB_0_PORT_init>:

void USB_0_PORT_init(void)
{
     32c:	b5f0      	push	{r4, r5, r6, r7, lr}
     32e:	46c6      	mov	lr, r8
     330:	b500      	push	{lr}
	((Port *)hw)->Group[submodule_index].DIRSET.reg = mask;
     332:	24c0      	movs	r4, #192	; 0xc0
     334:	05e4      	lsls	r4, r4, #23
     336:	2280      	movs	r2, #128	; 0x80
     338:	0452      	lsls	r2, r2, #17
     33a:	60a2      	str	r2, [r4, #8]
	((Port *)hw)->Group[submodule_index].WRCONFIG.reg = data;
     33c:	4b1c      	ldr	r3, [pc, #112]	; (3b0 <USB_0_PORT_init+0x84>)
     33e:	2780      	movs	r7, #128	; 0x80
     340:	05ff      	lsls	r7, r7, #23
     342:	629f      	str	r7, [r3, #40]	; 0x28
     344:	491b      	ldr	r1, [pc, #108]	; (3b4 <USB_0_PORT_init+0x88>)
     346:	6299      	str	r1, [r3, #40]	; 0x28
	((Port *)hw)->Group[submodule_index].OUTCLR.reg = mask;
     348:	6162      	str	r2, [r4, #20]
	((Port *)hw)->Group[submodule_index].PINCFG[index].reg &= ~PORT_PINCFG_PULLEN;
     34a:	2058      	movs	r0, #88	; 0x58
     34c:	5c19      	ldrb	r1, [r3, r0]
     34e:	2204      	movs	r2, #4
     350:	4690      	mov	r8, r2
     352:	4391      	bics	r1, r2
     354:	5419      	strb	r1, [r3, r0]
	tmp = ((Port *)hw)->Group[submodule_index].PINCFG[index].reg;
     356:	5c19      	ldrb	r1, [r3, r0]
	tmp &= ~PORT_PINCFG_PMUXEN;
     358:	2601      	movs	r6, #1
     35a:	43b1      	bics	r1, r6
	tmp |= value << PORT_PINCFG_PMUXEN_Pos;
     35c:	2501      	movs	r5, #1
     35e:	4329      	orrs	r1, r5
     360:	b2c9      	uxtb	r1, r1
	((Port *)hw)->Group[submodule_index].PINCFG[index].reg = tmp;
     362:	5419      	strb	r1, [r3, r0]
	tmp = ((Port *)hw)->Group[submodule_index].PMUX[index].reg;
     364:	381c      	subs	r0, #28
     366:	5c19      	ldrb	r1, [r3, r0]
	tmp &= ~PORT_PMUX_PMUXE_Msk;
     368:	320b      	adds	r2, #11
     36a:	4391      	bics	r1, r2
	tmp |= PORT_PMUX_PMUXE(data);
     36c:	2206      	movs	r2, #6
     36e:	4694      	mov	ip, r2
     370:	4662      	mov	r2, ip
     372:	4311      	orrs	r1, r2
     374:	b2c9      	uxtb	r1, r1
	((Port *)hw)->Group[submodule_index].PMUX[index].reg = tmp;
     376:	5419      	strb	r1, [r3, r0]
	((Port *)hw)->Group[submodule_index].DIRSET.reg = mask;
     378:	2180      	movs	r1, #128	; 0x80
     37a:	0489      	lsls	r1, r1, #18
     37c:	60a1      	str	r1, [r4, #8]
	((Port *)hw)->Group[submodule_index].WRCONFIG.reg = data;
     37e:	629f      	str	r7, [r3, #40]	; 0x28
     380:	4f0d      	ldr	r7, [pc, #52]	; (3b8 <USB_0_PORT_init+0x8c>)
     382:	629f      	str	r7, [r3, #40]	; 0x28
	((Port *)hw)->Group[submodule_index].OUTCLR.reg = mask;
     384:	6161      	str	r1, [r4, #20]
	((Port *)hw)->Group[submodule_index].PINCFG[index].reg &= ~PORT_PINCFG_PULLEN;
     386:	2159      	movs	r1, #89	; 0x59
     388:	5c5c      	ldrb	r4, [r3, r1]
     38a:	4642      	mov	r2, r8
     38c:	4394      	bics	r4, r2
     38e:	545c      	strb	r4, [r3, r1]
	tmp = ((Port *)hw)->Group[submodule_index].PINCFG[index].reg;
     390:	5c5a      	ldrb	r2, [r3, r1]
	tmp &= ~PORT_PINCFG_PMUXEN;
     392:	43b2      	bics	r2, r6
	tmp |= value << PORT_PINCFG_PMUXEN_Pos;
     394:	432a      	orrs	r2, r5
     396:	b2d2      	uxtb	r2, r2
	((Port *)hw)->Group[submodule_index].PINCFG[index].reg = tmp;
     398:	545a      	strb	r2, [r3, r1]
	tmp = ((Port *)hw)->Group[submodule_index].PMUX[index].reg;
     39a:	5c1a      	ldrb	r2, [r3, r0]
	tmp &= ~PORT_PMUX_PMUXO_Msk;
     39c:	394a      	subs	r1, #74	; 0x4a
     39e:	400a      	ands	r2, r1
	tmp |= PORT_PMUX_PMUXO(data);
     3a0:	2160      	movs	r1, #96	; 0x60
     3a2:	430a      	orrs	r2, r1
     3a4:	b2d2      	uxtb	r2, r2
	((Port *)hw)->Group[submodule_index].PMUX[index].reg = tmp;
     3a6:	541a      	strb	r2, [r3, r0]
	                      // <GPIO_PIN_FUNCTION_E"> E
	                      // <GPIO_PIN_FUNCTION_F"> F
	                      // <GPIO_PIN_FUNCTION_G"> G
	                      // <GPIO_PIN_FUNCTION_H"> H
	                      PINMUX_PA25G_USB_DP);
}
     3a8:	bc04      	pop	{r2}
     3aa:	4690      	mov	r8, r2
     3ac:	bdf0      	pop	{r4, r5, r6, r7, pc}
     3ae:	46c0      	nop			; (mov r8, r8)
     3b0:	41004400 	.word	0x41004400
     3b4:	c0000100 	.word	0xc0000100
     3b8:	c0000200 	.word	0xc0000200

000003bc <USB_0_CLOCK_init>:
			PM->APBBMASK.reg |= 1 << peripheral;
     3bc:	4b06      	ldr	r3, [pc, #24]	; (3d8 <USB_0_CLOCK_init+0x1c>)
     3be:	69da      	ldr	r2, [r3, #28]
     3c0:	2120      	movs	r1, #32
     3c2:	430a      	orrs	r2, r1
     3c4:	61da      	str	r2, [r3, #28]
			PM->AHBMASK.reg |= 1 << peripheral;
     3c6:	695a      	ldr	r2, [r3, #20]
     3c8:	3120      	adds	r1, #32
     3ca:	430a      	orrs	r2, r1
     3cc:	615a      	str	r2, [r3, #20]
     3ce:	4a03      	ldr	r2, [pc, #12]	; (3dc <USB_0_CLOCK_init+0x20>)
     3d0:	4b03      	ldr	r3, [pc, #12]	; (3e0 <USB_0_CLOCK_init+0x24>)
     3d2:	805a      	strh	r2, [r3, #2]
{

	_pm_enable_bus_clock(PM_BUS_APBB, USB);
	_pm_enable_bus_clock(PM_BUS_AHB, USB);
	_gclk_enable_channel(USB_GCLK_ID, CONF_GCLK_USB_SRC);
}
     3d4:	4770      	bx	lr
     3d6:	46c0      	nop			; (mov r8, r8)
     3d8:	40000400 	.word	0x40000400
     3dc:	00004006 	.word	0x00004006
     3e0:	40000c00 	.word	0x40000c00

000003e4 <USB_0_init>:

void USB_0_init(void)
{
     3e4:	b510      	push	{r4, lr}
	USB_0_CLOCK_init();
     3e6:	4b03      	ldr	r3, [pc, #12]	; (3f4 <USB_0_init+0x10>)
     3e8:	4798      	blx	r3
	usb_d_init();
     3ea:	4b03      	ldr	r3, [pc, #12]	; (3f8 <USB_0_init+0x14>)
     3ec:	4798      	blx	r3
	USB_0_PORT_init();
     3ee:	4b03      	ldr	r3, [pc, #12]	; (3fc <USB_0_init+0x18>)
     3f0:	4798      	blx	r3
}
     3f2:	bd10      	pop	{r4, pc}
     3f4:	000003bd 	.word	0x000003bd
     3f8:	00000a0d 	.word	0x00000a0d
     3fc:	0000032d 	.word	0x0000032d

00000400 <system_init>:

void system_init(void)
{
     400:	b570      	push	{r4, r5, r6, lr}
 * Currently the following initialization functions are supported:
 *  - System clock initialization
 */
static inline void init_mcu(void)
{
	_init_chip();
     402:	4b51      	ldr	r3, [pc, #324]	; (548 <STACK_SIZE+0x148>)
     404:	4798      	blx	r3
	tmp = ((Port *)hw)->Group[submodule_index].PINCFG[index].reg;
     406:	4b51      	ldr	r3, [pc, #324]	; (54c <STACK_SIZE+0x14c>)
     408:	2040      	movs	r0, #64	; 0x40
     40a:	5c1a      	ldrb	r2, [r3, r0]
	tmp &= ~PORT_PINCFG_PMUXEN;
     40c:	2101      	movs	r1, #1
     40e:	438a      	bics	r2, r1
	((Port *)hw)->Group[submodule_index].PINCFG[index].reg = tmp;
     410:	541a      	strb	r2, [r3, r0]
	tmp = ((Port *)hw)->Group[submodule_index].PINCFG[index].reg;
     412:	3001      	adds	r0, #1
     414:	5c1a      	ldrb	r2, [r3, r0]
	tmp &= ~PORT_PINCFG_PMUXEN;
     416:	438a      	bics	r2, r1
	((Port *)hw)->Group[submodule_index].PINCFG[index].reg = tmp;
     418:	541a      	strb	r2, [r3, r0]
	((Port *)hw)->Group[submodule_index].OUTCLR.reg = mask;
     41a:	22c0      	movs	r2, #192	; 0xc0
     41c:	05d2      	lsls	r2, r2, #23
     41e:	383d      	subs	r0, #61	; 0x3d
     420:	6150      	str	r0, [r2, #20]
	((Port *)hw)->Group[submodule_index].DIRSET.reg = mask;
     422:	6090      	str	r0, [r2, #8]
	((Port *)hw)->Group[submodule_index].WRCONFIG.reg = data;
     424:	484a      	ldr	r0, [pc, #296]	; (550 <STACK_SIZE+0x150>)
     426:	6298      	str	r0, [r3, #40]	; 0x28
     428:	20c0      	movs	r0, #192	; 0xc0
     42a:	0600      	lsls	r0, r0, #24
     42c:	6298      	str	r0, [r3, #40]	; 0x28
	tmp = ((Port *)hw)->Group[submodule_index].PINCFG[index].reg;
     42e:	2542      	movs	r5, #66	; 0x42
     430:	5d5c      	ldrb	r4, [r3, r5]
	tmp &= ~PORT_PINCFG_PMUXEN;
     432:	438c      	bics	r4, r1
	((Port *)hw)->Group[submodule_index].PINCFG[index].reg = tmp;
     434:	555c      	strb	r4, [r3, r5]
	((Port *)hw)->Group[submodule_index].OUTCLR.reg = mask;
     436:	2408      	movs	r4, #8
     438:	6154      	str	r4, [r2, #20]
	((Port *)hw)->Group[submodule_index].DIRSET.reg = mask;
     43a:	6094      	str	r4, [r2, #8]
	((Port *)hw)->Group[submodule_index].WRCONFIG.reg = data;
     43c:	4c45      	ldr	r4, [pc, #276]	; (554 <STACK_SIZE+0x154>)
     43e:	629c      	str	r4, [r3, #40]	; 0x28
     440:	6298      	str	r0, [r3, #40]	; 0x28
	tmp = ((Port *)hw)->Group[submodule_index].PINCFG[index].reg;
     442:	3501      	adds	r5, #1
     444:	5d5c      	ldrb	r4, [r3, r5]
	tmp &= ~PORT_PINCFG_PMUXEN;
     446:	438c      	bics	r4, r1
	((Port *)hw)->Group[submodule_index].PINCFG[index].reg = tmp;
     448:	555c      	strb	r4, [r3, r5]
	((Port *)hw)->Group[submodule_index].OUTCLR.reg = mask;
     44a:	2480      	movs	r4, #128	; 0x80
     44c:	6154      	str	r4, [r2, #20]
	((Port *)hw)->Group[submodule_index].DIRSET.reg = mask;
     44e:	6094      	str	r4, [r2, #8]
	((Port *)hw)->Group[submodule_index].WRCONFIG.reg = data;
     450:	4c41      	ldr	r4, [pc, #260]	; (558 <STACK_SIZE+0x158>)
     452:	629c      	str	r4, [r3, #40]	; 0x28
     454:	6298      	str	r0, [r3, #40]	; 0x28
	tmp = ((Port *)hw)->Group[submodule_index].PINCFG[index].reg;
     456:	3504      	adds	r5, #4
     458:	5d5c      	ldrb	r4, [r3, r5]
	tmp &= ~PORT_PINCFG_PMUXEN;
     45a:	438c      	bics	r4, r1
	((Port *)hw)->Group[submodule_index].PINCFG[index].reg = tmp;
     45c:	555c      	strb	r4, [r3, r5]
	((Port *)hw)->Group[submodule_index].OUTCLR.reg = mask;
     45e:	2480      	movs	r4, #128	; 0x80
     460:	0064      	lsls	r4, r4, #1
     462:	6154      	str	r4, [r2, #20]
	((Port *)hw)->Group[submodule_index].DIRSET.reg = mask;
     464:	6094      	str	r4, [r2, #8]
	((Port *)hw)->Group[submodule_index].WRCONFIG.reg = data;
     466:	4c3d      	ldr	r4, [pc, #244]	; (55c <STACK_SIZE+0x15c>)
     468:	629c      	str	r4, [r3, #40]	; 0x28
     46a:	6298      	str	r0, [r3, #40]	; 0x28
	tmp = ((Port *)hw)->Group[submodule_index].PINCFG[index].reg;
     46c:	3501      	adds	r5, #1
     46e:	5d5c      	ldrb	r4, [r3, r5]
	tmp &= ~PORT_PINCFG_PMUXEN;
     470:	438c      	bics	r4, r1
	((Port *)hw)->Group[submodule_index].PINCFG[index].reg = tmp;
     472:	555c      	strb	r4, [r3, r5]
	((Port *)hw)->Group[submodule_index].OUTCLR.reg = mask;
     474:	2480      	movs	r4, #128	; 0x80
     476:	00a4      	lsls	r4, r4, #2
     478:	6154      	str	r4, [r2, #20]
	((Port *)hw)->Group[submodule_index].DIRSET.reg = mask;
     47a:	6094      	str	r4, [r2, #8]
	((Port *)hw)->Group[submodule_index].WRCONFIG.reg = data;
     47c:	4c38      	ldr	r4, [pc, #224]	; (560 <STACK_SIZE+0x160>)
     47e:	629c      	str	r4, [r3, #40]	; 0x28
     480:	6298      	str	r0, [r3, #40]	; 0x28
	tmp = ((Port *)hw)->Group[submodule_index].PINCFG[index].reg;
     482:	3501      	adds	r5, #1
     484:	5d5c      	ldrb	r4, [r3, r5]
	tmp &= ~PORT_PINCFG_PMUXEN;
     486:	438c      	bics	r4, r1
	((Port *)hw)->Group[submodule_index].PINCFG[index].reg = tmp;
     488:	555c      	strb	r4, [r3, r5]
	((Port *)hw)->Group[submodule_index].OUTCLR.reg = mask;
     48a:	2480      	movs	r4, #128	; 0x80
     48c:	00e4      	lsls	r4, r4, #3
     48e:	6154      	str	r4, [r2, #20]
	((Port *)hw)->Group[submodule_index].DIRSET.reg = mask;
     490:	6094      	str	r4, [r2, #8]
	((Port *)hw)->Group[submodule_index].WRCONFIG.reg = data;
     492:	4c34      	ldr	r4, [pc, #208]	; (564 <STACK_SIZE+0x164>)
     494:	629c      	str	r4, [r3, #40]	; 0x28
     496:	6298      	str	r0, [r3, #40]	; 0x28
	tmp = ((Port *)hw)->Group[submodule_index].PINCFG[index].reg;
     498:	3501      	adds	r5, #1
     49a:	5d5c      	ldrb	r4, [r3, r5]
	tmp &= ~PORT_PINCFG_PMUXEN;
     49c:	438c      	bics	r4, r1
	((Port *)hw)->Group[submodule_index].PINCFG[index].reg = tmp;
     49e:	555c      	strb	r4, [r3, r5]
	((Port *)hw)->Group[submodule_index].OUTCLR.reg = mask;
     4a0:	2480      	movs	r4, #128	; 0x80
     4a2:	0124      	lsls	r4, r4, #4
     4a4:	6154      	str	r4, [r2, #20]
	((Port *)hw)->Group[submodule_index].DIRSET.reg = mask;
     4a6:	6094      	str	r4, [r2, #8]
	((Port *)hw)->Group[submodule_index].WRCONFIG.reg = data;
     4a8:	4c2f      	ldr	r4, [pc, #188]	; (568 <STACK_SIZE+0x168>)
     4aa:	629c      	str	r4, [r3, #40]	; 0x28
     4ac:	6298      	str	r0, [r3, #40]	; 0x28
	tmp = ((Port *)hw)->Group[submodule_index].PINCFG[index].reg;
     4ae:	244b      	movs	r4, #75	; 0x4b
     4b0:	5d18      	ldrb	r0, [r3, r4]
	tmp &= ~PORT_PINCFG_PMUXEN;
     4b2:	4388      	bics	r0, r1
	((Port *)hw)->Group[submodule_index].PINCFG[index].reg = tmp;
     4b4:	5518      	strb	r0, [r3, r4]
	tmp = ((Port *)hw)->Group[submodule_index].PINCFG[index].reg;
     4b6:	3403      	adds	r4, #3
     4b8:	5d18      	ldrb	r0, [r3, r4]
	tmp &= ~PORT_PINCFG_PMUXEN;
     4ba:	4388      	bics	r0, r1
	((Port *)hw)->Group[submodule_index].PINCFG[index].reg = tmp;
     4bc:	5518      	strb	r0, [r3, r4]
	tmp = ((Port *)hw)->Group[submodule_index].PINCFG[index].reg;
     4be:	3401      	adds	r4, #1
     4c0:	5d18      	ldrb	r0, [r3, r4]
	tmp &= ~PORT_PINCFG_PMUXEN;
     4c2:	4388      	bics	r0, r1
	((Port *)hw)->Group[submodule_index].PINCFG[index].reg = tmp;
     4c4:	5518      	strb	r0, [r3, r4]
	((Port *)hw)->Group[submodule_index].OUTCLR.reg = mask;
     4c6:	2080      	movs	r0, #128	; 0x80
     4c8:	0240      	lsls	r0, r0, #9
     4ca:	6150      	str	r0, [r2, #20]
	((Port *)hw)->Group[submodule_index].DIRSET.reg = mask;
     4cc:	6090      	str	r0, [r2, #8]
	((Port *)hw)->Group[submodule_index].WRCONFIG.reg = data;
     4ce:	2080      	movs	r0, #128	; 0x80
     4d0:	05c0      	lsls	r0, r0, #23
     4d2:	6298      	str	r0, [r3, #40]	; 0x28
     4d4:	4c25      	ldr	r4, [pc, #148]	; (56c <STACK_SIZE+0x16c>)
     4d6:	629c      	str	r4, [r3, #40]	; 0x28
	tmp = ((Port *)hw)->Group[submodule_index].PINCFG[index].reg;
     4d8:	3506      	adds	r5, #6
     4da:	5d5c      	ldrb	r4, [r3, r5]
	tmp &= ~PORT_PINCFG_PMUXEN;
     4dc:	438c      	bics	r4, r1
	((Port *)hw)->Group[submodule_index].PINCFG[index].reg = tmp;
     4de:	555c      	strb	r4, [r3, r5]
	((Port *)hw)->Group[submodule_index].OUTCLR.reg = mask;
     4e0:	2480      	movs	r4, #128	; 0x80
     4e2:	02a4      	lsls	r4, r4, #10
     4e4:	6154      	str	r4, [r2, #20]
	((Port *)hw)->Group[submodule_index].DIRSET.reg = mask;
     4e6:	6094      	str	r4, [r2, #8]
	((Port *)hw)->Group[submodule_index].WRCONFIG.reg = data;
     4e8:	6298      	str	r0, [r3, #40]	; 0x28
     4ea:	4c21      	ldr	r4, [pc, #132]	; (570 <STACK_SIZE+0x170>)
     4ec:	629c      	str	r4, [r3, #40]	; 0x28
	tmp = ((Port *)hw)->Group[submodule_index].PINCFG[index].reg;
     4ee:	3501      	adds	r5, #1
     4f0:	5d5c      	ldrb	r4, [r3, r5]
	tmp &= ~PORT_PINCFG_PMUXEN;
     4f2:	438c      	bics	r4, r1
	((Port *)hw)->Group[submodule_index].PINCFG[index].reg = tmp;
     4f4:	555c      	strb	r4, [r3, r5]
	((Port *)hw)->Group[submodule_index].OUTCLR.reg = mask;
     4f6:	2480      	movs	r4, #128	; 0x80
     4f8:	02e4      	lsls	r4, r4, #11
     4fa:	6154      	str	r4, [r2, #20]
	((Port *)hw)->Group[submodule_index].DIRSET.reg = mask;
     4fc:	6094      	str	r4, [r2, #8]
	((Port *)hw)->Group[submodule_index].WRCONFIG.reg = data;
     4fe:	6298      	str	r0, [r3, #40]	; 0x28
     500:	4c1c      	ldr	r4, [pc, #112]	; (574 <STACK_SIZE+0x174>)
     502:	629c      	str	r4, [r3, #40]	; 0x28
	tmp = ((Port *)hw)->Group[submodule_index].PINCFG[index].reg;
     504:	3501      	adds	r5, #1
     506:	5d5c      	ldrb	r4, [r3, r5]
	tmp &= ~PORT_PINCFG_PMUXEN;
     508:	438c      	bics	r4, r1
	((Port *)hw)->Group[submodule_index].PINCFG[index].reg = tmp;
     50a:	555c      	strb	r4, [r3, r5]
	((Port *)hw)->Group[submodule_index].OUTCLR.reg = mask;
     50c:	2480      	movs	r4, #128	; 0x80
     50e:	0324      	lsls	r4, r4, #12
     510:	6154      	str	r4, [r2, #20]
	((Port *)hw)->Group[submodule_index].DIRSET.reg = mask;
     512:	6094      	str	r4, [r2, #8]
	((Port *)hw)->Group[submodule_index].WRCONFIG.reg = data;
     514:	6298      	str	r0, [r3, #40]	; 0x28
     516:	4c18      	ldr	r4, [pc, #96]	; (578 <STACK_SIZE+0x178>)
     518:	629c      	str	r4, [r3, #40]	; 0x28
	tmp = ((Port *)hw)->Group[submodule_index].PINCFG[index].reg;
     51a:	3501      	adds	r5, #1
     51c:	5d5c      	ldrb	r4, [r3, r5]
	tmp &= ~PORT_PINCFG_PMUXEN;
     51e:	438c      	bics	r4, r1
	((Port *)hw)->Group[submodule_index].PINCFG[index].reg = tmp;
     520:	555c      	strb	r4, [r3, r5]
	((Port *)hw)->Group[submodule_index].OUTCLR.reg = mask;
     522:	2480      	movs	r4, #128	; 0x80
     524:	03e4      	lsls	r4, r4, #15
     526:	6154      	str	r4, [r2, #20]
	((Port *)hw)->Group[submodule_index].DIRSET.reg = mask;
     528:	6094      	str	r4, [r2, #8]
	((Port *)hw)->Group[submodule_index].WRCONFIG.reg = data;
     52a:	6298      	str	r0, [r3, #40]	; 0x28
     52c:	4a13      	ldr	r2, [pc, #76]	; (57c <STACK_SIZE+0x17c>)
     52e:	629a      	str	r2, [r3, #40]	; 0x28
	tmp = ((Port *)hw)->Group[submodule_index].PINCFG[index].reg;
     530:	2056      	movs	r0, #86	; 0x56
     532:	5c1a      	ldrb	r2, [r3, r0]
	tmp &= ~PORT_PINCFG_PMUXEN;
     534:	438a      	bics	r2, r1
	((Port *)hw)->Group[submodule_index].PINCFG[index].reg = tmp;
     536:	541a      	strb	r2, [r3, r0]
	// Set pin direction to output
	gpio_set_pin_direction(VSYNC, GPIO_DIRECTION_OUT);

	gpio_set_pin_function(VSYNC, GPIO_PIN_FUNCTION_OFF);

	SPI_0_init();
     538:	4b11      	ldr	r3, [pc, #68]	; (580 <STACK_SIZE+0x180>)
     53a:	4798      	blx	r3

	TIMER_0_init();
     53c:	4b11      	ldr	r3, [pc, #68]	; (584 <STACK_SIZE+0x184>)
     53e:	4798      	blx	r3

	USB_0_init();
     540:	4b11      	ldr	r3, [pc, #68]	; (588 <STACK_SIZE+0x188>)
     542:	4798      	blx	r3
}
     544:	bd70      	pop	{r4, r5, r6, pc}
     546:	46c0      	nop			; (mov r8, r8)
     548:	00000ae1 	.word	0x00000ae1
     54c:	41004400 	.word	0x41004400
     550:	40000004 	.word	0x40000004
     554:	40000008 	.word	0x40000008
     558:	40000080 	.word	0x40000080
     55c:	40000100 	.word	0x40000100
     560:	40000200 	.word	0x40000200
     564:	40000400 	.word	0x40000400
     568:	40000800 	.word	0x40000800
     56c:	c0000001 	.word	0xc0000001
     570:	c0000002 	.word	0xc0000002
     574:	c0000004 	.word	0xc0000004
     578:	c0000008 	.word	0xc0000008
     57c:	c0000040 	.word	0xc0000040
     580:	00000305 	.word	0x00000305
     584:	000001e9 	.word	0x000001e9
     588:	000003e5 	.word	0x000003e5

0000058c <atomic_enter_critical>:
 */
__STATIC_FORCEINLINE uint32_t __get_PRIMASK(void)
{
  uint32_t result;

  __ASM volatile ("MRS %0, primask" : "=r" (result) :: "memory");
     58c:	f3ef 8310 	mrs	r3, PRIMASK
/**
 * \brief Disable interrupts, enter critical section
 */
void atomic_enter_critical(hal_atomic_t volatile *atomic)
{
	*atomic = __get_PRIMASK();
     590:	6003      	str	r3, [r0, #0]
  __ASM volatile ("cpsid i" : : : "memory");
     592:	b672      	cpsid	i
  \details Ensures the apparent order of the explicit memory operations before
           and after the instruction, without ensuring their completion.
 */
__STATIC_FORCEINLINE void __DMB(void)
{
  __ASM volatile ("dmb 0xF":::"memory");
     594:	f3bf 8f5f 	dmb	sy
	__disable_irq();
	__DMB();
}
     598:	4770      	bx	lr

0000059a <atomic_leave_critical>:
     59a:	f3bf 8f5f 	dmb	sy
 * \brief Exit atomic section
 */
void atomic_leave_critical(hal_atomic_t volatile *atomic)
{
	__DMB();
	__set_PRIMASK(*atomic);
     59e:	6803      	ldr	r3, [r0, #0]
  __ASM volatile ("MSR primask, %0" : : "r" (priMask) : "memory");
     5a0:	f383 8810 	msr	PRIMASK, r3
}
     5a4:	4770      	bx	lr
	...

000005a8 <spi_m_sync_init>:
	ASSERT(spi);
	spi->func = (struct _spi_m_sync_hpl_interface *)func;
}

int32_t spi_m_sync_init(struct spi_m_sync_descriptor *spi, void *const hw)
{
     5a8:	b570      	push	{r4, r5, r6, lr}
     5aa:	0004      	movs	r4, r0
     5ac:	000d      	movs	r5, r1
	int32_t rc = 0;
	ASSERT(spi && hw);
     5ae:	2800      	cmp	r0, #0
     5b0:	d017      	beq.n	5e2 <spi_m_sync_init+0x3a>
     5b2:	2900      	cmp	r1, #0
     5b4:	d013      	beq.n	5de <spi_m_sync_init+0x36>
     5b6:	2001      	movs	r0, #1
     5b8:	2240      	movs	r2, #64	; 0x40
     5ba:	490b      	ldr	r1, [pc, #44]	; (5e8 <spi_m_sync_init+0x40>)
     5bc:	4b0b      	ldr	r3, [pc, #44]	; (5ec <spi_m_sync_init+0x44>)
     5be:	4798      	blx	r3
	spi->dev.prvt = (void *)hw;
     5c0:	6065      	str	r5, [r4, #4]
	rc            = _spi_m_sync_init(&spi->dev, hw);
     5c2:	1d20      	adds	r0, r4, #4
     5c4:	0029      	movs	r1, r5
     5c6:	4b0a      	ldr	r3, [pc, #40]	; (5f0 <spi_m_sync_init+0x48>)
     5c8:	4798      	blx	r3

	if (rc < 0) {
     5ca:	2800      	cmp	r0, #0
     5cc:	db06      	blt.n	5dc <spi_m_sync_init+0x34>
		return rc;
	}

	spi->flags    = SPI_DEACTIVATE_NEXT;
     5ce:	4b09      	ldr	r3, [pc, #36]	; (5f4 <spi_m_sync_init+0x4c>)
     5d0:	82a3      	strh	r3, [r4, #20]
	spi->io.read  = _spi_m_sync_io_read;
     5d2:	4b09      	ldr	r3, [pc, #36]	; (5f8 <spi_m_sync_init+0x50>)
     5d4:	6123      	str	r3, [r4, #16]
	spi->io.write = _spi_m_sync_io_write;
     5d6:	4b09      	ldr	r3, [pc, #36]	; (5fc <spi_m_sync_init+0x54>)
     5d8:	60e3      	str	r3, [r4, #12]

	return ERR_NONE;
     5da:	2000      	movs	r0, #0
}
     5dc:	bd70      	pop	{r4, r5, r6, pc}
	ASSERT(spi && hw);
     5de:	2000      	movs	r0, #0
     5e0:	e7ea      	b.n	5b8 <spi_m_sync_init+0x10>
     5e2:	2000      	movs	r0, #0
     5e4:	e7e8      	b.n	5b8 <spi_m_sync_init+0x10>
     5e6:	46c0      	nop			; (mov r8, r8)
     5e8:	00001e40 	.word	0x00001e40
     5ec:	00000a79 	.word	0x00000a79
     5f0:	00000c31 	.word	0x00000c31
     5f4:	ffff8000 	.word	0xffff8000
     5f8:	00000685 	.word	0x00000685
     5fc:	00000649 	.word	0x00000649

00000600 <spi_m_sync_transfer>:

	return spi_m_sync_transfer(spi, &xfer);
}

int32_t spi_m_sync_transfer(struct spi_m_sync_descriptor *spi, const struct spi_xfer *p_xfer)
{
     600:	b530      	push	{r4, r5, lr}
     602:	b087      	sub	sp, #28
     604:	0004      	movs	r4, r0
     606:	000d      	movs	r5, r1
	struct spi_msg msg;

	ASSERT(spi && p_xfer);
     608:	2800      	cmp	r0, #0
     60a:	d015      	beq.n	638 <spi_m_sync_transfer+0x38>
     60c:	2900      	cmp	r1, #0
     60e:	d011      	beq.n	634 <spi_m_sync_transfer+0x34>
     610:	2001      	movs	r0, #1
     612:	22b3      	movs	r2, #179	; 0xb3
     614:	4909      	ldr	r1, [pc, #36]	; (63c <spi_m_sync_transfer+0x3c>)
     616:	4b0a      	ldr	r3, [pc, #40]	; (640 <spi_m_sync_transfer+0x40>)
     618:	4798      	blx	r3

	msg.txbuf = p_xfer->txbuf;
     61a:	682b      	ldr	r3, [r5, #0]
     61c:	9303      	str	r3, [sp, #12]
	msg.rxbuf = p_xfer->rxbuf;
     61e:	686b      	ldr	r3, [r5, #4]
     620:	9304      	str	r3, [sp, #16]
	msg.size  = p_xfer->size;
     622:	68ab      	ldr	r3, [r5, #8]
     624:	9301      	str	r3, [sp, #4]
     626:	9305      	str	r3, [sp, #20]
	return _spi_m_sync_trans(&spi->dev, &msg);
     628:	1d20      	adds	r0, r4, #4
     62a:	a903      	add	r1, sp, #12
     62c:	4b05      	ldr	r3, [pc, #20]	; (644 <spi_m_sync_transfer+0x44>)
     62e:	4798      	blx	r3
}
     630:	b007      	add	sp, #28
     632:	bd30      	pop	{r4, r5, pc}
	ASSERT(spi && p_xfer);
     634:	2000      	movs	r0, #0
     636:	e7ec      	b.n	612 <spi_m_sync_transfer+0x12>
     638:	2000      	movs	r0, #0
     63a:	e7ea      	b.n	612 <spi_m_sync_transfer+0x12>
     63c:	00001e40 	.word	0x00001e40
     640:	00000a79 	.word	0x00000a79
     644:	00000e2d 	.word	0x00000e2d

00000648 <_spi_m_sync_io_write>:
{
     648:	b570      	push	{r4, r5, r6, lr}
     64a:	b084      	sub	sp, #16
     64c:	0004      	movs	r4, r0
     64e:	000e      	movs	r6, r1
     650:	0015      	movs	r5, r2
	ASSERT(io);
     652:	1e43      	subs	r3, r0, #1
     654:	4198      	sbcs	r0, r3
     656:	b2c0      	uxtb	r0, r0
     658:	22a3      	movs	r2, #163	; 0xa3
     65a:	4907      	ldr	r1, [pc, #28]	; (678 <_spi_m_sync_io_write+0x30>)
     65c:	4b07      	ldr	r3, [pc, #28]	; (67c <_spi_m_sync_io_write+0x34>)
     65e:	4798      	blx	r3
	struct spi_m_sync_descriptor *spi = CONTAINER_OF(io, struct spi_m_sync_descriptor, io);
     660:	0020      	movs	r0, r4
     662:	380c      	subs	r0, #12
	xfer.rxbuf = 0;
     664:	2300      	movs	r3, #0
     666:	9302      	str	r3, [sp, #8]
	xfer.txbuf = (uint8_t *)buf;
     668:	9601      	str	r6, [sp, #4]
	xfer.size  = length;
     66a:	9503      	str	r5, [sp, #12]
	return spi_m_sync_transfer(spi, &xfer);
     66c:	a901      	add	r1, sp, #4
     66e:	4b04      	ldr	r3, [pc, #16]	; (680 <_spi_m_sync_io_write+0x38>)
     670:	4798      	blx	r3
}
     672:	b004      	add	sp, #16
     674:	bd70      	pop	{r4, r5, r6, pc}
     676:	46c0      	nop			; (mov r8, r8)
     678:	00001e40 	.word	0x00001e40
     67c:	00000a79 	.word	0x00000a79
     680:	00000601 	.word	0x00000601

00000684 <_spi_m_sync_io_read>:
{
     684:	b570      	push	{r4, r5, r6, lr}
     686:	b084      	sub	sp, #16
     688:	0004      	movs	r4, r0
     68a:	000e      	movs	r6, r1
     68c:	0015      	movs	r5, r2
	ASSERT(io);
     68e:	1e43      	subs	r3, r0, #1
     690:	4198      	sbcs	r0, r3
     692:	b2c0      	uxtb	r0, r0
     694:	2287      	movs	r2, #135	; 0x87
     696:	4907      	ldr	r1, [pc, #28]	; (6b4 <_spi_m_sync_io_read+0x30>)
     698:	4b07      	ldr	r3, [pc, #28]	; (6b8 <_spi_m_sync_io_read+0x34>)
     69a:	4798      	blx	r3
	struct spi_m_sync_descriptor *spi = CONTAINER_OF(io, struct spi_m_sync_descriptor, io);
     69c:	0020      	movs	r0, r4
     69e:	380c      	subs	r0, #12
	xfer.rxbuf = buf;
     6a0:	9602      	str	r6, [sp, #8]
	xfer.txbuf = 0;
     6a2:	2300      	movs	r3, #0
     6a4:	9301      	str	r3, [sp, #4]
	xfer.size  = length;
     6a6:	9503      	str	r5, [sp, #12]
	return spi_m_sync_transfer(spi, &xfer);
     6a8:	a901      	add	r1, sp, #4
     6aa:	4b04      	ldr	r3, [pc, #16]	; (6bc <_spi_m_sync_io_read+0x38>)
     6ac:	4798      	blx	r3
}
     6ae:	b004      	add	sp, #16
     6b0:	bd70      	pop	{r4, r5, r6, pc}
     6b2:	46c0      	nop			; (mov r8, r8)
     6b4:	00001e40 	.word	0x00001e40
     6b8:	00000a79 	.word	0x00000a79
     6bc:	00000601 	.word	0x00000601

000006c0 <timer_add_timer_task>:
 * \param[in] head The pointer to the head of timer task list
 * \param[in] task The pointer to task to add
 * \param[in] time Current timer time
 */
static void timer_add_timer_task(struct list_descriptor *list, struct timer_task *const new_task, const uint32_t time)
{
     6c0:	b5f8      	push	{r3, r4, r5, r6, r7, lr}
 * \return A pointer to the head of the given list or NULL if the list is
 * empty
 */
static inline void *list_get_head(const struct list_descriptor *const list)
{
	return (void *)list->head;
     6c2:	6806      	ldr	r6, [r0, #0]
	struct timer_task *it, *prev = NULL, *head = (struct timer_task *)list_get_head(list);

	if (!head) {
     6c4:	2e00      	cmp	r6, #0
     6c6:	d002      	beq.n	6ce <timer_add_timer_task+0xe>
     6c8:	0033      	movs	r3, r6
     6ca:	2500      	movs	r5, #0
     6cc:	e00c      	b.n	6e8 <timer_add_timer_task+0x28>
		list_insert_as_head(list, new_task);
     6ce:	4b10      	ldr	r3, [pc, #64]	; (710 <timer_add_timer_task+0x50>)
     6d0:	4798      	blx	r3
		return;
     6d2:	e018      	b.n	706 <timer_add_timer_task+0x46>
		uint32_t time_left;

		if (it->time_label <= time) {
			time_left = it->interval - (time - it->time_label);
		} else {
			time_left = it->interval - (0xFFFFFFFF - it->time_label) - time;
     6d4:	689f      	ldr	r7, [r3, #8]
     6d6:	46bc      	mov	ip, r7
     6d8:	4464      	add	r4, ip
     6da:	1aa4      	subs	r4, r4, r2
     6dc:	3401      	adds	r4, #1
		}
		if (time_left >= new_task->interval)
     6de:	688f      	ldr	r7, [r1, #8]
     6e0:	42bc      	cmp	r4, r7
     6e2:	d20b      	bcs.n	6fc <timer_add_timer_task+0x3c>
			break;
		prev = it;
     6e4:	001d      	movs	r5, r3
	for (it = head; it; it = (struct timer_task *)list_get_next_element(it)) {
     6e6:	681b      	ldr	r3, [r3, #0]
     6e8:	2b00      	cmp	r3, #0
     6ea:	d007      	beq.n	6fc <timer_add_timer_task+0x3c>
		if (it->time_label <= time) {
     6ec:	685c      	ldr	r4, [r3, #4]
     6ee:	4294      	cmp	r4, r2
     6f0:	d8f0      	bhi.n	6d4 <timer_add_timer_task+0x14>
			time_left = it->interval - (time - it->time_label);
     6f2:	1aa4      	subs	r4, r4, r2
     6f4:	689f      	ldr	r7, [r3, #8]
     6f6:	46bc      	mov	ip, r7
     6f8:	4464      	add	r4, ip
     6fa:	e7f0      	b.n	6de <timer_add_timer_task+0x1e>
	}

	if (it == head) {
     6fc:	42b3      	cmp	r3, r6
     6fe:	d003      	beq.n	708 <timer_add_timer_task+0x48>
		list_insert_as_head(list, new_task);
	} else {
		list_insert_after(prev, new_task);
     700:	0028      	movs	r0, r5
     702:	4b04      	ldr	r3, [pc, #16]	; (714 <timer_add_timer_task+0x54>)
     704:	4798      	blx	r3
	}
}
     706:	bdf8      	pop	{r3, r4, r5, r6, r7, pc}
		list_insert_as_head(list, new_task);
     708:	4b01      	ldr	r3, [pc, #4]	; (710 <timer_add_timer_task+0x50>)
     70a:	4798      	blx	r3
     70c:	e7fb      	b.n	706 <timer_add_timer_task+0x46>
     70e:	46c0      	nop			; (mov r8, r8)
     710:	00000a99 	.word	0x00000a99
     714:	00000ac5 	.word	0x00000ac5

00000718 <timer_process_counted>:

/**
 * \internal Process interrupts
 */
static void timer_process_counted(struct _timer_device *device)
{
     718:	b5f8      	push	{r3, r4, r5, r6, r7, lr}
     71a:	0005      	movs	r5, r0
     71c:	6944      	ldr	r4, [r0, #20]
	struct timer_descriptor *timer = CONTAINER_OF(device, struct timer_descriptor, device);
	struct timer_task *      it    = (struct timer_task *)list_get_head(&timer->tasks);
	uint32_t                 time  = ++timer->time;
     71e:	6903      	ldr	r3, [r0, #16]
     720:	1c5e      	adds	r6, r3, #1
     722:	6106      	str	r6, [r0, #16]

	if ((timer->flags & TIMER_FLAG_QUEUE_IS_TAKEN) || (timer->flags & TIMER_FLAG_INTERRUPT_TRIGERRED)) {
     724:	7e03      	ldrb	r3, [r0, #24]
     726:	07db      	lsls	r3, r3, #31
     728:	d402      	bmi.n	730 <timer_process_counted+0x18>
     72a:	7e03      	ldrb	r3, [r0, #24]
     72c:	079b      	lsls	r3, r3, #30
     72e:	d50a      	bpl.n	746 <timer_process_counted+0x2e>
		timer->flags |= TIMER_FLAG_INTERRUPT_TRIGERRED;
     730:	7e2b      	ldrb	r3, [r5, #24]
     732:	2202      	movs	r2, #2
     734:	4313      	orrs	r3, r2
     736:	b2db      	uxtb	r3, r3
     738:	762b      	strb	r3, [r5, #24]
		}
		it = (struct timer_task *)list_get_head(&timer->tasks);

		tmp->cb(tmp);
	}
}
     73a:	bdf8      	pop	{r3, r4, r5, r6, r7, pc}
     73c:	696f      	ldr	r7, [r5, #20]
		tmp->cb(tmp);
     73e:	68e3      	ldr	r3, [r4, #12]
     740:	0020      	movs	r0, r4
     742:	4798      	blx	r3
		it = (struct timer_task *)list_get_head(&timer->tasks);
     744:	003c      	movs	r4, r7
	while (it && ((time - it->time_label) >= it->interval)) {
     746:	2c00      	cmp	r4, #0
     748:	d0f7      	beq.n	73a <timer_process_counted+0x22>
     74a:	6863      	ldr	r3, [r4, #4]
     74c:	1af3      	subs	r3, r6, r3
     74e:	68a2      	ldr	r2, [r4, #8]
     750:	4293      	cmp	r3, r2
     752:	d3f2      	bcc.n	73a <timer_process_counted+0x22>
		list_remove_head(&timer->tasks);
     754:	002f      	movs	r7, r5
     756:	3714      	adds	r7, #20
     758:	0038      	movs	r0, r7
     75a:	4b06      	ldr	r3, [pc, #24]	; (774 <timer_process_counted+0x5c>)
     75c:	4798      	blx	r3
		if (TIMER_TASK_REPEAT == tmp->mode) {
     75e:	7c23      	ldrb	r3, [r4, #16]
     760:	2b01      	cmp	r3, #1
     762:	d1eb      	bne.n	73c <timer_process_counted+0x24>
			tmp->time_label = time;
     764:	6066      	str	r6, [r4, #4]
			timer_add_timer_task(&timer->tasks, tmp, time);
     766:	0032      	movs	r2, r6
     768:	0021      	movs	r1, r4
     76a:	0038      	movs	r0, r7
     76c:	4b02      	ldr	r3, [pc, #8]	; (778 <timer_process_counted+0x60>)
     76e:	4798      	blx	r3
     770:	e7e4      	b.n	73c <timer_process_counted+0x24>
     772:	46c0      	nop			; (mov r8, r8)
     774:	00000acd 	.word	0x00000acd
     778:	000006c1 	.word	0x000006c1

0000077c <timer_init>:
{
     77c:	b570      	push	{r4, r5, r6, lr}
     77e:	0004      	movs	r4, r0
     780:	000d      	movs	r5, r1
	ASSERT(descr && hw);
     782:	2800      	cmp	r0, #0
     784:	d012      	beq.n	7ac <timer_init+0x30>
     786:	2900      	cmp	r1, #0
     788:	d00e      	beq.n	7a8 <timer_init+0x2c>
     78a:	2001      	movs	r0, #1
     78c:	223b      	movs	r2, #59	; 0x3b
     78e:	4908      	ldr	r1, [pc, #32]	; (7b0 <timer_init+0x34>)
     790:	4b08      	ldr	r3, [pc, #32]	; (7b4 <timer_init+0x38>)
     792:	4798      	blx	r3
	_timer_init(&descr->device, hw);
     794:	0029      	movs	r1, r5
     796:	0020      	movs	r0, r4
     798:	4b07      	ldr	r3, [pc, #28]	; (7b8 <timer_init+0x3c>)
     79a:	4798      	blx	r3
	descr->time                           = 0;
     79c:	2300      	movs	r3, #0
     79e:	6123      	str	r3, [r4, #16]
	descr->device.timer_cb.period_expired = timer_process_counted;
     7a0:	4b06      	ldr	r3, [pc, #24]	; (7bc <timer_init+0x40>)
     7a2:	6023      	str	r3, [r4, #0]
}
     7a4:	2000      	movs	r0, #0
     7a6:	bd70      	pop	{r4, r5, r6, pc}
	ASSERT(descr && hw);
     7a8:	2000      	movs	r0, #0
     7aa:	e7ef      	b.n	78c <timer_init+0x10>
     7ac:	2000      	movs	r0, #0
     7ae:	e7ed      	b.n	78c <timer_init+0x10>
     7b0:	00001e5c 	.word	0x00001e5c
     7b4:	00000a79 	.word	0x00000a79
     7b8:	00000bad 	.word	0x00000bad
     7bc:	00000719 	.word	0x00000719

000007c0 <_usb_d_find_ep>:
 * \return Index of endpoint descriptor.
 * \retval >=0 The index.
 * \retval <0 Not found (endpoint is not initialized).
 */
static int8_t _usb_d_find_ep(const uint8_t ep)
{
     7c0:	b510      	push	{r4, lr}
     7c2:	0001      	movs	r1, r0
	int8_t i;
	for (i = 0; i < CONF_USB_D_NUM_EP_SP; i++) {
     7c4:	2000      	movs	r0, #0
     7c6:	e001      	b.n	7cc <_usb_d_find_ep+0xc>
     7c8:	3001      	adds	r0, #1
     7ca:	b240      	sxtb	r0, r0
     7cc:	2803      	cmp	r0, #3
     7ce:	dc0f      	bgt.n	7f0 <_usb_d_find_ep+0x30>
		if (usb_d_inst.ep[i].xfer.hdr.ep == ep) {
     7d0:	0142      	lsls	r2, r0, #5
     7d2:	4b09      	ldr	r3, [pc, #36]	; (7f8 <_usb_d_find_ep+0x38>)
     7d4:	189b      	adds	r3, r3, r2
     7d6:	785a      	ldrb	r2, [r3, #1]
     7d8:	428a      	cmp	r2, r1
     7da:	d00b      	beq.n	7f4 <_usb_d_find_ep+0x34>
			return i;
		}
		if (usb_d_inst.ep[i].xfer.hdr.type == USB_EP_XTYPE_CTRL
     7dc:	0143      	lsls	r3, r0, #5
     7de:	4c06      	ldr	r4, [pc, #24]	; (7f8 <_usb_d_find_ep+0x38>)
     7e0:	5d1b      	ldrb	r3, [r3, r4]
     7e2:	2b00      	cmp	r3, #0
     7e4:	d1f0      	bne.n	7c8 <_usb_d_find_ep+0x8>
		    && (ep & USB_EP_N_MASK) == usb_d_inst.ep[i].xfer.hdr.ep) {
     7e6:	330f      	adds	r3, #15
     7e8:	400b      	ands	r3, r1
     7ea:	4293      	cmp	r3, r2
     7ec:	d1ec      	bne.n	7c8 <_usb_d_find_ep+0x8>
     7ee:	e001      	b.n	7f4 <_usb_d_find_ep+0x34>
			return i;
		}
	}
	return -1;
     7f0:	2001      	movs	r0, #1
     7f2:	4240      	negs	r0, r0
}
     7f4:	bd10      	pop	{r4, pc}
     7f6:	46c0      	nop			; (mov r8, r8)
     7f8:	2000001c 	.word	0x2000001c

000007fc <usb_d_dummy_cb_false>:
{
	(void)unused0;
	(void)unused1;
	(void)unused2;
	return false;
}
     7fc:	2000      	movs	r0, #0
     7fe:	4770      	bx	lr

00000800 <usb_d_cb_trans_more>:
 * \brief Callback invoked when request more data
 * \param[in] ep Endpoint number with transfer direction on bit 8.
 * \param[in] transfered Number of bytes transfered.
 */
static bool usb_d_cb_trans_more(const uint8_t ep, const uint32_t transfered)
{
     800:	b570      	push	{r4, r5, r6, lr}
     802:	0004      	movs	r4, r0
     804:	000d      	movs	r5, r1
	int8_t           ep_index = _usb_d_find_ep(ep);
     806:	4b08      	ldr	r3, [pc, #32]	; (828 <usb_d_cb_trans_more+0x28>)
     808:	4798      	blx	r3
	struct usb_d_ep *ept      = &usb_d_inst.ep[ep_index];
	if (ept->xfer.hdr.state == USB_EP_S_X_DATA) {
     80a:	0142      	lsls	r2, r0, #5
     80c:	4b07      	ldr	r3, [pc, #28]	; (82c <usb_d_cb_trans_more+0x2c>)
     80e:	189b      	adds	r3, r3, r2
     810:	789b      	ldrb	r3, [r3, #2]
     812:	2b03      	cmp	r3, #3
     814:	d001      	beq.n	81a <usb_d_cb_trans_more+0x1a>
		return ept->callbacks.more(ep, transfered);
	}
	return false;
     816:	2000      	movs	r0, #0
}
     818:	bd70      	pop	{r4, r5, r6, pc}
		return ept->callbacks.more(ep, transfered);
     81a:	4b04      	ldr	r3, [pc, #16]	; (82c <usb_d_cb_trans_more+0x2c>)
     81c:	1898      	adds	r0, r3, r2
     81e:	6983      	ldr	r3, [r0, #24]
     820:	0029      	movs	r1, r5
     822:	0020      	movs	r0, r4
     824:	4798      	blx	r3
     826:	e7f7      	b.n	818 <usb_d_cb_trans_more+0x18>
     828:	000007c1 	.word	0x000007c1
     82c:	2000001c 	.word	0x2000001c

00000830 <_usb_d_cb_trans_done>:

/**
 * Callback when USB transactions are finished.
 */
static void _usb_d_cb_trans_done(const uint8_t ep, const int32_t code, const uint32_t transferred)
{
     830:	b5f0      	push	{r4, r5, r6, r7, lr}
     832:	b087      	sub	sp, #28
     834:	0005      	movs	r5, r0
     836:	000f      	movs	r7, r1
     838:	9201      	str	r2, [sp, #4]
	int8_t           ep_index = _usb_d_find_ep(ep);
     83a:	4b4a      	ldr	r3, [pc, #296]	; (964 <_usb_d_cb_trans_done+0x134>)
     83c:	4798      	blx	r3
     83e:	0004      	movs	r4, r0
	struct usb_d_ep *ept      = &usb_d_inst.ep[ep_index];
     840:	0146      	lsls	r6, r0, #5
     842:	4a49      	ldr	r2, [pc, #292]	; (968 <_usb_d_cb_trans_done+0x138>)
     844:	1996      	adds	r6, r2, r6

	if (code == USB_TRANS_DONE) {
     846:	2f00      	cmp	r7, #0
     848:	d151      	bne.n	8ee <_usb_d_cb_trans_done+0xbe>
		ept->xfer.hdr.status = USB_XFER_DONE;
     84a:	0013      	movs	r3, r2
     84c:	0142      	lsls	r2, r0, #5
     84e:	2000      	movs	r0, #0
     850:	70f0      	strb	r0, [r6, #3]
		if (ept->xfer.hdr.type == USB_EP_XTYPE_CTRL) {
     852:	5cd3      	ldrb	r3, [r2, r3]
     854:	2b00      	cmp	r3, #0
     856:	d00e      	beq.n	876 <_usb_d_cb_trans_done+0x46>
			usb_d_ctrl_trans_done(ept);
			return;
		}
		ept->xfer.hdr.state = USB_EP_S_IDLE;
     858:	0162      	lsls	r2, r4, #5
     85a:	4b43      	ldr	r3, [pc, #268]	; (968 <_usb_d_cb_trans_done+0x138>)
     85c:	189b      	adds	r3, r3, r2
     85e:	2201      	movs	r2, #1
     860:	709a      	strb	r2, [r3, #2]
	} else {
		ept->xfer.hdr.state  = USB_EP_S_ERROR;
		ept->xfer.hdr.status = USB_XFER_ERROR;
	}

	ept->callbacks.xfer(ep, (enum usb_xfer_code)ept->xfer.hdr.status, (void *)transferred);
     862:	0164      	lsls	r4, r4, #5
     864:	4b40      	ldr	r3, [pc, #256]	; (968 <_usb_d_cb_trans_done+0x138>)
     866:	191c      	adds	r4, r3, r4
     868:	69e3      	ldr	r3, [r4, #28]
     86a:	78e1      	ldrb	r1, [r4, #3]
     86c:	9a01      	ldr	r2, [sp, #4]
     86e:	0028      	movs	r0, r5
     870:	4798      	blx	r3
}
     872:	b007      	add	sp, #28
     874:	bdf0      	pop	{r4, r5, r6, r7, pc}
	uint8_t state   = ept->xfer.hdr.state;
     876:	78b3      	ldrb	r3, [r6, #2]
     878:	240c      	movs	r4, #12
     87a:	5734      	ldrsb	r4, [r6, r4]
	if (state == USB_EP_S_X_DATA) {
     87c:	2b03      	cmp	r3, #3
     87e:	d008      	beq.n	892 <_usb_d_cb_trans_done+0x62>
		ept->callbacks.xfer(ept->xfer.hdr.ep, USB_XFER_DONE, ept->xfer.req);
     880:	0032      	movs	r2, r6
     882:	320c      	adds	r2, #12
     884:	7870      	ldrb	r0, [r6, #1]
     886:	2100      	movs	r1, #0
     888:	69f3      	ldr	r3, [r6, #28]
     88a:	4798      	blx	r3
		ept->xfer.hdr.state = USB_EP_S_X_SETUP;
     88c:	2302      	movs	r3, #2
     88e:	70b3      	strb	r3, [r6, #2]
     890:	e7ef      	b.n	872 <_usb_d_cb_trans_done+0x42>
		bool err = ept->callbacks.xfer(ept->xfer.hdr.ep, USB_XFER_DATA, ept->xfer.req);
     892:	7870      	ldrb	r0, [r6, #1]
     894:	0032      	movs	r2, r6
     896:	320c      	adds	r2, #12
     898:	2101      	movs	r1, #1
     89a:	69f3      	ldr	r3, [r6, #28]
     89c:	4798      	blx	r3
		if (err) {
     89e:	2800      	cmp	r0, #0
     8a0:	d010      	beq.n	8c4 <_usb_d_cb_trans_done+0x94>
			ept->xfer.hdr.state  = USB_EP_S_HALTED;
     8a2:	2305      	movs	r3, #5
     8a4:	70b3      	strb	r3, [r6, #2]
			ept->xfer.hdr.status = USB_XFER_HALT;
     8a6:	3b03      	subs	r3, #3
     8a8:	70f3      	strb	r3, [r6, #3]
			_usb_d_dev_ep_stall(req_dir ? ept->xfer.hdr.ep : (ept->xfer.hdr.ep | USB_EP_DIR), USB_EP_STALL_SET);
     8aa:	2c00      	cmp	r4, #0
     8ac:	db08      	blt.n	8c0 <_usb_d_cb_trans_done+0x90>
     8ae:	7873      	ldrb	r3, [r6, #1]
     8b0:	2080      	movs	r0, #128	; 0x80
     8b2:	4240      	negs	r0, r0
     8b4:	4318      	orrs	r0, r3
     8b6:	b2c0      	uxtb	r0, r0
     8b8:	2101      	movs	r1, #1
     8ba:	4b2c      	ldr	r3, [pc, #176]	; (96c <_usb_d_cb_trans_done+0x13c>)
     8bc:	4798      	blx	r3
     8be:	e7d8      	b.n	872 <_usb_d_cb_trans_done+0x42>
     8c0:	7870      	ldrb	r0, [r6, #1]
     8c2:	e7f9      	b.n	8b8 <_usb_d_cb_trans_done+0x88>
			ept->xfer.hdr.state = USB_EP_S_X_STATUS;
     8c4:	2304      	movs	r3, #4
     8c6:	70b3      	strb	r3, [r6, #2]
			_usb_d_trans(ept->xfer.hdr.ep, !req_dir, NULL, 0, 1);
     8c8:	7871      	ldrb	r1, [r6, #1]
	struct usb_d_transfer trans
     8ca:	2200      	movs	r2, #0
     8cc:	9203      	str	r2, [sp, #12]
     8ce:	9204      	str	r2, [sp, #16]
     8d0:	2c00      	cmp	r4, #0
     8d2:	db09      	blt.n	8e8 <_usb_d_cb_trans_done+0xb8>
     8d4:	3b84      	subs	r3, #132	; 0x84
     8d6:	430b      	orrs	r3, r1
     8d8:	b2da      	uxtb	r2, r3
     8da:	a803      	add	r0, sp, #12
     8dc:	7202      	strb	r2, [r0, #8]
     8de:	2301      	movs	r3, #1
     8e0:	7243      	strb	r3, [r0, #9]
	return _usb_d_dev_ep_trans(&trans);
     8e2:	4b23      	ldr	r3, [pc, #140]	; (970 <_usb_d_cb_trans_done+0x140>)
     8e4:	4798      	blx	r3
     8e6:	e7c4      	b.n	872 <_usb_d_cb_trans_done+0x42>
	struct usb_d_transfer trans
     8e8:	220f      	movs	r2, #15
     8ea:	400a      	ands	r2, r1
     8ec:	e7f5      	b.n	8da <_usb_d_cb_trans_done+0xaa>
	} else if (code == USB_TRANS_STALL) {
     8ee:	2f01      	cmp	r7, #1
     8f0:	d00a      	beq.n	908 <_usb_d_cb_trans_done+0xd8>
	} else if (code == USB_TRANS_ABORT) {
     8f2:	2f02      	cmp	r7, #2
     8f4:	d01d      	beq.n	932 <_usb_d_cb_trans_done+0x102>
	} else if (code == USB_TRANS_RESET) {
     8f6:	2f03      	cmp	r7, #3
     8f8:	d02c      	beq.n	954 <_usb_d_cb_trans_done+0x124>
		ept->xfer.hdr.state  = USB_EP_S_ERROR;
     8fa:	0142      	lsls	r2, r0, #5
     8fc:	4b1a      	ldr	r3, [pc, #104]	; (968 <_usb_d_cb_trans_done+0x138>)
     8fe:	189b      	adds	r3, r3, r2
     900:	2206      	movs	r2, #6
     902:	709a      	strb	r2, [r3, #2]
		ept->xfer.hdr.status = USB_XFER_ERROR;
     904:	70da      	strb	r2, [r3, #3]
     906:	e7ac      	b.n	862 <_usb_d_cb_trans_done+0x32>
		ept->xfer.hdr.status = USB_XFER_HALT;
     908:	4b17      	ldr	r3, [pc, #92]	; (968 <_usb_d_cb_trans_done+0x138>)
     90a:	0142      	lsls	r2, r0, #5
     90c:	1899      	adds	r1, r3, r2
     90e:	2002      	movs	r0, #2
     910:	70c8      	strb	r0, [r1, #3]
		if (ept->xfer.hdr.type == USB_EP_XTYPE_CTRL) {
     912:	5cd3      	ldrb	r3, [r2, r3]
     914:	2b00      	cmp	r3, #0
     916:	d005      	beq.n	924 <_usb_d_cb_trans_done+0xf4>
			ept->xfer.hdr.state = USB_EP_S_HALTED;
     918:	0162      	lsls	r2, r4, #5
     91a:	4b13      	ldr	r3, [pc, #76]	; (968 <_usb_d_cb_trans_done+0x138>)
     91c:	189b      	adds	r3, r3, r2
     91e:	2205      	movs	r2, #5
     920:	709a      	strb	r2, [r3, #2]
     922:	e79e      	b.n	862 <_usb_d_cb_trans_done+0x32>
			ept->xfer.hdr.state = USB_EP_S_X_SETUP;
     924:	2202      	movs	r2, #2
     926:	708a      	strb	r2, [r1, #2]
			_usb_d_dev_ep_stall(ep, USB_EP_STALL_CLR);
     928:	2100      	movs	r1, #0
     92a:	0028      	movs	r0, r5
     92c:	4b0f      	ldr	r3, [pc, #60]	; (96c <_usb_d_cb_trans_done+0x13c>)
     92e:	4798      	blx	r3
     930:	e797      	b.n	862 <_usb_d_cb_trans_done+0x32>
		ept->xfer.hdr.status = USB_XFER_ABORT;
     932:	4b0d      	ldr	r3, [pc, #52]	; (968 <_usb_d_cb_trans_done+0x138>)
     934:	0142      	lsls	r2, r0, #5
     936:	1899      	adds	r1, r3, r2
     938:	2004      	movs	r0, #4
     93a:	70c8      	strb	r0, [r1, #3]
		if (ept->xfer.hdr.type == USB_EP_XTYPE_CTRL) {
     93c:	5cd3      	ldrb	r3, [r2, r3]
     93e:	2b00      	cmp	r3, #0
     940:	d005      	beq.n	94e <_usb_d_cb_trans_done+0x11e>
		ept->xfer.hdr.state = USB_EP_S_IDLE;
     942:	0162      	lsls	r2, r4, #5
     944:	4b08      	ldr	r3, [pc, #32]	; (968 <_usb_d_cb_trans_done+0x138>)
     946:	189b      	adds	r3, r3, r2
     948:	2201      	movs	r2, #1
     94a:	709a      	strb	r2, [r3, #2]
     94c:	e789      	b.n	862 <_usb_d_cb_trans_done+0x32>
			ept->xfer.hdr.state = USB_EP_S_X_SETUP;
     94e:	2302      	movs	r3, #2
     950:	708b      	strb	r3, [r1, #2]
			return;
     952:	e78e      	b.n	872 <_usb_d_cb_trans_done+0x42>
		ept->xfer.hdr.state  = USB_EP_S_DISABLED;
     954:	0142      	lsls	r2, r0, #5
     956:	4b04      	ldr	r3, [pc, #16]	; (968 <_usb_d_cb_trans_done+0x138>)
     958:	189b      	adds	r3, r3, r2
     95a:	2200      	movs	r2, #0
     95c:	709a      	strb	r2, [r3, #2]
		ept->xfer.hdr.status = USB_XFER_RESET;
     95e:	3205      	adds	r2, #5
     960:	70da      	strb	r2, [r3, #3]
     962:	e77e      	b.n	862 <_usb_d_cb_trans_done+0x32>
     964:	000007c1 	.word	0x000007c1
     968:	2000001c 	.word	0x2000001c
     96c:	000019b9 	.word	0x000019b9
     970:	00001b89 	.word	0x00001b89

00000974 <usb_d_cb_trans_setup>:
{
     974:	b5f0      	push	{r4, r5, r6, r7, lr}
     976:	46c6      	mov	lr, r8
     978:	b500      	push	{lr}
     97a:	0005      	movs	r5, r0
	int8_t           ep_index = _usb_d_find_ep(ep);
     97c:	4b1f      	ldr	r3, [pc, #124]	; (9fc <usb_d_cb_trans_setup+0x88>)
     97e:	4798      	blx	r3
     980:	0006      	movs	r6, r0
	uint8_t *        req      = ept->xfer.req;
     982:	0143      	lsls	r3, r0, #5
     984:	3308      	adds	r3, #8
     986:	4c1e      	ldr	r4, [pc, #120]	; (a00 <usb_d_cb_trans_setup+0x8c>)
     988:	18e4      	adds	r4, r4, r3
     98a:	3404      	adds	r4, #4
	uint8_t n = _usb_d_dev_ep_read_req(ep, req);
     98c:	0021      	movs	r1, r4
     98e:	0028      	movs	r0, r5
     990:	4b1c      	ldr	r3, [pc, #112]	; (a04 <usb_d_cb_trans_setup+0x90>)
     992:	4798      	blx	r3
     994:	b2c0      	uxtb	r0, r0
	if (n != 8) {
     996:	2808      	cmp	r0, #8
     998:	d00c      	beq.n	9b4 <usb_d_cb_trans_setup+0x40>
		_usb_d_dev_ep_stall(ep, USB_EP_STALL_SET);
     99a:	2101      	movs	r1, #1
     99c:	0028      	movs	r0, r5
     99e:	4c1a      	ldr	r4, [pc, #104]	; (a08 <usb_d_cb_trans_setup+0x94>)
     9a0:	47a0      	blx	r4
		_usb_d_dev_ep_stall(ep | USB_EP_DIR, USB_EP_STALL_SET);
     9a2:	2080      	movs	r0, #128	; 0x80
     9a4:	4240      	negs	r0, r0
     9a6:	4328      	orrs	r0, r5
     9a8:	b2c0      	uxtb	r0, r0
     9aa:	2101      	movs	r1, #1
     9ac:	47a0      	blx	r4
}
     9ae:	bc04      	pop	{r2}
     9b0:	4690      	mov	r8, r2
     9b2:	bdf0      	pop	{r4, r5, r6, r7, pc}
	_usb_d_dev_ep_stall(ep, USB_EP_STALL_CLR);
     9b4:	2100      	movs	r1, #0
     9b6:	0028      	movs	r0, r5
     9b8:	4b13      	ldr	r3, [pc, #76]	; (a08 <usb_d_cb_trans_setup+0x94>)
     9ba:	4698      	mov	r8, r3
     9bc:	4798      	blx	r3
	_usb_d_dev_ep_stall(ep | USB_EP_DIR, USB_EP_STALL_CLR);
     9be:	2780      	movs	r7, #128	; 0x80
     9c0:	427f      	negs	r7, r7
     9c2:	432f      	orrs	r7, r5
     9c4:	b2ff      	uxtb	r7, r7
     9c6:	2100      	movs	r1, #0
     9c8:	0038      	movs	r0, r7
     9ca:	47c0      	blx	r8
	ept->xfer.hdr.state = USB_EP_S_IDLE;
     9cc:	0172      	lsls	r2, r6, #5
     9ce:	4b0c      	ldr	r3, [pc, #48]	; (a00 <usb_d_cb_trans_setup+0x8c>)
     9d0:	189b      	adds	r3, r3, r2
     9d2:	2201      	movs	r2, #1
     9d4:	709a      	strb	r2, [r3, #2]
	if (!ept->callbacks.req(ep, req)) {
     9d6:	695b      	ldr	r3, [r3, #20]
     9d8:	0021      	movs	r1, r4
     9da:	0028      	movs	r0, r5
     9dc:	4798      	blx	r3
     9de:	2800      	cmp	r0, #0
     9e0:	d1e5      	bne.n	9ae <usb_d_cb_trans_setup+0x3a>
		ept->xfer.hdr.state = USB_EP_S_HALTED;
     9e2:	0176      	lsls	r6, r6, #5
     9e4:	4b06      	ldr	r3, [pc, #24]	; (a00 <usb_d_cb_trans_setup+0x8c>)
     9e6:	199e      	adds	r6, r3, r6
     9e8:	2305      	movs	r3, #5
     9ea:	70b3      	strb	r3, [r6, #2]
		_usb_d_dev_ep_stall(ep, USB_EP_STALL_SET);
     9ec:	2101      	movs	r1, #1
     9ee:	0028      	movs	r0, r5
     9f0:	4c05      	ldr	r4, [pc, #20]	; (a08 <usb_d_cb_trans_setup+0x94>)
     9f2:	47a0      	blx	r4
		_usb_d_dev_ep_stall(ep | USB_EP_DIR, USB_EP_STALL_SET);
     9f4:	2101      	movs	r1, #1
     9f6:	0038      	movs	r0, r7
     9f8:	47a0      	blx	r4
     9fa:	e7d8      	b.n	9ae <usb_d_cb_trans_setup+0x3a>
     9fc:	000007c1 	.word	0x000007c1
     a00:	2000001c 	.word	0x2000001c
     a04:	00001b11 	.word	0x00001b11
     a08:	000019b9 	.word	0x000019b9

00000a0c <usb_d_init>:

int32_t usb_d_init(void)
{
     a0c:	b510      	push	{r4, lr}
	int32_t rc = _usb_d_dev_init();
     a0e:	4b12      	ldr	r3, [pc, #72]	; (a58 <usb_d_init+0x4c>)
     a10:	4798      	blx	r3
	uint8_t i;
	if (rc < 0) {
     a12:	2800      	cmp	r0, #0
     a14:	db1e      	blt.n	a54 <usb_d_init+0x48>
		return rc;
	}
	memset(usb_d_inst.ep, 0x00, sizeof(struct usb_d_ep) * CONF_USB_D_NUM_EP_SP);
     a16:	2280      	movs	r2, #128	; 0x80
     a18:	2100      	movs	r1, #0
     a1a:	4810      	ldr	r0, [pc, #64]	; (a5c <usb_d_init+0x50>)
     a1c:	4b10      	ldr	r3, [pc, #64]	; (a60 <usb_d_init+0x54>)
     a1e:	4798      	blx	r3
	for (i = 0; i < CONF_USB_D_NUM_EP_SP; i++) {
     a20:	2200      	movs	r2, #0
     a22:	e00a      	b.n	a3a <usb_d_init+0x2e>
		usb_d_inst.ep[i].xfer.hdr.ep    = 0xFF;
     a24:	0151      	lsls	r1, r2, #5
     a26:	4b0d      	ldr	r3, [pc, #52]	; (a5c <usb_d_init+0x50>)
     a28:	185b      	adds	r3, r3, r1
     a2a:	21ff      	movs	r1, #255	; 0xff
     a2c:	7059      	strb	r1, [r3, #1]
		usb_d_inst.ep[i].callbacks.req  = (usb_d_ep_cb_setup_t)usb_d_dummy_cb_false;
     a2e:	490d      	ldr	r1, [pc, #52]	; (a64 <usb_d_init+0x58>)
     a30:	6159      	str	r1, [r3, #20]
		usb_d_inst.ep[i].callbacks.more = (usb_d_ep_cb_more_t)usb_d_dummy_cb_false;
     a32:	6199      	str	r1, [r3, #24]
		usb_d_inst.ep[i].callbacks.xfer = (usb_d_ep_cb_xfer_t)usb_d_dummy_cb_false;
     a34:	61d9      	str	r1, [r3, #28]
	for (i = 0; i < CONF_USB_D_NUM_EP_SP; i++) {
     a36:	3201      	adds	r2, #1
     a38:	b2d2      	uxtb	r2, r2
     a3a:	2a03      	cmp	r2, #3
     a3c:	d9f2      	bls.n	a24 <usb_d_init+0x18>
	}
	/* Handles device driver endpoint callbacks to build transfer. */
	_usb_d_dev_register_ep_callback(USB_D_DEV_EP_CB_SETUP, (FUNC_PTR)usb_d_cb_trans_setup);
     a3e:	490a      	ldr	r1, [pc, #40]	; (a68 <usb_d_init+0x5c>)
     a40:	2000      	movs	r0, #0
     a42:	4c0a      	ldr	r4, [pc, #40]	; (a6c <usb_d_init+0x60>)
     a44:	47a0      	blx	r4
	_usb_d_dev_register_ep_callback(USB_D_DEV_EP_CB_MORE, (FUNC_PTR)usb_d_cb_trans_more);
     a46:	490a      	ldr	r1, [pc, #40]	; (a70 <usb_d_init+0x64>)
     a48:	2001      	movs	r0, #1
     a4a:	47a0      	blx	r4
	_usb_d_dev_register_ep_callback(USB_D_DEV_EP_CB_DONE, (FUNC_PTR)_usb_d_cb_trans_done);
     a4c:	4909      	ldr	r1, [pc, #36]	; (a74 <usb_d_init+0x68>)
     a4e:	2002      	movs	r0, #2
     a50:	47a0      	blx	r4
	return ERR_NONE;
     a52:	2000      	movs	r0, #0
}
     a54:	bd10      	pop	{r4, pc}
     a56:	46c0      	nop			; (mov r8, r8)
     a58:	00001915 	.word	0x00001915
     a5c:	2000001c 	.word	0x2000001c
     a60:	00001e2f 	.word	0x00001e2f
     a64:	000007fd 	.word	0x000007fd
     a68:	00000975 	.word	0x00000975
     a6c:	00001d61 	.word	0x00001d61
     a70:	00000801 	.word	0x00000801
     a74:	00000831 	.word	0x00000831

00000a78 <assert>:
/**
 * \brief Assert function
 */
void assert(const bool condition, const char *const file, const int line)
{
	if (!(condition)) {
     a78:	2800      	cmp	r0, #0
     a7a:	d100      	bne.n	a7e <assert+0x6>
		__asm("BKPT #0");
     a7c:	be00      	bkpt	0x0000
	}
	(void)file;
	(void)line;
}
     a7e:	4770      	bx	lr

00000a80 <is_list_element>:
 * \brief Check whether element belongs to list
 */
bool is_list_element(const struct list_descriptor *const list, const void *const element)
{
	struct list_element *it;
	for (it = list->head; it; it = it->next) {
     a80:	6803      	ldr	r3, [r0, #0]
     a82:	2b00      	cmp	r3, #0
     a84:	d003      	beq.n	a8e <is_list_element+0xe>
		if (it == element) {
     a86:	428b      	cmp	r3, r1
     a88:	d003      	beq.n	a92 <is_list_element+0x12>
	for (it = list->head; it; it = it->next) {
     a8a:	681b      	ldr	r3, [r3, #0]
     a8c:	e7f9      	b.n	a82 <is_list_element+0x2>
			return true;
		}
	}

	return false;
     a8e:	2000      	movs	r0, #0
}
     a90:	4770      	bx	lr
			return true;
     a92:	2001      	movs	r0, #1
     a94:	e7fc      	b.n	a90 <is_list_element+0x10>
	...

00000a98 <list_insert_as_head>:

/**
 * \brief Insert an element as list head
 */
void list_insert_as_head(struct list_descriptor *const list, void *const element)
{
     a98:	b570      	push	{r4, r5, r6, lr}
     a9a:	0004      	movs	r4, r0
     a9c:	000d      	movs	r5, r1
	ASSERT(!is_list_element(list, element));
     a9e:	4b06      	ldr	r3, [pc, #24]	; (ab8 <list_insert_as_head+0x20>)
     aa0:	4798      	blx	r3
     aa2:	2301      	movs	r3, #1
     aa4:	4058      	eors	r0, r3
     aa6:	b2c0      	uxtb	r0, r0
     aa8:	2239      	movs	r2, #57	; 0x39
     aaa:	4904      	ldr	r1, [pc, #16]	; (abc <list_insert_as_head+0x24>)
     aac:	4b04      	ldr	r3, [pc, #16]	; (ac0 <list_insert_as_head+0x28>)
     aae:	4798      	blx	r3

	((struct list_element *)element)->next = list->head;
     ab0:	6823      	ldr	r3, [r4, #0]
     ab2:	602b      	str	r3, [r5, #0]
	list->head                             = (struct list_element *)element;
     ab4:	6025      	str	r5, [r4, #0]
}
     ab6:	bd70      	pop	{r4, r5, r6, pc}
     ab8:	00000a81 	.word	0x00000a81
     abc:	00001e74 	.word	0x00001e74
     ac0:	00000a79 	.word	0x00000a79

00000ac4 <list_insert_after>:
/**
 * \brief Insert an element after the given list element
 */
void list_insert_after(void *const after, void *const element)
{
	((struct list_element *)element)->next = ((struct list_element *)after)->next;
     ac4:	6803      	ldr	r3, [r0, #0]
     ac6:	600b      	str	r3, [r1, #0]
	((struct list_element *)after)->next   = (struct list_element *)element;
     ac8:	6001      	str	r1, [r0, #0]
}
     aca:	4770      	bx	lr

00000acc <list_remove_head>:
/**
 * \brief Removes list head
 */
void *list_remove_head(struct list_descriptor *const list)
{
	if (list->head) {
     acc:	6803      	ldr	r3, [r0, #0]
     ace:	2b00      	cmp	r3, #0
     ad0:	d003      	beq.n	ada <list_remove_head+0xe>
		struct list_element *tmp = list->head;

		list->head = list->head->next;
     ad2:	681a      	ldr	r2, [r3, #0]
     ad4:	6002      	str	r2, [r0, #0]
		return (void *)tmp;
     ad6:	0018      	movs	r0, r3
	}

	return NULL;
}
     ad8:	4770      	bx	lr
	return NULL;
     ada:	2000      	movs	r0, #0
     adc:	e7fc      	b.n	ad8 <list_remove_head+0xc>
	...

00000ae0 <_init_chip>:

/**
 * \brief Initialize the hardware abstraction layer
 */
void _init_chip(void)
{
     ae0:	b510      	push	{r4, lr}
}

static inline void hri_nvmctrl_set_CTRLB_RWS_bf(const void *const hw, hri_nvmctrl_ctrlb_reg_t mask)
{
	NVMCTRL_CRITICAL_SECTION_ENTER();
	((Nvmctrl *)hw)->CTRLB.reg |= NVMCTRL_CTRLB_RWS(mask);
     ae2:	4b07      	ldr	r3, [pc, #28]	; (b00 <_init_chip+0x20>)
     ae4:	685a      	ldr	r2, [r3, #4]
     ae6:	605a      	str	r2, [r3, #4]
	hri_nvmctrl_set_CTRLB_RWS_bf(NVMCTRL, CONF_NVM_WAIT_STATE);

	_pm_init();
     ae8:	4b06      	ldr	r3, [pc, #24]	; (b04 <_init_chip+0x24>)
     aea:	4798      	blx	r3
	_sysctrl_init_sources();
     aec:	4b06      	ldr	r3, [pc, #24]	; (b08 <_init_chip+0x28>)
     aee:	4798      	blx	r3
#if _GCLK_INIT_1ST
	_gclk_init_generators_by_fref(_GCLK_INIT_1ST);
     af0:	2002      	movs	r0, #2
     af2:	4c06      	ldr	r4, [pc, #24]	; (b0c <_init_chip+0x2c>)
     af4:	47a0      	blx	r4
#endif
	_sysctrl_init_referenced_generators();
     af6:	4b06      	ldr	r3, [pc, #24]	; (b10 <_init_chip+0x30>)
     af8:	4798      	blx	r3
	_gclk_init_generators_by_fref(_GCLK_INIT_LAST);
     afa:	20fd      	movs	r0, #253	; 0xfd
     afc:	47a0      	blx	r4
#if CONF_DMAC_ENABLE
	_pm_enable_bus_clock(PM_BUS_AHB, DMAC);
	_pm_enable_bus_clock(PM_BUS_APBB, DMAC);
	_dma_init();
#endif
}
     afe:	bd10      	pop	{r4, pc}
     b00:	41004000 	.word	0x41004000
     b04:	00000b71 	.word	0x00000b71
     b08:	00000f41 	.word	0x00000f41
     b0c:	00000b15 	.word	0x00000b15
     b10:	00000f8d 	.word	0x00000f8d

00000b14 <_gclk_init_generators_by_fref>:

void _gclk_init_generators_by_fref(uint32_t bm)
{

#if CONF_GCLK_GENERATOR_0_CONFIG == 1
	if (bm & (1ul << 0)) {
     b14:	07c3      	lsls	r3, r0, #31
     b16:	d509      	bpl.n	b2c <_gclk_init_generators_by_fref+0x18>
}

static inline void hri_gclk_write_GENDIV_reg(const void *const hw, hri_gclk_gendiv_reg_t data)
{
	GCLK_CRITICAL_SECTION_ENTER();
	((Gclk *)hw)->GENDIV.reg = data;
     b18:	4b11      	ldr	r3, [pc, #68]	; (b60 <_gclk_init_generators_by_fref+0x4c>)
     b1a:	2280      	movs	r2, #128	; 0x80
     b1c:	0052      	lsls	r2, r2, #1
     b1e:	609a      	str	r2, [r3, #8]
	((Gclk *)hw)->GENCTRL.reg = data;
     b20:	4a10      	ldr	r2, [pc, #64]	; (b64 <_gclk_init_generators_by_fref+0x50>)
     b22:	605a      	str	r2, [r3, #4]
	while (((const Gclk *)hw)->STATUS.bit.SYNCBUSY)
     b24:	4b0e      	ldr	r3, [pc, #56]	; (b60 <_gclk_init_generators_by_fref+0x4c>)
     b26:	785b      	ldrb	r3, [r3, #1]
     b28:	09db      	lsrs	r3, r3, #7
     b2a:	d1fb      	bne.n	b24 <_gclk_init_generators_by_fref+0x10>
		        | (CONF_GCLK_GENERATOR_0_CONFIG << GCLK_GENCTRL_GENEN_Pos) | CONF_GCLK_GEN_0_SRC | GCLK_GENCTRL_ID(0));
	}
#endif

#if CONF_GCLK_GENERATOR_1_CONFIG == 1
	if (bm & (1ul << 1)) {
     b2c:	0783      	lsls	r3, r0, #30
     b2e:	d509      	bpl.n	b44 <_gclk_init_generators_by_fref+0x30>
	((Gclk *)hw)->GENDIV.reg = data;
     b30:	4b0b      	ldr	r3, [pc, #44]	; (b60 <_gclk_init_generators_by_fref+0x4c>)
     b32:	2202      	movs	r2, #2
     b34:	32ff      	adds	r2, #255	; 0xff
     b36:	609a      	str	r2, [r3, #8]
	((Gclk *)hw)->GENCTRL.reg = data;
     b38:	4a0b      	ldr	r2, [pc, #44]	; (b68 <_gclk_init_generators_by_fref+0x54>)
     b3a:	605a      	str	r2, [r3, #4]
	while (((const Gclk *)hw)->STATUS.bit.SYNCBUSY)
     b3c:	4b08      	ldr	r3, [pc, #32]	; (b60 <_gclk_init_generators_by_fref+0x4c>)
     b3e:	785b      	ldrb	r3, [r3, #1]
     b40:	09db      	lsrs	r3, r3, #7
     b42:	d1fb      	bne.n	b3c <_gclk_init_generators_by_fref+0x28>
		        | (CONF_GCLK_GENERATOR_1_CONFIG << GCLK_GENCTRL_GENEN_Pos) | CONF_GCLK_GEN_1_SRC | GCLK_GENCTRL_ID(1));
	}
#endif

#if CONF_GCLK_GENERATOR_2_CONFIG == 1
	if (bm & (1ul << 2)) {
     b44:	0743      	lsls	r3, r0, #29
     b46:	d509      	bpl.n	b5c <_gclk_init_generators_by_fref+0x48>
	((Gclk *)hw)->GENDIV.reg = data;
     b48:	4b05      	ldr	r3, [pc, #20]	; (b60 <_gclk_init_generators_by_fref+0x4c>)
     b4a:	2281      	movs	r2, #129	; 0x81
     b4c:	0052      	lsls	r2, r2, #1
     b4e:	609a      	str	r2, [r3, #8]
	((Gclk *)hw)->GENCTRL.reg = data;
     b50:	4a06      	ldr	r2, [pc, #24]	; (b6c <_gclk_init_generators_by_fref+0x58>)
     b52:	605a      	str	r2, [r3, #4]
	while (((const Gclk *)hw)->STATUS.bit.SYNCBUSY)
     b54:	4b02      	ldr	r3, [pc, #8]	; (b60 <_gclk_init_generators_by_fref+0x4c>)
     b56:	785b      	ldrb	r3, [r3, #1]
     b58:	09db      	lsrs	r3, r3, #7
     b5a:	d1fb      	bne.n	b54 <_gclk_init_generators_by_fref+0x40>
		        | (CONF_GCLK_GEN_8_DIVSEL << GCLK_GENCTRL_DIVSEL_Pos) | (CONF_GCLK_GEN_8_OE << GCLK_GENCTRL_OE_Pos)
		        | (CONF_GCLK_GEN_8_OOV << GCLK_GENCTRL_OOV_Pos) | (CONF_GCLK_GEN_8_IDC << GCLK_GENCTRL_IDC_Pos)
		        | (CONF_GCLK_GENERATOR_8_CONFIG << GCLK_GENCTRL_GENEN_Pos) | CONF_GCLK_GEN_8_SRC | GCLK_GENCTRL_ID(8));
	}
#endif
}
     b5c:	4770      	bx	lr
     b5e:	46c0      	nop			; (mov r8, r8)
     b60:	40000c00 	.word	0x40000c00
     b64:	00010700 	.word	0x00010700
     b68:	00010501 	.word	0x00010501
     b6c:	00010002 	.word	0x00010002

00000b70 <_pm_init>:
}

static inline void hri_pm_set_CPUSEL_CPUDIV_bf(const void *const hw, hri_pm_cpusel_reg_t mask)
{
	PM_CRITICAL_SECTION_ENTER();
	((Pm *)hw)->CPUSEL.reg |= PM_CPUSEL_CPUDIV(mask);
     b70:	4b06      	ldr	r3, [pc, #24]	; (b8c <_pm_init+0x1c>)
     b72:	7a1a      	ldrb	r2, [r3, #8]
     b74:	b2d2      	uxtb	r2, r2
     b76:	721a      	strb	r2, [r3, #8]
}

static inline void hri_pm_set_APBASEL_APBADIV_bf(const void *const hw, hri_pm_apbasel_reg_t mask)
{
	PM_CRITICAL_SECTION_ENTER();
	((Pm *)hw)->APBASEL.reg |= PM_APBASEL_APBADIV(mask);
     b78:	7a5a      	ldrb	r2, [r3, #9]
     b7a:	b2d2      	uxtb	r2, r2
     b7c:	725a      	strb	r2, [r3, #9]
}

static inline void hri_pm_set_APBBSEL_APBBDIV_bf(const void *const hw, hri_pm_apbbsel_reg_t mask)
{
	PM_CRITICAL_SECTION_ENTER();
	((Pm *)hw)->APBBSEL.reg |= PM_APBBSEL_APBBDIV(mask);
     b7e:	7a9a      	ldrb	r2, [r3, #10]
     b80:	b2d2      	uxtb	r2, r2
     b82:	729a      	strb	r2, [r3, #10]
}

static inline void hri_pm_set_APBCSEL_APBCDIV_bf(const void *const hw, hri_pm_apbcsel_reg_t mask)
{
	PM_CRITICAL_SECTION_ENTER();
	((Pm *)hw)->APBCSEL.reg |= PM_APBCSEL_APBCDIV(mask);
     b84:	7ada      	ldrb	r2, [r3, #11]
     b86:	b2d2      	uxtb	r2, r2
     b88:	72da      	strb	r2, [r3, #11]
{
	hri_pm_set_CPUSEL_CPUDIV_bf(PM, CONF_CPU_DIV);
	hri_pm_set_APBASEL_APBADIV_bf(PM, CONF_APBA_DIV);
	hri_pm_set_APBBSEL_APBBDIV_bf(PM, CONF_APBB_DIV);
	hri_pm_set_APBCSEL_APBCDIV_bf(PM, CONF_APBC_DIV);
}
     b8a:	4770      	bx	lr
     b8c:	40000400 	.word	0x40000400

00000b90 <_rtc_timer_interrupt_handler>:
 * \brief RTC Timer interrupt handler
 *
 * \param[in] p The pointer to calendar device struct
 */
static void _rtc_timer_interrupt_handler(struct _timer_device *dev)
{
     b90:	b510      	push	{r4, lr}
     b92:	0004      	movs	r4, r0
	return tmp;
}

static inline hri_rtcmode0_intflag_reg_t hri_rtcmode0_read_INTFLAG_reg(const void *const hw)
{
	return ((Rtc *)hw)->MODE0.INTFLAG.reg;
     b94:	68c3      	ldr	r3, [r0, #12]
     b96:	7a1b      	ldrb	r3, [r3, #8]
	/* Read and mask interrupt flag register */
	uint16_t flag = hri_rtcmode0_read_INTFLAG_reg(dev->hw);

	if (flag & RTC_MODE0_INTFLAG_CMP0) {
     b98:	07db      	lsls	r3, r3, #31
     b9a:	d506      	bpl.n	baa <_rtc_timer_interrupt_handler+0x1a>
		if (dev->timer_cb.period_expired) {
     b9c:	6803      	ldr	r3, [r0, #0]
     b9e:	2b00      	cmp	r3, #0
     ba0:	d000      	beq.n	ba4 <_rtc_timer_interrupt_handler+0x14>
			dev->timer_cb.period_expired(dev);
     ba2:	4798      	blx	r3
		}

		/* Clear interrupt flag */
		hri_rtcmode0_clear_interrupt_CMP0_bit(dev->hw);
     ba4:	68e3      	ldr	r3, [r4, #12]
	((Rtc *)hw)->MODE0.INTFLAG.reg = RTC_MODE0_INTFLAG_CMP0;
     ba6:	2201      	movs	r2, #1
     ba8:	721a      	strb	r2, [r3, #8]
	}
}
     baa:	bd10      	pop	{r4, pc}

00000bac <_timer_init>:
{
     bac:	b570      	push	{r4, r5, r6, lr}
     bae:	0004      	movs	r4, r0
     bb0:	000d      	movs	r5, r1
	ASSERT(dev);
     bb2:	1e43      	subs	r3, r0, #1
     bb4:	4198      	sbcs	r0, r3
     bb6:	b2c0      	uxtb	r0, r0
     bb8:	2233      	movs	r2, #51	; 0x33
     bba:	4910      	ldr	r1, [pc, #64]	; (bfc <_timer_init+0x50>)
     bbc:	4b10      	ldr	r3, [pc, #64]	; (c00 <_timer_init+0x54>)
     bbe:	4798      	blx	r3
	dev->hw = hw;
     bc0:	60e5      	str	r5, [r4, #12]
}

static inline void hri_rtcmode0_write_CTRL_reg(const void *const hw, hri_rtcmode0_ctrl_reg_t data)
{
	RTC_CRITICAL_SECTION_ENTER();
	((Rtc *)hw)->MODE0.CTRL.reg = data;
     bc2:	2301      	movs	r3, #1
     bc4:	802b      	strh	r3, [r5, #0]
	while (((const Rtc *)hw)->MODE0.STATUS.bit.SYNCBUSY)
     bc6:	7aab      	ldrb	r3, [r5, #10]
     bc8:	09db      	lsrs	r3, r3, #7
     bca:	d1fc      	bne.n	bc6 <_timer_init+0x1a>
	hri_rtcmode0_wait_for_sync(dev->hw);
     bcc:	68e2      	ldr	r2, [r4, #12]
     bce:	7a93      	ldrb	r3, [r2, #10]
     bd0:	09db      	lsrs	r3, r3, #7
     bd2:	d1fc      	bne.n	bce <_timer_init+0x22>
	((Rtc *)hw)->MODE0.CTRL.reg = data;
     bd4:	3380      	adds	r3, #128	; 0x80
     bd6:	8013      	strh	r3, [r2, #0]
	while (((const Rtc *)hw)->MODE0.STATUS.bit.SYNCBUSY)
     bd8:	7a93      	ldrb	r3, [r2, #10]
     bda:	09db      	lsrs	r3, r3, #7
     bdc:	d1fc      	bne.n	bd8 <_timer_init+0x2c>
	hri_rtcmode0_write_COMP_COMP_bf(dev->hw, 0, CONF_RTC_COMP_VAL);
     bde:	68e2      	ldr	r2, [r4, #12]

static inline void hri_rtcmode0_write_COMP_COMP_bf(const void *const hw, uint8_t index, hri_rtcmode0_comp_reg_t data)
{
	uint32_t tmp;
	RTC_CRITICAL_SECTION_ENTER();
	tmp = ((Rtc *)hw)->MODE0.COMP[index].reg;
     be0:	6993      	ldr	r3, [r2, #24]
	tmp &= ~RTC_MODE0_COMP_COMP_Msk;
	tmp |= RTC_MODE0_COMP_COMP(data);
	((Rtc *)hw)->MODE0.COMP[index].reg = tmp;
     be2:	2380      	movs	r3, #128	; 0x80
     be4:	00db      	lsls	r3, r3, #3
     be6:	6193      	str	r3, [r2, #24]
	while (((const Rtc *)hw)->MODE0.STATUS.bit.SYNCBUSY)
     be8:	7a93      	ldrb	r3, [r2, #10]
     bea:	09db      	lsrs	r3, r3, #7
     bec:	d1fc      	bne.n	be8 <_timer_init+0x3c>
	((Rtc *)hw)->MODE0.INTENSET.reg = RTC_MODE0_INTENSET_CMP0;
     bee:	3301      	adds	r3, #1
     bf0:	68e2      	ldr	r2, [r4, #12]
     bf2:	71d3      	strb	r3, [r2, #7]
	_rtc_dev = dev;
     bf4:	4b03      	ldr	r3, [pc, #12]	; (c04 <_timer_init+0x58>)
     bf6:	601c      	str	r4, [r3, #0]
}
     bf8:	2000      	movs	r0, #0
     bfa:	bd70      	pop	{r4, r5, r6, pc}
     bfc:	00001e94 	.word	0x00001e94
     c00:	00000a79 	.word	0x00000a79
     c04:	2000009c 	.word	0x2000009c

00000c08 <_rtc_get_timer>:
 * \brief Retrieve timer helper functions
 */
struct _timer_hpl_interface *_rtc_get_timer(void)
{
	return NULL;
}
     c08:	2000      	movs	r0, #0
     c0a:	4770      	bx	lr

00000c0c <RTC_Handler>:

/**
 * \brief Rtc interrupt handler
 */
void RTC_Handler(void)
{
     c0c:	b510      	push	{r4, lr}
	_rtc_timer_interrupt_handler(_rtc_dev);
     c0e:	4b02      	ldr	r3, [pc, #8]	; (c18 <RTC_Handler+0xc>)
     c10:	6818      	ldr	r0, [r3, #0]
     c12:	4b02      	ldr	r3, [pc, #8]	; (c1c <RTC_Handler+0x10>)
     c14:	4798      	blx	r3
}
     c16:	bd10      	pop	{r4, pc}
     c18:	2000009c 	.word	0x2000009c
     c1c:	00000b91 	.word	0x00000b91

00000c20 <_sercom_get_hardware_index>:
{
#ifdef _UNIT_TEST_
	return ((uint32_t)hw - (uint32_t)SERCOM0) / sizeof(Sercom);
#endif

	return ((uint32_t)hw - (uint32_t)SERCOM0) >> 10;
     c20:	4b02      	ldr	r3, [pc, #8]	; (c2c <_sercom_get_hardware_index+0xc>)
     c22:	469c      	mov	ip, r3
     c24:	4460      	add	r0, ip
     c26:	0a80      	lsrs	r0, r0, #10
     c28:	b2c0      	uxtb	r0, r0
}
     c2a:	4770      	bx	lr
     c2c:	bdfff800 	.word	0xbdfff800

00000c30 <_spi_m_sync_init>:

	return NULL;
}

int32_t _spi_m_sync_init(struct _spi_m_sync_dev *dev, void *const hw)
{
     c30:	b570      	push	{r4, r5, r6, lr}
     c32:	0006      	movs	r6, r0
     c34:	000c      	movs	r4, r1
	uint8_t n = _sercom_get_hardware_index((const void *)hw_addr);
     c36:	0008      	movs	r0, r1
     c38:	4b71      	ldr	r3, [pc, #452]	; (e00 <_spi_m_sync_init+0x1d0>)
     c3a:	4798      	blx	r3
	for (i = 0; i < sizeof(sercomspi_regs) / sizeof(struct sercomspi_regs_cfg); i++) {
     c3c:	2300      	movs	r3, #0
     c3e:	2b00      	cmp	r3, #0
     c40:	d100      	bne.n	c44 <_spi_m_sync_init+0x14>
     c42:	e084      	b.n	d4e <_spi_m_sync_init+0x11e>
	return NULL;
     c44:	2500      	movs	r5, #0
	const struct sercomspi_regs_cfg *regs = _spi_get_regs((uint32_t)hw);

	ASSERT(dev && hw);
     c46:	2e00      	cmp	r6, #0
     c48:	d100      	bne.n	c4c <_spi_m_sync_init+0x1c>
     c4a:	e08d      	b.n	d68 <_spi_m_sync_init+0x138>
     c4c:	2c00      	cmp	r4, #0
     c4e:	d100      	bne.n	c52 <_spi_m_sync_init+0x22>
     c50:	e088      	b.n	d64 <_spi_m_sync_init+0x134>
     c52:	2001      	movs	r0, #1
     c54:	4a6b      	ldr	r2, [pc, #428]	; (e04 <_spi_m_sync_init+0x1d4>)
     c56:	496c      	ldr	r1, [pc, #432]	; (e08 <_spi_m_sync_init+0x1d8>)
     c58:	4b6c      	ldr	r3, [pc, #432]	; (e0c <_spi_m_sync_init+0x1dc>)
     c5a:	4798      	blx	r3

	if (regs == NULL) {
     c5c:	2d00      	cmp	r5, #0
     c5e:	d100      	bne.n	c62 <_spi_m_sync_init+0x32>
     c60:	e0cb      	b.n	dfa <_spi_m_sync_init+0x1ca>
	};
}

static inline bool hri_sercomspi_is_syncing(const void *const hw, hri_sercomspi_syncbusy_reg_t reg)
{
	return ((Sercom *)hw)->SPI.SYNCBUSY.reg & reg;
     c62:	69e3      	ldr	r3, [r4, #28]
		return ERR_INVALID_ARG;
	}

	if (!hri_sercomspi_is_syncing(hw, SERCOM_SPI_SYNCBUSY_SWRST)) {
     c64:	07db      	lsls	r3, r3, #31
     c66:	d421      	bmi.n	cac <_spi_m_sync_init+0x7c>
		uint32_t mode = regs->ctrla & SERCOM_SPI_CTRLA_MODE_Msk;
     c68:	782a      	ldrb	r2, [r5, #0]
     c6a:	786b      	ldrb	r3, [r5, #1]
     c6c:	021b      	lsls	r3, r3, #8
     c6e:	4313      	orrs	r3, r2
     c70:	78aa      	ldrb	r2, [r5, #2]
     c72:	0412      	lsls	r2, r2, #16
     c74:	4313      	orrs	r3, r2
     c76:	78ea      	ldrb	r2, [r5, #3]
     c78:	0612      	lsls	r2, r2, #24
     c7a:	431a      	orrs	r2, r3
     c7c:	231c      	movs	r3, #28
     c7e:	401a      	ands	r2, r3
	while (((Sercom *)hw)->SPI.SYNCBUSY.reg & reg) {
     c80:	69e3      	ldr	r3, [r4, #28]
     c82:	079b      	lsls	r3, r3, #30
     c84:	d1fc      	bne.n	c80 <_spi_m_sync_init+0x50>
static inline hri_sercomspi_ctrla_reg_t hri_sercomspi_get_CTRLA_reg(const void *const         hw,
                                                                    hri_sercomspi_ctrla_reg_t mask)
{
	uint32_t tmp;
	hri_sercomspi_wait_for_sync(hw, SERCOM_SPI_SYNCBUSY_SWRST | SERCOM_SPI_SYNCBUSY_ENABLE);
	tmp = ((Sercom *)hw)->SPI.CTRLA.reg;
     c86:	6823      	ldr	r3, [r4, #0]
		if (hri_sercomspi_get_CTRLA_reg(hw, SERCOM_SPI_CTRLA_ENABLE)) {
     c88:	079b      	lsls	r3, r3, #30
     c8a:	d509      	bpl.n	ca0 <_spi_m_sync_init+0x70>
	((Sercom *)hw)->SPI.CTRLA.reg &= ~SERCOM_SPI_CTRLA_ENABLE;
     c8c:	6823      	ldr	r3, [r4, #0]
     c8e:	2102      	movs	r1, #2
     c90:	438b      	bics	r3, r1
     c92:	6023      	str	r3, [r4, #0]
	while (((Sercom *)hw)->SPI.SYNCBUSY.reg & reg) {
     c94:	69e3      	ldr	r3, [r4, #28]
     c96:	079b      	lsls	r3, r3, #30
     c98:	d1fc      	bne.n	c94 <_spi_m_sync_init+0x64>
     c9a:	69e3      	ldr	r3, [r4, #28]
     c9c:	079b      	lsls	r3, r3, #30
     c9e:	d4fc      	bmi.n	c9a <_spi_m_sync_init+0x6a>
			hri_sercomspi_clear_CTRLA_ENABLE_bit(hw);
			hri_sercomspi_wait_for_sync(hw, SERCOM_SPI_SYNCBUSY_ENABLE);
		}
		hri_sercomspi_write_CTRLA_reg(hw, SERCOM_SPI_CTRLA_SWRST | mode);
     ca0:	2301      	movs	r3, #1
     ca2:	4313      	orrs	r3, r2
}

static inline void hri_sercomspi_write_CTRLA_reg(const void *const hw, hri_sercomspi_ctrla_reg_t data)
{
	SERCOM_CRITICAL_SECTION_ENTER();
	((Sercom *)hw)->SPI.CTRLA.reg = data;
     ca4:	6023      	str	r3, [r4, #0]
	while (((Sercom *)hw)->SPI.SYNCBUSY.reg & reg) {
     ca6:	69e3      	ldr	r3, [r4, #28]
     ca8:	079b      	lsls	r3, r3, #30
     caa:	d1fc      	bne.n	ca6 <_spi_m_sync_init+0x76>
     cac:	69e3      	ldr	r3, [r4, #28]
     cae:	07db      	lsls	r3, r3, #31
     cb0:	d4fc      	bmi.n	cac <_spi_m_sync_init+0x7c>
	}
	hri_sercomspi_wait_for_sync(hw, SERCOM_SPI_SYNCBUSY_SWRST);

	dev->prvt = hw;
     cb2:	6034      	str	r4, [r6, #0]

	if ((regs->ctrla & SERCOM_SPI_CTRLA_MODE_Msk) == SERCOM_USART_CTRLA_MODE_SPI_SLAVE) {
     cb4:	782b      	ldrb	r3, [r5, #0]
     cb6:	786a      	ldrb	r2, [r5, #1]
     cb8:	0212      	lsls	r2, r2, #8
     cba:	431a      	orrs	r2, r3
     cbc:	78ab      	ldrb	r3, [r5, #2]
     cbe:	041b      	lsls	r3, r3, #16
     cc0:	431a      	orrs	r2, r3
     cc2:	78eb      	ldrb	r3, [r5, #3]
     cc4:	061b      	lsls	r3, r3, #24
     cc6:	4313      	orrs	r3, r2
     cc8:	221c      	movs	r2, #28
     cca:	4013      	ands	r3, r2
     ccc:	2b08      	cmp	r3, #8
     cce:	d04d      	beq.n	d6c <_spi_m_sync_init+0x13c>
	ASSERT(hw && regs);
     cd0:	2c00      	cmp	r4, #0
     cd2:	d100      	bne.n	cd6 <_spi_m_sync_init+0xa6>
     cd4:	e08d      	b.n	df2 <_spi_m_sync_init+0x1c2>
     cd6:	2d00      	cmp	r5, #0
     cd8:	d100      	bne.n	cdc <_spi_m_sync_init+0xac>
     cda:	e088      	b.n	dee <_spi_m_sync_init+0x1be>
     cdc:	2001      	movs	r0, #1
     cde:	4a4c      	ldr	r2, [pc, #304]	; (e10 <_spi_m_sync_init+0x1e0>)
     ce0:	4949      	ldr	r1, [pc, #292]	; (e08 <_spi_m_sync_init+0x1d8>)
     ce2:	4b4a      	ldr	r3, [pc, #296]	; (e0c <_spi_m_sync_init+0x1dc>)
     ce4:	4798      	blx	r3
	    hw, regs->ctrla & ~(SERCOM_SPI_CTRLA_IBON | SERCOM_SPI_CTRLA_ENABLE | SERCOM_SPI_CTRLA_SWRST));
     ce6:	782b      	ldrb	r3, [r5, #0]
     ce8:	786a      	ldrb	r2, [r5, #1]
     cea:	0212      	lsls	r2, r2, #8
     cec:	431a      	orrs	r2, r3
     cee:	78ab      	ldrb	r3, [r5, #2]
     cf0:	041b      	lsls	r3, r3, #16
     cf2:	431a      	orrs	r2, r3
     cf4:	78eb      	ldrb	r3, [r5, #3]
     cf6:	061b      	lsls	r3, r3, #24
     cf8:	4313      	orrs	r3, r2
	hri_sercomspi_write_CTRLA_reg(
     cfa:	4a46      	ldr	r2, [pc, #280]	; (e14 <_spi_m_sync_init+0x1e4>)
     cfc:	4013      	ands	r3, r2
	((Sercom *)hw)->SPI.CTRLA.reg = data;
     cfe:	6023      	str	r3, [r4, #0]
	while (((Sercom *)hw)->SPI.SYNCBUSY.reg & reg) {
     d00:	69e3      	ldr	r3, [r4, #28]
     d02:	079b      	lsls	r3, r3, #30
     d04:	d1fc      	bne.n	d00 <_spi_m_sync_init+0xd0>
	    (regs->ctrlb
     d06:	792b      	ldrb	r3, [r5, #4]
     d08:	796a      	ldrb	r2, [r5, #5]
     d0a:	0212      	lsls	r2, r2, #8
     d0c:	431a      	orrs	r2, r3
     d0e:	79ab      	ldrb	r3, [r5, #6]
     d10:	041b      	lsls	r3, r3, #16
     d12:	431a      	orrs	r2, r3
     d14:	79eb      	ldrb	r3, [r5, #7]
     d16:	061b      	lsls	r3, r3, #24
     d18:	4313      	orrs	r3, r2
	        | (SERCOM_SPI_CTRLB_RXEN));
     d1a:	4a3f      	ldr	r2, [pc, #252]	; (e18 <_spi_m_sync_init+0x1e8>)
     d1c:	4013      	ands	r3, r2
	hri_sercomspi_write_CTRLB_reg(
     d1e:	2280      	movs	r2, #128	; 0x80
     d20:	0292      	lsls	r2, r2, #10
     d22:	4313      	orrs	r3, r2
}

static inline void hri_sercomspi_write_CTRLB_reg(const void *const hw, hri_sercomspi_ctrlb_reg_t data)
{
	SERCOM_CRITICAL_SECTION_ENTER();
	((Sercom *)hw)->SPI.CTRLB.reg = data;
     d24:	6063      	str	r3, [r4, #4]
	while (((Sercom *)hw)->SPI.SYNCBUSY.reg & reg) {
     d26:	69e3      	ldr	r3, [r4, #28]
     d28:	075b      	lsls	r3, r3, #29
     d2a:	d1fc      	bne.n	d26 <_spi_m_sync_init+0xf6>
	hri_sercomspi_write_BAUD_reg(hw, regs->baud);
     d2c:	7b2b      	ldrb	r3, [r5, #12]
}

static inline void hri_sercomspi_write_BAUD_reg(const void *const hw, hri_sercomspi_baud_reg_t data)
{
	SERCOM_CRITICAL_SECTION_ENTER();
	((Sercom *)hw)->SPI.BAUD.reg = data;
     d2e:	7323      	strb	r3, [r4, #12]
	hri_sercomspi_write_DBGCTRL_reg(hw, regs->dbgctrl);
     d30:	7b6a      	ldrb	r2, [r5, #13]
}

static inline void hri_sercomspi_write_DBGCTRL_reg(const void *const hw, hri_sercomspi_dbgctrl_reg_t data)
{
	SERCOM_CRITICAL_SECTION_ENTER();
	((Sercom *)hw)->SPI.DBGCTRL.reg = data;
     d32:	2330      	movs	r3, #48	; 0x30
     d34:	54e2      	strb	r2, [r4, r3]
	} else {
		_spi_load_regs_master(hw, regs);
	}

	/* Load character size from default hardware configuration */
	dev->char_size = ((regs->ctrlb & SERCOM_SPI_CTRLB_CHSIZE_Msk) == 0) ? 1 : 2;
     d36:	792b      	ldrb	r3, [r5, #4]
     d38:	075b      	lsls	r3, r3, #29
     d3a:	d15c      	bne.n	df6 <_spi_m_sync_init+0x1c6>
     d3c:	2301      	movs	r3, #1
     d3e:	7133      	strb	r3, [r6, #4]

	dev->dummy_byte = regs->dummy_byte;
     d40:	7baa      	ldrb	r2, [r5, #14]
     d42:	7beb      	ldrb	r3, [r5, #15]
     d44:	021b      	lsls	r3, r3, #8
     d46:	4313      	orrs	r3, r2
     d48:	80f3      	strh	r3, [r6, #6]

	return ERR_NONE;
     d4a:	2000      	movs	r0, #0
}
     d4c:	bd70      	pop	{r4, r5, r6, pc}
		if (sercomspi_regs[i].n == n) {
     d4e:	2800      	cmp	r0, #0
     d50:	d002      	beq.n	d58 <_spi_m_sync_init+0x128>
	for (i = 0; i < sizeof(sercomspi_regs) / sizeof(struct sercomspi_regs_cfg); i++) {
     d52:	3301      	adds	r3, #1
     d54:	b2db      	uxtb	r3, r3
     d56:	e772      	b.n	c3e <_spi_m_sync_init+0xe>
			return &sercomspi_regs[i];
     d58:	011d      	lsls	r5, r3, #4
     d5a:	18ea      	adds	r2, r5, r3
     d5c:	4d2f      	ldr	r5, [pc, #188]	; (e1c <_spi_m_sync_init+0x1ec>)
     d5e:	353c      	adds	r5, #60	; 0x3c
     d60:	18ad      	adds	r5, r5, r2
     d62:	e770      	b.n	c46 <_spi_m_sync_init+0x16>
	ASSERT(dev && hw);
     d64:	2000      	movs	r0, #0
     d66:	e775      	b.n	c54 <_spi_m_sync_init+0x24>
     d68:	2000      	movs	r0, #0
     d6a:	e773      	b.n	c54 <_spi_m_sync_init+0x24>
	ASSERT(hw && regs);
     d6c:	2c00      	cmp	r4, #0
     d6e:	d03c      	beq.n	dea <_spi_m_sync_init+0x1ba>
     d70:	2d00      	cmp	r5, #0
     d72:	d038      	beq.n	de6 <_spi_m_sync_init+0x1b6>
     d74:	2001      	movs	r0, #1
     d76:	4a2a      	ldr	r2, [pc, #168]	; (e20 <_spi_m_sync_init+0x1f0>)
     d78:	4923      	ldr	r1, [pc, #140]	; (e08 <_spi_m_sync_init+0x1d8>)
     d7a:	4b24      	ldr	r3, [pc, #144]	; (e0c <_spi_m_sync_init+0x1dc>)
     d7c:	4798      	blx	r3
	    hw, regs->ctrla & ~(SERCOM_SPI_CTRLA_IBON | SERCOM_SPI_CTRLA_ENABLE | SERCOM_SPI_CTRLA_SWRST));
     d7e:	782b      	ldrb	r3, [r5, #0]
     d80:	786a      	ldrb	r2, [r5, #1]
     d82:	0212      	lsls	r2, r2, #8
     d84:	431a      	orrs	r2, r3
     d86:	78ab      	ldrb	r3, [r5, #2]
     d88:	041b      	lsls	r3, r3, #16
     d8a:	431a      	orrs	r2, r3
     d8c:	78eb      	ldrb	r3, [r5, #3]
     d8e:	061b      	lsls	r3, r3, #24
     d90:	4313      	orrs	r3, r2
	hri_sercomspi_write_CTRLA_reg(
     d92:	4a20      	ldr	r2, [pc, #128]	; (e14 <_spi_m_sync_init+0x1e4>)
     d94:	4013      	ands	r3, r2
	((Sercom *)hw)->SPI.CTRLA.reg = data;
     d96:	6023      	str	r3, [r4, #0]
	while (((Sercom *)hw)->SPI.SYNCBUSY.reg & reg) {
     d98:	69e3      	ldr	r3, [r4, #28]
     d9a:	079b      	lsls	r3, r3, #30
     d9c:	d1fc      	bne.n	d98 <_spi_m_sync_init+0x168>
	                              (regs->ctrlb & ~(SERCOM_SPI_CTRLB_MSSEN))
     d9e:	792b      	ldrb	r3, [r5, #4]
     da0:	796a      	ldrb	r2, [r5, #5]
     da2:	0212      	lsls	r2, r2, #8
     da4:	431a      	orrs	r2, r3
     da6:	79ab      	ldrb	r3, [r5, #6]
     da8:	041b      	lsls	r3, r3, #16
     daa:	431a      	orrs	r2, r3
     dac:	79eb      	ldrb	r3, [r5, #7]
     dae:	061b      	lsls	r3, r3, #24
     db0:	4313      	orrs	r3, r2
	                                  | (SERCOM_SPI_CTRLB_RXEN | SERCOM_SPI_CTRLB_SSDE | SERCOM_SPI_CTRLB_PLOADEN));
     db2:	4a1c      	ldr	r2, [pc, #112]	; (e24 <_spi_m_sync_init+0x1f4>)
     db4:	4013      	ands	r3, r2
	hri_sercomspi_write_CTRLB_reg(hw,
     db6:	4a1c      	ldr	r2, [pc, #112]	; (e28 <_spi_m_sync_init+0x1f8>)
     db8:	4313      	orrs	r3, r2
	((Sercom *)hw)->SPI.CTRLB.reg = data;
     dba:	6063      	str	r3, [r4, #4]
	while (((Sercom *)hw)->SPI.SYNCBUSY.reg & reg) {
     dbc:	69e3      	ldr	r3, [r4, #28]
     dbe:	075b      	lsls	r3, r3, #29
     dc0:	d1fc      	bne.n	dbc <_spi_m_sync_init+0x18c>
	hri_sercomspi_write_ADDR_reg(hw, regs->addr);
     dc2:	7a2b      	ldrb	r3, [r5, #8]
     dc4:	7a6a      	ldrb	r2, [r5, #9]
     dc6:	0212      	lsls	r2, r2, #8
     dc8:	431a      	orrs	r2, r3
     dca:	7aab      	ldrb	r3, [r5, #10]
     dcc:	041b      	lsls	r3, r3, #16
     dce:	431a      	orrs	r2, r3
     dd0:	7aeb      	ldrb	r3, [r5, #11]
     dd2:	061b      	lsls	r3, r3, #24
     dd4:	4313      	orrs	r3, r2
	((Sercom *)hw)->SPI.ADDR.reg = data;
     dd6:	6263      	str	r3, [r4, #36]	; 0x24
	hri_sercomspi_write_DBGCTRL_reg(hw, regs->dbgctrl);
     dd8:	7b6a      	ldrb	r2, [r5, #13]
	((Sercom *)hw)->SPI.DBGCTRL.reg = data;
     dda:	2330      	movs	r3, #48	; 0x30
     ddc:	54e2      	strb	r2, [r4, r3]
	return ((Sercom *)hw)->SPI.SYNCBUSY.reg & reg;
     dde:	69e3      	ldr	r3, [r4, #28]
	while (hri_sercomspi_is_syncing(hw, 0xFFFFFFFF))
     de0:	2b00      	cmp	r3, #0
     de2:	d1fc      	bne.n	dde <_spi_m_sync_init+0x1ae>
     de4:	e7a7      	b.n	d36 <_spi_m_sync_init+0x106>
	ASSERT(hw && regs);
     de6:	2000      	movs	r0, #0
     de8:	e7c5      	b.n	d76 <_spi_m_sync_init+0x146>
     dea:	2000      	movs	r0, #0
     dec:	e7c3      	b.n	d76 <_spi_m_sync_init+0x146>
	ASSERT(hw && regs);
     dee:	2000      	movs	r0, #0
     df0:	e775      	b.n	cde <_spi_m_sync_init+0xae>
     df2:	2000      	movs	r0, #0
     df4:	e773      	b.n	cde <_spi_m_sync_init+0xae>
	dev->char_size = ((regs->ctrlb & SERCOM_SPI_CTRLB_CHSIZE_Msk) == 0) ? 1 : 2;
     df6:	2302      	movs	r3, #2
     df8:	e7a1      	b.n	d3e <_spi_m_sync_init+0x10e>
		return ERR_INVALID_ARG;
     dfa:	200d      	movs	r0, #13
     dfc:	4240      	negs	r0, r0
     dfe:	e7a5      	b.n	d4c <_spi_m_sync_init+0x11c>
     e00:	00000c21 	.word	0x00000c21
     e04:	00000925 	.word	0x00000925
     e08:	00001efc 	.word	0x00001efc
     e0c:	00000a79 	.word	0x00000a79
     e10:	000008ef 	.word	0x000008ef
     e14:	fffffefc 	.word	0xfffffefc
     e18:	fffd1dbf 	.word	0xfffd1dbf
     e1c:	00001eac 	.word	0x00001eac
     e20:	00000903 	.word	0x00000903
     e24:	fffdddbf 	.word	0xfffdddbf
     e28:	00020240 	.word	0x00020240

00000e2c <_spi_m_sync_trans>:

	return ERR_NONE;
}

int32_t _spi_m_sync_trans(struct _spi_m_sync_dev *dev, const struct spi_msg *msg)
{
     e2c:	b5f0      	push	{r4, r5, r6, r7, lr}
     e2e:	46ce      	mov	lr, r9
     e30:	4647      	mov	r7, r8
     e32:	b580      	push	{r7, lr}
     e34:	b089      	sub	sp, #36	; 0x24
     e36:	4681      	mov	r9, r0
     e38:	000d      	movs	r5, r1
	void *                 hw   = dev->prvt;
     e3a:	6804      	ldr	r4, [r0, #0]
	int32_t                rc   = 0;
	struct _spi_trans_ctrl ctrl = {msg->txbuf, msg->rxbuf, 0, 0, dev->char_size};
     e3c:	680b      	ldr	r3, [r1, #0]
     e3e:	9303      	str	r3, [sp, #12]
     e40:	684b      	ldr	r3, [r1, #4]
     e42:	9304      	str	r3, [sp, #16]
     e44:	2300      	movs	r3, #0
     e46:	9305      	str	r3, [sp, #20]
     e48:	9306      	str	r3, [sp, #24]
     e4a:	7906      	ldrb	r6, [r0, #4]

	ASSERT(dev && hw);
     e4c:	2800      	cmp	r0, #0
     e4e:	d014      	beq.n	e7a <_spi_m_sync_trans+0x4e>
     e50:	2c00      	cmp	r4, #0
     e52:	d010      	beq.n	e76 <_spi_m_sync_trans+0x4a>
     e54:	2001      	movs	r0, #1
     e56:	4a37      	ldr	r2, [pc, #220]	; (f34 <_spi_m_sync_trans+0x108>)
     e58:	4937      	ldr	r1, [pc, #220]	; (f38 <_spi_m_sync_trans+0x10c>)
     e5a:	4b38      	ldr	r3, [pc, #224]	; (f3c <_spi_m_sync_trans+0x110>)
     e5c:	4798      	blx	r3
     e5e:	69e3      	ldr	r3, [r4, #28]

	/* If settings are not applied (pending), we can not go on */
	if (hri_sercomspi_is_syncing(
     e60:	075b      	lsls	r3, r3, #29
     e62:	d164      	bne.n	f2e <_spi_m_sync_trans+0x102>
	while (((Sercom *)hw)->SPI.SYNCBUSY.reg & reg) {
     e64:	69e3      	ldr	r3, [r4, #28]
     e66:	079b      	lsls	r3, r3, #30
     e68:	d1fc      	bne.n	e64 <_spi_m_sync_trans+0x38>
	tmp = ((Sercom *)hw)->SPI.CTRLA.reg;
     e6a:	6823      	ldr	r3, [r4, #0]
	        hw, (SERCOM_SPI_SYNCBUSY_SWRST | SERCOM_SPI_SYNCBUSY_ENABLE | SERCOM_SPI_SYNCBUSY_CTRLB))) {
		return ERR_BUSY;
	}

	/* SPI must be enabled to start synchronous transfer */
	if (!hri_sercomspi_get_CTRLA_ENABLE_bit(hw)) {
     e6c:	079b      	lsls	r3, r3, #30
     e6e:	d420      	bmi.n	eb2 <_spi_m_sync_trans+0x86>
		return ERR_NOT_INITIALIZED;
     e70:	2014      	movs	r0, #20
     e72:	4240      	negs	r0, r0
     e74:	e056      	b.n	f24 <_spi_m_sync_trans+0xf8>
	ASSERT(dev && hw);
     e76:	2000      	movs	r0, #0
     e78:	e7ed      	b.n	e56 <_spi_m_sync_trans+0x2a>
     e7a:	2000      	movs	r0, #0
     e7c:	e7eb      	b.n	e56 <_spi_m_sync_trans+0x2a>
		return false;
     e7e:	2200      	movs	r2, #0
     e80:	e02d      	b.n	ede <_spi_m_sync_trans+0xb2>
			data |= (*ctrl->txbuf) << 8;
     e82:	7848      	ldrb	r0, [r1, #1]
     e84:	0200      	lsls	r0, r0, #8
     e86:	4647      	mov	r7, r8
     e88:	4307      	orrs	r7, r0
     e8a:	46b8      	mov	r8, r7
			ctrl->txbuf++;
     e8c:	3102      	adds	r1, #2
     e8e:	9103      	str	r1, [sp, #12]
	ctrl->txcnt++;
     e90:	3201      	adds	r2, #1
     e92:	9205      	str	r2, [sp, #20]
	((Sercom *)hw)->SPI.DATA.reg = data;
     e94:	4642      	mov	r2, r8
     e96:	62a2      	str	r2, [r4, #40]	; 0x28
	if (SERCOM_SPI_INTFLAG_ERROR & iflag) {
     e98:	b25b      	sxtb	r3, r3
     e9a:	2b00      	cmp	r3, #0
     e9c:	db35      	blt.n	f0a <_spi_m_sync_trans+0xde>
	return ERR_NONE;
     e9e:	2000      	movs	r0, #0
			}
		}

		rc = _spi_err_check(iflag, hw);

		if (rc < 0) {
     ea0:	2800      	cmp	r0, #0
     ea2:	db3a      	blt.n	f1a <_spi_m_sync_trans+0xee>
			break;
		}
		if (ctrl.txcnt >= msg->size && ctrl.rxcnt >= msg->size) {
     ea4:	9805      	ldr	r0, [sp, #20]
     ea6:	68ab      	ldr	r3, [r5, #8]
     ea8:	4298      	cmp	r0, r3
     eaa:	d302      	bcc.n	eb2 <_spi_m_sync_trans+0x86>
     eac:	9a06      	ldr	r2, [sp, #24]
     eae:	4293      	cmp	r3, r2
     eb0:	d933      	bls.n	f1a <_spi_m_sync_trans+0xee>
	return ((Sercom *)hw)->SPI.INTFLAG.reg;
     eb2:	7e23      	ldrb	r3, [r4, #24]
     eb4:	b2db      	uxtb	r3, r3
	if (!(iflag & SERCOM_SPI_INTFLAG_RXC)) {
     eb6:	075a      	lsls	r2, r3, #29
     eb8:	d5e1      	bpl.n	e7e <_spi_m_sync_trans+0x52>
	return ((Sercom *)hw)->SPI.DATA.reg;
     eba:	6aa1      	ldr	r1, [r4, #40]	; 0x28
	if (ctrl->rxbuf) {
     ebc:	9a04      	ldr	r2, [sp, #16]
     ebe:	2a00      	cmp	r2, #0
     ec0:	d008      	beq.n	ed4 <_spi_m_sync_trans+0xa8>
		*ctrl->rxbuf++ = (uint8_t)data;
     ec2:	1c50      	adds	r0, r2, #1
     ec4:	9004      	str	r0, [sp, #16]
     ec6:	7011      	strb	r1, [r2, #0]
		if (ctrl->char_size > 1) {
     ec8:	2e01      	cmp	r6, #1
     eca:	d903      	bls.n	ed4 <_spi_m_sync_trans+0xa8>
			*ctrl->rxbuf++ = (uint8_t)(data >> 8);
     ecc:	1c90      	adds	r0, r2, #2
     ece:	9004      	str	r0, [sp, #16]
     ed0:	0a09      	lsrs	r1, r1, #8
     ed2:	7051      	strb	r1, [r2, #1]
	ctrl->rxcnt++;
     ed4:	9a06      	ldr	r2, [sp, #24]
     ed6:	9201      	str	r2, [sp, #4]
     ed8:	3201      	adds	r2, #1
     eda:	9206      	str	r2, [sp, #24]
	return true;
     edc:	2201      	movs	r2, #1
		if (!_spi_rx_check_and_receive(hw, iflag, &ctrl)) {
     ede:	2a00      	cmp	r2, #0
     ee0:	d1da      	bne.n	e98 <_spi_m_sync_trans+0x6c>
			if (ctrl.rxcnt >= ctrl.txcnt) {
     ee2:	9906      	ldr	r1, [sp, #24]
     ee4:	9a05      	ldr	r2, [sp, #20]
     ee6:	4291      	cmp	r1, r2
     ee8:	d3d6      	bcc.n	e98 <_spi_m_sync_trans+0x6c>
				_spi_tx_check_and_send(hw, iflag, &ctrl, dev->dummy_byte);
     eea:	4649      	mov	r1, r9
     eec:	88c8      	ldrh	r0, [r1, #6]
	if (!(SERCOM_SPI_INTFLAG_DRE & iflag)) {
     eee:	07d9      	lsls	r1, r3, #31
     ef0:	d5d2      	bpl.n	e98 <_spi_m_sync_trans+0x6c>
	if (ctrl->txbuf) {
     ef2:	9903      	ldr	r1, [sp, #12]
     ef4:	2900      	cmp	r1, #0
     ef6:	d006      	beq.n	f06 <_spi_m_sync_trans+0xda>
		data = *ctrl->txbuf++;
     ef8:	1c48      	adds	r0, r1, #1
     efa:	9003      	str	r0, [sp, #12]
     efc:	7808      	ldrb	r0, [r1, #0]
     efe:	4680      	mov	r8, r0
		if (ctrl->char_size > 1) {
     f00:	2e01      	cmp	r6, #1
     f02:	d8be      	bhi.n	e82 <_spi_m_sync_trans+0x56>
     f04:	e7c4      	b.n	e90 <_spi_m_sync_trans+0x64>
		data = dummy;
     f06:	4680      	mov	r8, r0
     f08:	e7c2      	b.n	e90 <_spi_m_sync_trans+0x64>
}

static inline void hri_sercomspi_clear_STATUS_reg(const void *const hw, hri_sercomspi_status_reg_t mask)
{
	SERCOM_CRITICAL_SECTION_ENTER();
	((Sercom *)hw)->SPI.STATUS.reg = mask;
     f0a:	2301      	movs	r3, #1
     f0c:	425b      	negs	r3, r3
     f0e:	8363      	strh	r3, [r4, #26]
	((Sercom *)hw)->SPI.INTFLAG.reg = mask;
     f10:	3381      	adds	r3, #129	; 0x81
     f12:	7623      	strb	r3, [r4, #24]
		return ERR_OVERFLOW;
     f14:	2013      	movs	r0, #19
     f16:	4240      	negs	r0, r0
     f18:	e7c2      	b.n	ea0 <_spi_m_sync_trans+0x74>
	tmp = ((Sercom *)hw)->SPI.INTFLAG.reg;
     f1a:	7e23      	ldrb	r3, [r4, #24]
	while (!(hri_sercomspi_get_INTFLAG_reg(hw, SERCOM_SPI_INTFLAG_TXC | SERCOM_SPI_INTFLAG_DRE))) {
     f1c:	079b      	lsls	r3, r3, #30
     f1e:	d0fc      	beq.n	f1a <_spi_m_sync_trans+0xee>
	((Sercom *)hw)->SPI.INTFLAG.reg = mask;
     f20:	2303      	movs	r3, #3
     f22:	7623      	strb	r3, [r4, #24]
	}
	/* Wait until SPI bus idle */
	_spi_wait_bus_idle(hw);

	return rc;
}
     f24:	b009      	add	sp, #36	; 0x24
     f26:	bc0c      	pop	{r2, r3}
     f28:	4690      	mov	r8, r2
     f2a:	4699      	mov	r9, r3
     f2c:	bdf0      	pop	{r4, r5, r6, r7, pc}
		return ERR_BUSY;
     f2e:	2004      	movs	r0, #4
     f30:	4240      	negs	r0, r0
     f32:	e7f7      	b.n	f24 <_spi_m_sync_trans+0xf8>
     f34:	00000a85 	.word	0x00000a85
     f38:	00001efc 	.word	0x00001efc
     f3c:	00000a79 	.word	0x00000a79

00000f40 <_sysctrl_init_sources>:
}

static inline void hri_sysctrl_write_XOSC32K_reg(const void *const hw, hri_sysctrl_xosc32k_reg_t data)
{
	SYSCTRL_CRITICAL_SECTION_ENTER();
	((Sysctrl *)hw)->XOSC32K.reg = data;
     f40:	4b10      	ldr	r3, [pc, #64]	; (f84 <_sysctrl_init_sources+0x44>)
     f42:	2206      	movs	r2, #6
     f44:	829a      	strh	r2, [r3, #20]
	((Sysctrl *)hw)->XOSC.reg = data;
     f46:	4a10      	ldr	r2, [pc, #64]	; (f88 <_sysctrl_init_sources+0x48>)
     f48:	821a      	strh	r2, [r3, #16]
}

static inline void hri_sysctrl_set_OSC32K_ENABLE_bit(const void *const hw)
{
	SYSCTRL_CRITICAL_SECTION_ENTER();
	((Sysctrl *)hw)->OSC32K.reg |= SYSCTRL_OSC32K_ENABLE;
     f4a:	699a      	ldr	r2, [r3, #24]
     f4c:	2102      	movs	r1, #2
     f4e:	430a      	orrs	r2, r1
     f50:	619a      	str	r2, [r3, #24]
}

static inline hri_sysctrl_osculp32k_reg_t hri_sysctrl_read_OSCULP32K_CALIB_bf(const void *const hw)
{
	uint8_t tmp;
	tmp = ((Sysctrl *)hw)->OSCULP32K.reg;
     f52:	7f1a      	ldrb	r2, [r3, #28]
	tmp = (tmp & SYSCTRL_OSCULP32K_CALIB_Msk) >> SYSCTRL_OSCULP32K_CALIB_Pos;
     f54:	311d      	adds	r1, #29
     f56:	400a      	ands	r2, r1
}

static inline void hri_sysctrl_write_OSCULP32K_reg(const void *const hw, hri_sysctrl_osculp32k_reg_t data)
{
	SYSCTRL_CRITICAL_SECTION_ENTER();
	((Sysctrl *)hw)->OSCULP32K.reg = data;
     f58:	771a      	strb	r2, [r3, #28]
	return (((Sysctrl *)hw)->PCLKSR.reg & SYSCTRL_PCLKSR_XOSC32KRDY) >> SYSCTRL_PCLKSR_XOSC32KRDY_Pos;
     f5a:	4b0a      	ldr	r3, [pc, #40]	; (f84 <_sysctrl_init_sources+0x44>)
     f5c:	68db      	ldr	r3, [r3, #12]
	                                    (CONF_OSC32K_WRTLOCK << SYSCTRL_OSCULP32K_WRTLOCK_Pos));
#endif

#if CONF_XOSC32K_CONFIG == 1
#if CONF_XOSC32K_ENABLE == 1
	while (!hri_sysctrl_get_PCLKSR_XOSC32KRDY_bit(hw))
     f5e:	079b      	lsls	r3, r3, #30
     f60:	d5fb      	bpl.n	f5a <_sysctrl_init_sources+0x1a>
	((Sysctrl *)hw)->XOSC32K.reg |= SYSCTRL_XOSC32K_ONDEMAND;
     f62:	4a08      	ldr	r2, [pc, #32]	; (f84 <_sysctrl_init_sources+0x44>)
     f64:	8a93      	ldrh	r3, [r2, #20]
     f66:	2180      	movs	r1, #128	; 0x80
     f68:	430b      	orrs	r3, r1
     f6a:	b29b      	uxth	r3, r3
     f6c:	8293      	strh	r3, [r2, #20]
	return (((Sysctrl *)hw)->PCLKSR.reg & SYSCTRL_PCLKSR_XOSCRDY) >> SYSCTRL_PCLKSR_XOSCRDY_Pos;
     f6e:	4b05      	ldr	r3, [pc, #20]	; (f84 <_sysctrl_init_sources+0x44>)
     f70:	68db      	ldr	r3, [r3, #12]
#endif
#endif

#if CONF_XOSC_CONFIG == 1
#if CONF_XOSC_ENABLE == 1
	while (!hri_sysctrl_get_PCLKSR_XOSCRDY_bit(hw))
     f72:	07db      	lsls	r3, r3, #31
     f74:	d5fb      	bpl.n	f6e <_sysctrl_init_sources+0x2e>
	((Sysctrl *)hw)->XOSC.reg |= SYSCTRL_XOSC_AMPGC;
     f76:	4a03      	ldr	r2, [pc, #12]	; (f84 <_sysctrl_init_sources+0x44>)
     f78:	8a13      	ldrh	r3, [r2, #16]
     f7a:	2180      	movs	r1, #128	; 0x80
     f7c:	0109      	lsls	r1, r1, #4
     f7e:	430b      	orrs	r3, r1
     f80:	8213      	strh	r3, [r2, #16]
	hri_sysctrl_set_OSC8M_ONDEMAND_bit(hw);
#endif
#endif

	(void)calib, (void)hw;
}
     f82:	4770      	bx	lr
     f84:	40000800 	.word	0x40000800
     f88:	00000406 	.word	0x00000406

00000f8c <_sysctrl_init_referenced_generators>:
	((Gclk *)hw)->CLKCTRL.reg = data;
     f8c:	2282      	movs	r2, #130	; 0x82
     f8e:	01d2      	lsls	r2, r2, #7
     f90:	4b1c      	ldr	r3, [pc, #112]	; (1004 <_sysctrl_init_referenced_generators+0x78>)
     f92:	805a      	strh	r2, [r3, #2]
}

static inline void hri_sysctrl_write_DFLLCTRL_reg(const void *const hw, hri_sysctrl_dfllctrl_reg_t data)
{
	SYSCTRL_CRITICAL_SECTION_ENTER();
	((Sysctrl *)hw)->DFLLCTRL.reg = data;
     f94:	2202      	movs	r2, #2
     f96:	4b1c      	ldr	r3, [pc, #112]	; (1008 <_sysctrl_init_referenced_generators+0x7c>)
     f98:	849a      	strh	r2, [r3, #36]	; 0x24
	return (((Sysctrl *)hw)->PCLKSR.reg & SYSCTRL_PCLKSR_DFLLRDY) >> SYSCTRL_PCLKSR_DFLLRDY_Pos;
     f9a:	4b1b      	ldr	r3, [pc, #108]	; (1008 <_sysctrl_init_referenced_generators+0x7c>)
     f9c:	68db      	ldr	r3, [r3, #12]
	hri_gclk_write_CLKCTRL_reg(GCLK,
	                           GCLK_CLKCTRL_ID(0) | GCLK_CLKCTRL_GEN(CONF_DFLL_GCLK) | (1 << GCLK_CLKCTRL_CLKEN_Pos));
#endif

	hri_sysctrl_write_DFLLCTRL_reg(hw, SYSCTRL_DFLLCTRL_ENABLE);
	while (!hri_sysctrl_get_PCLKSR_DFLLRDY_bit(hw))
     f9e:	06db      	lsls	r3, r3, #27
     fa0:	d5fb      	bpl.n	f9a <_sysctrl_init_referenced_generators+0xe>
}

static inline void hri_sysctrl_write_DFLLMUL_reg(const void *const hw, hri_sysctrl_dfllmul_reg_t data)
{
	SYSCTRL_CRITICAL_SECTION_ENTER();
	((Sysctrl *)hw)->DFLLMUL.reg = data;
     fa2:	4a1a      	ldr	r2, [pc, #104]	; (100c <_sysctrl_init_referenced_generators+0x80>)
     fa4:	4b18      	ldr	r3, [pc, #96]	; (1008 <_sysctrl_init_referenced_generators+0x7c>)
     fa6:	62da      	str	r2, [r3, #44]	; 0x2c
		;

	hri_sysctrl_write_DFLLMUL_reg(hw,
	                              SYSCTRL_DFLLMUL_CSTEP(CONF_DFLL_CSTEP) | SYSCTRL_DFLLMUL_FSTEP(CONF_DFLL_FSTEP)
	                                  | SYSCTRL_DFLLMUL_MUL(CONF_DFLL_MUL));
	hri_sysctrl_write_DFLLVAL_reg(hw, CONF_DFLLVAL);
     fa8:	4b19      	ldr	r3, [pc, #100]	; (1010 <_sysctrl_init_referenced_generators+0x84>)
     faa:	681b      	ldr	r3, [r3, #0]
     fac:	0e9b      	lsrs	r3, r3, #26
     fae:	2b3f      	cmp	r3, #63	; 0x3f
     fb0:	d020      	beq.n	ff4 <_sysctrl_init_referenced_generators+0x68>
     fb2:	029b      	lsls	r3, r3, #10
     fb4:	2280      	movs	r2, #128	; 0x80
     fb6:	0092      	lsls	r2, r2, #2
     fb8:	4313      	orrs	r3, r2
	((Sysctrl *)hw)->DFLLVAL.reg = data;
     fba:	4a13      	ldr	r2, [pc, #76]	; (1008 <_sysctrl_init_referenced_generators+0x7c>)
     fbc:	6293      	str	r3, [r2, #40]	; 0x28
	((Sysctrl *)hw)->DFLLCTRL.reg = data;
     fbe:	2346      	movs	r3, #70	; 0x46
     fc0:	8493      	strh	r3, [r2, #36]	; 0x24
	tmp = ((Sysctrl *)hw)->DFLLCTRL.reg;
     fc2:	8c93      	ldrh	r3, [r2, #36]	; 0x24
	        | SYSCTRL_DPLLCTRLB_FILTER(CONF_DPLL_FILTER));
#endif

#if CONF_DFLL_CONFIG == 1
#if CONF_DFLL_ENABLE == 1
	if (hri_sysctrl_get_DFLLCTRL_MODE_bit(hw)) {
     fc4:	075b      	lsls	r3, r3, #29
     fc6:	d518      	bpl.n	ffa <_sysctrl_init_referenced_generators+0x6e>
	tmp = ((Sysctrl *)hw)->PCLKSR.reg;
     fc8:	4b0f      	ldr	r3, [pc, #60]	; (1008 <_sysctrl_init_referenced_generators+0x7c>)
     fca:	68da      	ldr	r2, [r3, #12]
	tmp &= mask;
     fcc:	23d0      	movs	r3, #208	; 0xd0
     fce:	4013      	ands	r3, r2
		    = SYSCTRL_PCLKSR_DFLLRDY | SYSCTRL_PCLKSR_DFLLLCKF | SYSCTRL_PCLKSR_DFLLLCKC;
#else
		hri_sysctrl_pclksr_reg_t status_mask = SYSCTRL_PCLKSR_DFLLRDY;
#endif

		while (hri_sysctrl_get_PCLKSR_reg(hw, status_mask) != status_mask)
     fd0:	2bd0      	cmp	r3, #208	; 0xd0
     fd2:	d1f9      	bne.n	fc8 <_sysctrl_init_referenced_generators+0x3c>
	((Sysctrl *)hw)->DFLLCTRL.reg |= SYSCTRL_DFLLCTRL_ONDEMAND;
     fd4:	4a0c      	ldr	r2, [pc, #48]	; (1008 <_sysctrl_init_referenced_generators+0x7c>)
     fd6:	8c93      	ldrh	r3, [r2, #36]	; 0x24
     fd8:	2180      	movs	r1, #128	; 0x80
     fda:	430b      	orrs	r3, r1
     fdc:	b29b      	uxth	r3, r3
     fde:	8493      	strh	r3, [r2, #36]	; 0x24
	return (((Gclk *)hw)->STATUS.reg & GCLK_STATUS_SYNCBUSY) >> GCLK_STATUS_SYNCBUSY_Pos;
     fe0:	4b08      	ldr	r3, [pc, #32]	; (1004 <_sysctrl_init_referenced_generators+0x78>)
     fe2:	785b      	ldrb	r3, [r3, #1]
	hri_sysctrl_set_DPLLCTRLA_ONDEMAND_bit(hw);
#endif
#endif

#if CONF_DFLL_CONFIG == 1
	while (hri_gclk_get_STATUS_SYNCBUSY_bit(GCLK))
     fe4:	09db      	lsrs	r3, r3, #7
     fe6:	d1fb      	bne.n	fe0 <_sysctrl_init_referenced_generators+0x54>
	((Sysctrl *)hw)->OSC32K.reg &= ~SYSCTRL_OSC32K_ENABLE;
     fe8:	4a07      	ldr	r2, [pc, #28]	; (1008 <_sysctrl_init_referenced_generators+0x7c>)
     fea:	6993      	ldr	r3, [r2, #24]
     fec:	2102      	movs	r1, #2
     fee:	438b      	bics	r3, r1
     ff0:	6193      	str	r3, [r2, #24]
	/* Disable after all possible configurations needs sync written. */
	hri_sysctrl_clear_OSC32K_ENABLE_bit(hw);
#endif

	(void)hw;
}
     ff2:	4770      	bx	lr
	hri_sysctrl_write_DFLLVAL_reg(hw, CONF_DFLLVAL);
     ff4:	23fc      	movs	r3, #252	; 0xfc
     ff6:	01db      	lsls	r3, r3, #7
     ff8:	e7df      	b.n	fba <_sysctrl_init_referenced_generators+0x2e>
	return (((Sysctrl *)hw)->PCLKSR.reg & SYSCTRL_PCLKSR_DFLLRDY) >> SYSCTRL_PCLKSR_DFLLRDY_Pos;
     ffa:	4b03      	ldr	r3, [pc, #12]	; (1008 <_sysctrl_init_referenced_generators+0x7c>)
     ffc:	68db      	ldr	r3, [r3, #12]
		while (!hri_sysctrl_get_PCLKSR_DFLLRDY_bit(hw))
     ffe:	06db      	lsls	r3, r3, #27
    1000:	d5fb      	bpl.n	ffa <_sysctrl_init_referenced_generators+0x6e>
    1002:	e7e7      	b.n	fd4 <_sysctrl_init_referenced_generators+0x48>
    1004:	40000c00 	.word	0x40000c00
    1008:	40000800 	.word	0x40000800
    100c:	7dff05b9 	.word	0x7dff05b9
    1010:	00806024 	.word	0x00806024

00001014 <_dummy_func_no_return>:
static bool _dummy_func_no_return(uint32_t unused0, uint32_t unused1)
{
	(void)unused0;
	(void)unused1;
	return false;
}
    1014:	2000      	movs	r0, #0
    1016:	4770      	bx	lr

00001018 <_usb_load_calib>:
#define NVM_USB_PAD_TRANSP_SIZE 5
#define NVM_USB_PAD_TRIM_POS 55
#define NVM_USB_PAD_TRIM_SIZE 3
	Usb *    hw = USB;
	uint32_t pad_transn
	    = (*((uint32_t *)(NVMCTRL_OTP4) + (NVM_USB_PAD_TRANSN_POS / 32)) >> (NVM_USB_PAD_TRANSN_POS % 32))
    1018:	4b12      	ldr	r3, [pc, #72]	; (1064 <_usb_load_calib+0x4c>)
    101a:	681a      	ldr	r2, [r3, #0]
    101c:	0b53      	lsrs	r3, r2, #13
	uint32_t pad_transn
    101e:	211f      	movs	r1, #31
    1020:	400b      	ands	r3, r1
	      & ((1 << NVM_USB_PAD_TRANSN_SIZE) - 1);
	uint32_t pad_transp
	    = (*((uint32_t *)(NVMCTRL_OTP4) + (NVM_USB_PAD_TRANSP_POS / 32)) >> (NVM_USB_PAD_TRANSP_POS % 32))
    1022:	0c90      	lsrs	r0, r2, #18
	uint32_t pad_transp
    1024:	4001      	ands	r1, r0
	      & ((1 << NVM_USB_PAD_TRANSP_SIZE) - 1);
	uint32_t pad_trim = (*((uint32_t *)(NVMCTRL_OTP4) + (NVM_USB_PAD_TRIM_POS / 32)) >> (NVM_USB_PAD_TRIM_POS % 32))
    1026:	0dd0      	lsrs	r0, r2, #23
    1028:	2207      	movs	r2, #7
    102a:	4002      	ands	r2, r0
	                    & ((1 << NVM_USB_PAD_TRIM_SIZE) - 1);
	if (pad_transn == 0x1F) {
    102c:	2b1f      	cmp	r3, #31
    102e:	d012      	beq.n	1056 <_usb_load_calib+0x3e>
		pad_transn = 5;
	}
	if (pad_transp == 0x1F) {
    1030:	291f      	cmp	r1, #31
    1032:	d012      	beq.n	105a <_usb_load_calib+0x42>
		pad_transp = 29;
	}
	if (pad_trim == 0x7) {
    1034:	2a07      	cmp	r2, #7
    1036:	d012      	beq.n	105e <_usb_load_calib+0x46>
		pad_trim = 5;
	}

	hw->DEVICE.PADCAL.reg = USB_PADCAL_TRANSN(pad_transn) | USB_PADCAL_TRANSP(pad_transp) | USB_PADCAL_TRIM(pad_trim);
    1038:	019b      	lsls	r3, r3, #6
    103a:	430b      	orrs	r3, r1
    103c:	0312      	lsls	r2, r2, #12
    103e:	4313      	orrs	r3, r2
    1040:	4a09      	ldr	r2, [pc, #36]	; (1068 <_usb_load_calib+0x50>)
    1042:	8513      	strh	r3, [r2, #40]	; 0x28

	hw->DEVICE.QOSCTRL.bit.CQOS = 3;
    1044:	78d3      	ldrb	r3, [r2, #3]
    1046:	2103      	movs	r1, #3
    1048:	430b      	orrs	r3, r1
    104a:	70d3      	strb	r3, [r2, #3]
	hw->DEVICE.QOSCTRL.bit.DQOS = 3;
    104c:	78d3      	ldrb	r3, [r2, #3]
    104e:	210c      	movs	r1, #12
    1050:	430b      	orrs	r3, r1
    1052:	70d3      	strb	r3, [r2, #3]
}
    1054:	4770      	bx	lr
		pad_transn = 5;
    1056:	3b1a      	subs	r3, #26
    1058:	e7ea      	b.n	1030 <_usb_load_calib+0x18>
		pad_transp = 29;
    105a:	3902      	subs	r1, #2
    105c:	e7ea      	b.n	1034 <_usb_load_calib+0x1c>
		pad_trim = 5;
    105e:	3a02      	subs	r2, #2
    1060:	e7ea      	b.n	1038 <_usb_load_calib+0x20>
    1062:	46c0      	nop			; (mov r8, r8)
    1064:	00806024 	.word	0x00806024
    1068:	41005000 	.word	0x41005000

0000106c <_usb_d_dev_handle_setup>:
/**
 * \brief Handles setup received interrupt
 * \param[in] ept Pointer to endpoint information.
 */
static void _usb_d_dev_handle_setup(struct _usb_d_dev_ep *ept)
{
    106c:	b570      	push	{r4, r5, r6, lr}
	uint8_t epn     = USB_EP_GET_N(ept->ep);
    106e:	7c83      	ldrb	r3, [r0, #18]
    1070:	220f      	movs	r2, #15
    1072:	4013      	ands	r3, r2
	bool    is_ctrl = _usb_d_dev_ep_is_ctrl(ept);
    1074:	7cc1      	ldrb	r1, [r0, #19]
    1076:	3a08      	subs	r2, #8
    1078:	400a      	ands	r2, r1

	if (!is_ctrl) {
    107a:	2a01      	cmp	r2, #1
    107c:	d00d      	beq.n	109a <_usb_d_dev_handle_setup+0x2e>
}

static inline void hri_usbendpoint_clear_EPINTFLAG_reg(const void *const hw, uint8_t submodule_index,
                                                       hri_usbendpoint_epintflag_reg_t mask)
{
	((UsbDevice *)hw)->DeviceEndpoint[submodule_index].EPINTFLAG.reg = mask;
    107e:	001a      	movs	r2, r3
    1080:	3208      	adds	r2, #8
    1082:	0152      	lsls	r2, r2, #5
    1084:	4919      	ldr	r1, [pc, #100]	; (10ec <_usb_d_dev_handle_setup+0x80>)
    1086:	468c      	mov	ip, r1
    1088:	4462      	add	r2, ip
    108a:	2110      	movs	r1, #16
    108c:	71d1      	strb	r1, [r2, #7]
	}
}

static inline void hri_usbendpoint_clear_EPINTEN_RXSTP_bit(const void *const hw, uint8_t submodule_index)
{
	((UsbDevice *)hw)->DeviceEndpoint[submodule_index].EPINTENCLR.reg = USB_DEVICE_EPINTENSET_RXSTP;
    108e:	015b      	lsls	r3, r3, #5
    1090:	4a17      	ldr	r2, [pc, #92]	; (10f0 <_usb_d_dev_handle_setup+0x84>)
    1092:	4694      	mov	ip, r2
    1094:	4463      	add	r3, ip
    1096:	7019      	strb	r1, [r3, #0]
	_usbd_ep_clear_bank_status(epn, 1);
	_usbd_ep_int_ack(epn, USB_D_BANK0_INT_FLAGS | USB_D_BANK1_INT_FLAGS);
	_usbd_ep_int_dis(epn, USB_D_BANK0_INT_FLAGS | USB_D_BANK1_INT_FLAGS);
	/* Invoke callback. */
	dev_inst.ep_callbacks.setup(ept->ep);
}
    1098:	bd70      	pop	{r4, r5, r6, pc}
	if (_usb_d_dev_ep_is_busy(ept)) {
    109a:	064a      	lsls	r2, r1, #25
    109c:	d50c      	bpl.n	10b8 <_usb_d_dev_handle_setup+0x4c>
		ept->flags.bits.is_busy = 0;
    109e:	7cc2      	ldrb	r2, [r0, #19]
    10a0:	2140      	movs	r1, #64	; 0x40
    10a2:	438a      	bics	r2, r1
    10a4:	74c2      	strb	r2, [r0, #19]
	((UsbDevice *)hw)->DeviceEndpoint[submodule_index].EPSTATUSCLR.reg = mask;
    10a6:	001a      	movs	r2, r3
    10a8:	3208      	adds	r2, #8
    10aa:	0152      	lsls	r2, r2, #5
    10ac:	4c0f      	ldr	r4, [pc, #60]	; (10ec <_usb_d_dev_handle_setup+0x80>)
    10ae:	46a4      	mov	ip, r4
    10b0:	4462      	add	r2, ip
    10b2:	2480      	movs	r4, #128	; 0x80
    10b4:	7114      	strb	r4, [r2, #4]
	((UsbDevice *)hw)->DeviceEndpoint[submodule_index].EPSTATUSSET.reg = mask;
    10b6:	7151      	strb	r1, [r2, #5]
	ept->flags.bits.is_stalled = 0;
    10b8:	7cc2      	ldrb	r2, [r0, #19]
    10ba:	2108      	movs	r1, #8
    10bc:	438a      	bics	r2, r1
    10be:	74c2      	strb	r2, [r0, #19]
	bank->STATUS_BK.reg     = 0;
    10c0:	490c      	ldr	r1, [pc, #48]	; (10f4 <_usb_d_dev_handle_setup+0x88>)
    10c2:	015a      	lsls	r2, r3, #5
    10c4:	188c      	adds	r4, r1, r2
    10c6:	2500      	movs	r5, #0
    10c8:	72a5      	strb	r5, [r4, #10]
    10ca:	76a5      	strb	r5, [r4, #26]
	((UsbDevice *)hw)->DeviceEndpoint[submodule_index].EPINTFLAG.reg = mask;
    10cc:	3308      	adds	r3, #8
    10ce:	015b      	lsls	r3, r3, #5
    10d0:	4c06      	ldr	r4, [pc, #24]	; (10ec <_usb_d_dev_handle_setup+0x80>)
    10d2:	46a4      	mov	ip, r4
    10d4:	4463      	add	r3, ip
    10d6:	246f      	movs	r4, #111	; 0x6f
    10d8:	71dc      	strb	r4, [r3, #7]
}

static inline void hri_usbendpoint_clear_EPINTEN_reg(const void *const hw, uint8_t submodule_index,
                                                     hri_usbendpoint_epintenset_reg_t mask)
{
	((UsbDevice *)hw)->DeviceEndpoint[submodule_index].EPINTENCLR.reg = mask;
    10da:	4b05      	ldr	r3, [pc, #20]	; (10f0 <_usb_d_dev_handle_setup+0x84>)
    10dc:	469c      	mov	ip, r3
    10de:	4462      	add	r2, ip
    10e0:	7014      	strb	r4, [r2, #0]
	dev_inst.ep_callbacks.setup(ept->ep);
    10e2:	6e8b      	ldr	r3, [r1, #104]	; 0x68
    10e4:	7c80      	ldrb	r0, [r0, #18]
    10e6:	4798      	blx	r3
    10e8:	e7d6      	b.n	1098 <_usb_d_dev_handle_setup+0x2c>
    10ea:	46c0      	nop			; (mov r8, r8)
    10ec:	41005000 	.word	0x41005000
    10f0:	41005108 	.word	0x41005108
    10f4:	200000a0 	.word	0x200000a0

000010f8 <_usb_d_dev_handle_stall>:
 * \brief Handles stall sent interrupt
 * \param[in] ept Pointer to endpoint information.
 * \param[in] bank_n Bank number.
 */
static void _usb_d_dev_handle_stall(struct _usb_d_dev_ep *ept, const uint8_t bank_n)
{
    10f8:	b510      	push	{r4, lr}
	uint8_t epn = USB_EP_GET_N(ept->ep);
    10fa:	7c82      	ldrb	r2, [r0, #18]
    10fc:	230f      	movs	r3, #15
    10fe:	4013      	ands	r3, r2
		_usbd_ep_int_dis(epn, USB_DEVICE_EPINTFLAG_STALL0 << bank_n);
    1100:	2220      	movs	r2, #32
    1102:	408a      	lsls	r2, r1
	hri_usbendpoint_clear_EPINTEN_reg(USB, epn, flags);
    1104:	b2d2      	uxtb	r2, r2
    1106:	015b      	lsls	r3, r3, #5
    1108:	4905      	ldr	r1, [pc, #20]	; (1120 <_usb_d_dev_handle_stall+0x28>)
    110a:	468c      	mov	ip, r1
    110c:	4463      	add	r3, ip
    110e:	701a      	strb	r2, [r3, #0]
	/* Clear interrupt enable. Leave status there for status check. */
	_usbd_ep_int_stall_en(epn, bank_n, false);
	dev_inst.ep_callbacks.done(ept->ep, USB_TRANS_STALL, ept->trans_count);
    1110:	4b04      	ldr	r3, [pc, #16]	; (1124 <_usb_d_dev_handle_stall+0x2c>)
    1112:	6f1b      	ldr	r3, [r3, #112]	; 0x70
    1114:	6882      	ldr	r2, [r0, #8]
    1116:	7c80      	ldrb	r0, [r0, #18]
    1118:	2101      	movs	r1, #1
    111a:	4798      	blx	r3
}
    111c:	bd10      	pop	{r4, pc}
    111e:	46c0      	nop			; (mov r8, r8)
    1120:	41005108 	.word	0x41005108
    1124:	200000a0 	.word	0x200000a0

00001128 <_usb_d_dev_trans_done>:
 *  \brief Finish the transaction and invoke callback
 * \param[in, out] ept Pointer to endpoint information.
 * \param[in] code Information code passed.
 */
static void _usb_d_dev_trans_done(struct _usb_d_dev_ep *ept, const int32_t code)
{
    1128:	b510      	push	{r4, lr}
	if (!(_usb_d_dev_ep_is_used(ept) && _usb_d_dev_ep_is_busy(ept))) {
    112a:	7c83      	ldrb	r3, [r0, #18]
    112c:	2bff      	cmp	r3, #255	; 0xff
    112e:	d002      	beq.n	1136 <_usb_d_dev_trans_done+0xe>
    1130:	7cc2      	ldrb	r2, [r0, #19]
    1132:	0652      	lsls	r2, r2, #25
    1134:	d400      	bmi.n	1138 <_usb_d_dev_trans_done+0x10>
		return;
	}
	ept->flags.bits.is_busy = 0;
	dev_inst.ep_callbacks.done(ept->ep, code, ept->trans_count);
}
    1136:	bd10      	pop	{r4, pc}
	ept->flags.bits.is_busy = 0;
    1138:	7cc2      	ldrb	r2, [r0, #19]
    113a:	2440      	movs	r4, #64	; 0x40
    113c:	43a2      	bics	r2, r4
    113e:	74c2      	strb	r2, [r0, #19]
	dev_inst.ep_callbacks.done(ept->ep, code, ept->trans_count);
    1140:	4a02      	ldr	r2, [pc, #8]	; (114c <_usb_d_dev_trans_done+0x24>)
    1142:	6f14      	ldr	r4, [r2, #112]	; 0x70
    1144:	6882      	ldr	r2, [r0, #8]
    1146:	0018      	movs	r0, r3
    1148:	47a0      	blx	r4
    114a:	e7f4      	b.n	1136 <_usb_d_dev_trans_done+0xe>
    114c:	200000a0 	.word	0x200000a0

00001150 <_usb_d_dev_trans_stop>:
 * \param[in, out] ept Pointer to endpoint information.
 * \param[in] dir Endpoint direction.
 * \param[in] code Information code passed.
 */
static void _usb_d_dev_trans_stop(struct _usb_d_dev_ep *ept, bool dir, const int32_t code)
{
    1150:	b5f0      	push	{r4, r5, r6, r7, lr}
    1152:	b083      	sub	sp, #12
	uint8_t epn = USB_EP_GET_N(ept->ep);
    1154:	7c84      	ldrb	r4, [r0, #18]
    1156:	230f      	movs	r3, #15
    1158:	4023      	ands	r3, r4
	;
	const uint8_t intflags[2] = {USB_D_BANK0_INT_FLAGS, USB_D_BANK1_INT_FLAGS};
    115a:	4d18      	ldr	r5, [pc, #96]	; (11bc <_usb_d_dev_trans_stop+0x6c>)
    115c:	882e      	ldrh	r6, [r5, #0]
    115e:	ad01      	add	r5, sp, #4
    1160:	802e      	strh	r6, [r5, #0]
	if (!(_usb_d_dev_ep_is_used(ept) && _usb_d_dev_ep_is_busy(ept))) {
    1162:	2cff      	cmp	r4, #255	; 0xff
    1164:	d01e      	beq.n	11a4 <_usb_d_dev_trans_stop+0x54>
    1166:	7cc4      	ldrb	r4, [r0, #19]
    1168:	0664      	lsls	r4, r4, #25
    116a:	d51b      	bpl.n	11a4 <_usb_d_dev_trans_stop+0x54>
		return;
	}
	/* Stop transfer */
	if (dir) {
    116c:	2900      	cmp	r1, #0
    116e:	d01b      	beq.n	11a8 <_usb_d_dev_trans_stop+0x58>
	((UsbDevice *)hw)->DeviceEndpoint[submodule_index].EPSTATUSCLR.reg = mask;
    1170:	001c      	movs	r4, r3
    1172:	3408      	adds	r4, #8
    1174:	0164      	lsls	r4, r4, #5
    1176:	4d12      	ldr	r5, [pc, #72]	; (11c0 <_usb_d_dev_trans_stop+0x70>)
    1178:	46ac      	mov	ip, r5
    117a:	4464      	add	r4, ip
    117c:	2580      	movs	r5, #128	; 0x80
    117e:	7125      	strb	r5, [r4, #4]
		_usbd_ep_set_in_rdy(epn, 1, false);
	} else {
		/* NAK OUT */
		_usbd_ep_set_out_rdy(epn, 0, false);
	}
	_usbd_ep_int_ack(epn, intflags[dir]);
    1180:	ad01      	add	r5, sp, #4
    1182:	5c6e      	ldrb	r6, [r5, r1]
	((UsbDevice *)hw)->DeviceEndpoint[submodule_index].EPINTFLAG.reg = mask;
    1184:	001c      	movs	r4, r3
    1186:	3408      	adds	r4, #8
    1188:	0164      	lsls	r4, r4, #5
    118a:	4f0d      	ldr	r7, [pc, #52]	; (11c0 <_usb_d_dev_trans_stop+0x70>)
    118c:	46bc      	mov	ip, r7
    118e:	4464      	add	r4, ip
    1190:	71e6      	strb	r6, [r4, #7]
	_usbd_ep_int_dis(epn, intflags[dir]);
    1192:	5c69      	ldrb	r1, [r5, r1]
	((UsbDevice *)hw)->DeviceEndpoint[submodule_index].EPINTENCLR.reg = mask;
    1194:	015b      	lsls	r3, r3, #5
    1196:	4c0b      	ldr	r4, [pc, #44]	; (11c4 <_usb_d_dev_trans_stop+0x74>)
    1198:	46a4      	mov	ip, r4
    119a:	4463      	add	r3, ip
    119c:	7019      	strb	r1, [r3, #0]
	_usb_d_dev_trans_done(ept, code);
    119e:	0011      	movs	r1, r2
    11a0:	4b09      	ldr	r3, [pc, #36]	; (11c8 <_usb_d_dev_trans_stop+0x78>)
    11a2:	4798      	blx	r3
}
    11a4:	b003      	add	sp, #12
    11a6:	bdf0      	pop	{r4, r5, r6, r7, pc}
	((UsbDevice *)hw)->DeviceEndpoint[submodule_index].EPSTATUSSET.reg = mask;
    11a8:	001c      	movs	r4, r3
    11aa:	3408      	adds	r4, #8
    11ac:	0164      	lsls	r4, r4, #5
    11ae:	4d04      	ldr	r5, [pc, #16]	; (11c0 <_usb_d_dev_trans_stop+0x70>)
    11b0:	46ac      	mov	ip, r5
    11b2:	4464      	add	r4, ip
    11b4:	2540      	movs	r5, #64	; 0x40
    11b6:	7165      	strb	r5, [r4, #5]
    11b8:	e7e2      	b.n	1180 <_usb_d_dev_trans_stop+0x30>
    11ba:	46c0      	nop			; (mov r8, r8)
    11bc:	00001f18 	.word	0x00001f18
    11c0:	41005000 	.word	0x41005000
    11c4:	41005108 	.word	0x41005108
    11c8:	00001129 	.word	0x00001129

000011cc <_usb_d_dev_handle_trfail>:
{
    11cc:	b5f0      	push	{r4, r5, r6, r7, lr}
    11ce:	b083      	sub	sp, #12
	uint8_t            epn     = USB_EP_GET_N(ept->ep);
    11d0:	7c83      	ldrb	r3, [r0, #18]
    11d2:	220f      	movs	r2, #15
    11d4:	4013      	ands	r3, r2
	const uint8_t      fail[2] = {USB_DEVICE_EPINTFLAG_TRFAIL0, USB_DEVICE_EPINTFLAG_TRFAIL1};
    11d6:	4a3c      	ldr	r2, [pc, #240]	; (12c8 <_usb_d_dev_handle_trfail+0xfc>)
    11d8:	8894      	ldrh	r4, [r2, #4]
    11da:	aa01      	add	r2, sp, #4
    11dc:	8014      	strh	r4, [r2, #0]
	UsbDeviceDescBank *bank    = prvt_inst.desc_table[epn].DeviceDescBank;
    11de:	015a      	lsls	r2, r3, #5
    11e0:	4c3a      	ldr	r4, [pc, #232]	; (12cc <_usb_d_dev_handle_trfail+0x100>)
    11e2:	18a4      	adds	r4, r4, r2
	uint8_t            eptype
    11e4:	2900      	cmp	r1, #0
    11e6:	d033      	beq.n	1250 <_usb_d_dev_handle_trfail+0x84>

static inline hri_usbendpoint_epcfg_reg_t hri_usbendpoint_read_EPCFG_EPTYPE1_bf(const void *const hw,
                                                                                uint8_t           submodule_index)
{
	uint8_t tmp;
	tmp = ((UsbDevice *)hw)->DeviceEndpoint[submodule_index].EPCFG.reg;
    11e8:	001a      	movs	r2, r3
    11ea:	3208      	adds	r2, #8
    11ec:	0152      	lsls	r2, r2, #5
    11ee:	4d38      	ldr	r5, [pc, #224]	; (12d0 <_usb_d_dev_handle_trfail+0x104>)
    11f0:	5d52      	ldrb	r2, [r2, r5]
	tmp = (tmp & USB_DEVICE_EPCFG_EPTYPE1_Msk) >> USB_DEVICE_EPCFG_EPTYPE1_Pos;
    11f2:	0912      	lsrs	r2, r2, #4
    11f4:	2507      	movs	r5, #7
    11f6:	4015      	ands	r5, r2
	bool                      is_ctrl = _usb_d_dev_ep_is_ctrl(ept);
    11f8:	7cc2      	ldrb	r2, [r0, #19]
    11fa:	2607      	movs	r6, #7
    11fc:	4016      	ands	r6, r2
	st.reg = bank[bank_n].STATUS_BK.reg;
    11fe:	010a      	lsls	r2, r1, #4
    1200:	18a2      	adds	r2, r4, r2
    1202:	7a94      	ldrb	r4, [r2, #10]
    1204:	b2e4      	uxtb	r4, r4
	if ((eptype == USB_D_EPTYPE_ISOCH) && st.bit.CRCERR) {
    1206:	2d02      	cmp	r5, #2
    1208:	d02a      	beq.n	1260 <_usb_d_dev_handle_trfail+0x94>
	} else if (st.bit.ERRORFLOW) {
    120a:	07a4      	lsls	r4, r4, #30
    120c:	d544      	bpl.n	1298 <_usb_d_dev_handle_trfail+0xcc>
		bank[bank_n].STATUS_BK.bit.ERRORFLOW = 0;
    120e:	7a94      	ldrb	r4, [r2, #10]
    1210:	2502      	movs	r5, #2
    1212:	43ac      	bics	r4, r5
    1214:	7294      	strb	r4, [r2, #10]
		hri_usbendpoint_clear_EPINTFLAG_reg(hw, epn, fail[bank_n]);
    1216:	ac01      	add	r4, sp, #4
    1218:	5c65      	ldrb	r5, [r4, r1]
	((UsbDevice *)hw)->DeviceEndpoint[submodule_index].EPINTFLAG.reg = mask;
    121a:	001a      	movs	r2, r3
    121c:	3208      	adds	r2, #8
    121e:	0152      	lsls	r2, r2, #5
    1220:	4f2b      	ldr	r7, [pc, #172]	; (12d0 <_usb_d_dev_handle_trfail+0x104>)
    1222:	46bc      	mov	ip, r7
    1224:	4462      	add	r2, ip
    1226:	71d5      	strb	r5, [r2, #7]
		hri_usbendpoint_clear_EPINTEN_reg(hw, epn, fail[bank_n]);
    1228:	5c62      	ldrb	r2, [r4, r1]
	((UsbDevice *)hw)->DeviceEndpoint[submodule_index].EPINTENCLR.reg = mask;
    122a:	015b      	lsls	r3, r3, #5
    122c:	4c29      	ldr	r4, [pc, #164]	; (12d4 <_usb_d_dev_handle_trfail+0x108>)
    122e:	46a4      	mov	ip, r4
    1230:	4463      	add	r3, ip
    1232:	701a      	strb	r2, [r3, #0]
		if (is_ctrl && _usb_d_dev_ep_is_busy(ept)) {
    1234:	2e01      	cmp	r6, #1
    1236:	d145      	bne.n	12c4 <_usb_d_dev_handle_trfail+0xf8>
    1238:	7cc3      	ldrb	r3, [r0, #19]
    123a:	065b      	lsls	r3, r3, #25
    123c:	d542      	bpl.n	12c4 <_usb_d_dev_handle_trfail+0xf8>
			if (bank_n != _usb_d_dev_ep_is_in(ept)) {
    123e:	7cc3      	ldrb	r3, [r0, #19]
    1240:	09db      	lsrs	r3, r3, #7
    1242:	4299      	cmp	r1, r3
    1244:	d03e      	beq.n	12c4 <_usb_d_dev_handle_trfail+0xf8>
				_usb_d_dev_trans_stop(ept, _usb_d_dev_ep_is_in(ept), USB_TRANS_DONE);
    1246:	2200      	movs	r2, #0
    1248:	0019      	movs	r1, r3
    124a:	4b23      	ldr	r3, [pc, #140]	; (12d8 <_usb_d_dev_handle_trfail+0x10c>)
    124c:	4798      	blx	r3
    124e:	e039      	b.n	12c4 <_usb_d_dev_handle_trfail+0xf8>
	tmp = ((UsbDevice *)hw)->DeviceEndpoint[submodule_index].EPCFG.reg;
    1250:	001a      	movs	r2, r3
    1252:	3208      	adds	r2, #8
    1254:	0152      	lsls	r2, r2, #5
    1256:	4d1e      	ldr	r5, [pc, #120]	; (12d0 <_usb_d_dev_handle_trfail+0x104>)
    1258:	5d55      	ldrb	r5, [r2, r5]
	tmp = (tmp & USB_DEVICE_EPCFG_EPTYPE0_Msk) >> USB_DEVICE_EPCFG_EPTYPE0_Pos;
    125a:	2207      	movs	r2, #7
    125c:	4015      	ands	r5, r2
    125e:	e7cb      	b.n	11f8 <_usb_d_dev_handle_trfail+0x2c>
	if ((eptype == USB_D_EPTYPE_ISOCH) && st.bit.CRCERR) {
    1260:	07e5      	lsls	r5, r4, #31
    1262:	d5d2      	bpl.n	120a <_usb_d_dev_handle_trfail+0x3e>
		bank[bank_n].STATUS_BK.bit.CRCERR = 0;
    1264:	7a94      	ldrb	r4, [r2, #10]
    1266:	2501      	movs	r5, #1
    1268:	43ac      	bics	r4, r5
    126a:	7294      	strb	r4, [r2, #10]
		hri_usbendpoint_clear_EPINTFLAG_reg(hw, epn, fail[bank_n]);
    126c:	ac01      	add	r4, sp, #4
    126e:	5c65      	ldrb	r5, [r4, r1]
	((UsbDevice *)hw)->DeviceEndpoint[submodule_index].EPINTFLAG.reg = mask;
    1270:	001a      	movs	r2, r3
    1272:	3208      	adds	r2, #8
    1274:	0152      	lsls	r2, r2, #5
    1276:	4e16      	ldr	r6, [pc, #88]	; (12d0 <_usb_d_dev_handle_trfail+0x104>)
    1278:	46b4      	mov	ip, r6
    127a:	4462      	add	r2, ip
    127c:	71d5      	strb	r5, [r2, #7]
		hri_usbendpoint_clear_EPINTEN_reg(hw, epn, fail[bank_n]);
    127e:	5c62      	ldrb	r2, [r4, r1]
	((UsbDevice *)hw)->DeviceEndpoint[submodule_index].EPINTENCLR.reg = mask;
    1280:	015b      	lsls	r3, r3, #5
    1282:	4c14      	ldr	r4, [pc, #80]	; (12d4 <_usb_d_dev_handle_trfail+0x108>)
    1284:	46a4      	mov	ip, r4
    1286:	4463      	add	r3, ip
    1288:	701a      	strb	r2, [r3, #0]
		_usb_d_dev_trans_stop(ept, bank_n, USB_TRANS_ERROR);
    128a:	1e4b      	subs	r3, r1, #1
    128c:	4199      	sbcs	r1, r3
    128e:	b2c9      	uxtb	r1, r1
    1290:	2204      	movs	r2, #4
    1292:	4b11      	ldr	r3, [pc, #68]	; (12d8 <_usb_d_dev_handle_trfail+0x10c>)
    1294:	4798      	blx	r3
    1296:	e015      	b.n	12c4 <_usb_d_dev_handle_trfail+0xf8>
	bank->STATUS_BK.reg     = 0;
    1298:	005a      	lsls	r2, r3, #1
    129a:	1852      	adds	r2, r2, r1
    129c:	0112      	lsls	r2, r2, #4
    129e:	480b      	ldr	r0, [pc, #44]	; (12cc <_usb_d_dev_handle_trfail+0x100>)
    12a0:	1882      	adds	r2, r0, r2
    12a2:	2000      	movs	r0, #0
    12a4:	7290      	strb	r0, [r2, #10]
		hri_usbendpoint_clear_EPINTFLAG_reg(hw, epn, fail[bank_n]);
    12a6:	a801      	add	r0, sp, #4
    12a8:	5c44      	ldrb	r4, [r0, r1]
	((UsbDevice *)hw)->DeviceEndpoint[submodule_index].EPINTFLAG.reg = mask;
    12aa:	001a      	movs	r2, r3
    12ac:	3208      	adds	r2, #8
    12ae:	0152      	lsls	r2, r2, #5
    12b0:	4d07      	ldr	r5, [pc, #28]	; (12d0 <_usb_d_dev_handle_trfail+0x104>)
    12b2:	46ac      	mov	ip, r5
    12b4:	4462      	add	r2, ip
    12b6:	71d4      	strb	r4, [r2, #7]
		hri_usbendpoint_clear_EPINTEN_reg(hw, epn, fail[bank_n]);
    12b8:	5c42      	ldrb	r2, [r0, r1]
	((UsbDevice *)hw)->DeviceEndpoint[submodule_index].EPINTENCLR.reg = mask;
    12ba:	015b      	lsls	r3, r3, #5
    12bc:	4905      	ldr	r1, [pc, #20]	; (12d4 <_usb_d_dev_handle_trfail+0x108>)
    12be:	468c      	mov	ip, r1
    12c0:	4463      	add	r3, ip
    12c2:	701a      	strb	r2, [r3, #0]
}
    12c4:	b003      	add	sp, #12
    12c6:	bdf0      	pop	{r4, r5, r6, r7, pc}
    12c8:	00001f18 	.word	0x00001f18
    12cc:	200000a0 	.word	0x200000a0
    12d0:	41005000 	.word	0x41005000
    12d4:	41005108 	.word	0x41005108
    12d8:	00001151 	.word	0x00001151

000012dc <_usb_d_dev_reset_epts>:
{
    12dc:	b570      	push	{r4, r5, r6, lr}
	for (i = 0; i < USB_D_N_EP; i++) {
    12de:	2500      	movs	r5, #0
    12e0:	e018      	b.n	1314 <_usb_d_dev_reset_epts+0x38>
		_usb_d_dev_trans_done(&dev_inst.ep[i], USB_TRANS_RESET);
    12e2:	4c10      	ldr	r4, [pc, #64]	; (1324 <_usb_d_dev_reset_epts+0x48>)
    12e4:	3460      	adds	r4, #96	; 0x60
    12e6:	00ae      	lsls	r6, r5, #2
    12e8:	1973      	adds	r3, r6, r5
    12ea:	0098      	lsls	r0, r3, #2
    12ec:	3010      	adds	r0, #16
    12ee:	1820      	adds	r0, r4, r0
    12f0:	3004      	adds	r0, #4
    12f2:	2103      	movs	r1, #3
    12f4:	4b0c      	ldr	r3, [pc, #48]	; (1328 <_usb_d_dev_reset_epts+0x4c>)
    12f6:	4798      	blx	r3
		dev_inst.ep[i].ep       = 0xFF;
    12f8:	1972      	adds	r2, r6, r5
    12fa:	0093      	lsls	r3, r2, #2
    12fc:	18e3      	adds	r3, r4, r3
    12fe:	3326      	adds	r3, #38	; 0x26
    1300:	22ff      	movs	r2, #255	; 0xff
    1302:	701a      	strb	r2, [r3, #0]
		dev_inst.ep[i].flags.u8 = 0;
    1304:	1976      	adds	r6, r6, r5
    1306:	00b3      	lsls	r3, r6, #2
    1308:	18e4      	adds	r4, r4, r3
    130a:	3427      	adds	r4, #39	; 0x27
    130c:	2300      	movs	r3, #0
    130e:	7023      	strb	r3, [r4, #0]
	for (i = 0; i < USB_D_N_EP; i++) {
    1310:	3501      	adds	r5, #1
    1312:	b2ed      	uxtb	r5, r5
    1314:	2d08      	cmp	r5, #8
    1316:	d9e4      	bls.n	12e2 <_usb_d_dev_reset_epts+0x6>
	memset(prvt_inst.desc_table, 0, sizeof(UsbDeviceDescriptor) * (CONF_USB_D_MAX_EP_N + 1));
    1318:	2260      	movs	r2, #96	; 0x60
    131a:	2100      	movs	r1, #0
    131c:	4801      	ldr	r0, [pc, #4]	; (1324 <_usb_d_dev_reset_epts+0x48>)
    131e:	4b03      	ldr	r3, [pc, #12]	; (132c <_usb_d_dev_reset_epts+0x50>)
    1320:	4798      	blx	r3
}
    1322:	bd70      	pop	{r4, r5, r6, pc}
    1324:	200000a0 	.word	0x200000a0
    1328:	00001129 	.word	0x00001129
    132c:	00001e2f 	.word	0x00001e2f

00001330 <_usb_d_dev_in_next>:
{
    1330:	b5f0      	push	{r4, r5, r6, r7, lr}
    1332:	46c6      	mov	lr, r8
    1334:	b500      	push	{lr}
    1336:	0005      	movs	r5, r0
    1338:	000e      	movs	r6, r1
	uint8_t            epn         = USB_EP_GET_N(ept->ep);
    133a:	7c83      	ldrb	r3, [r0, #18]
    133c:	240f      	movs	r4, #15
    133e:	401c      	ands	r4, r3
	UsbDeviceDescBank *bank        = &prvt_inst.desc_table[epn].DeviceDescBank[0];
    1340:	0162      	lsls	r2, r4, #5
    1342:	4b56      	ldr	r3, [pc, #344]	; (149c <_usb_d_dev_in_next+0x16c>)
    1344:	189b      	adds	r3, r3, r2
	uint16_t           trans_count = isr ? bank[1].PCKSIZE.bit.BYTE_COUNT : 0;
    1346:	2900      	cmp	r1, #0
    1348:	d058      	beq.n	13fc <_usb_d_dev_in_next+0xcc>
    134a:	6959      	ldr	r1, [r3, #20]
    134c:	0489      	lsls	r1, r1, #18
    134e:	0c89      	lsrs	r1, r1, #18
	uint16_t           last_pkt = trans_count & ((ept->size == 1023) ? ept->size : (ept->size - 1));
    1350:	8a2b      	ldrh	r3, [r5, #16]
    1352:	4a53      	ldr	r2, [pc, #332]	; (14a0 <_usb_d_dev_in_next+0x170>)
    1354:	4293      	cmp	r3, r2
    1356:	d053      	beq.n	1400 <_usb_d_dev_in_next+0xd0>
    1358:	3b01      	subs	r3, #1
    135a:	b21b      	sxth	r3, r3
    135c:	400b      	ands	r3, r1
	bool               is_ctrl  = _usb_d_dev_ep_is_ctrl(ept);
    135e:	7cea      	ldrb	r2, [r5, #19]
    1360:	2707      	movs	r7, #7
    1362:	4017      	ands	r7, r2
	if (isr) {
    1364:	2e00      	cmp	r6, #0
    1366:	d007      	beq.n	1378 <_usb_d_dev_in_next+0x48>
	((UsbDevice *)hw)->DeviceEndpoint[submodule_index].EPINTFLAG.reg = mask;
    1368:	0022      	movs	r2, r4
    136a:	3208      	adds	r2, #8
    136c:	0152      	lsls	r2, r2, #5
    136e:	484d      	ldr	r0, [pc, #308]	; (14a4 <_usb_d_dev_in_next+0x174>)
    1370:	4684      	mov	ip, r0
    1372:	4462      	add	r2, ip
    1374:	2002      	movs	r0, #2
    1376:	71d0      	strb	r0, [r2, #7]
	ept->trans_count += trans_count;
    1378:	68aa      	ldr	r2, [r5, #8]
    137a:	4694      	mov	ip, r2
    137c:	4461      	add	r1, ip
    137e:	60a9      	str	r1, [r5, #8]
	if (ept->trans_count < ept->trans_size) {
    1380:	686a      	ldr	r2, [r5, #4]
    1382:	4291      	cmp	r1, r2
    1384:	d24e      	bcs.n	1424 <_usb_d_dev_in_next+0xf4>
		trans_next = ept->trans_size - ept->trans_count;
    1386:	b292      	uxth	r2, r2
    1388:	b28b      	uxth	r3, r1
    138a:	1ad2      	subs	r2, r2, r3
    138c:	b292      	uxth	r2, r2
		if (ept->flags.bits.use_cache) {
    138e:	7ceb      	ldrb	r3, [r5, #19]
    1390:	069b      	lsls	r3, r3, #26
    1392:	d537      	bpl.n	1404 <_usb_d_dev_in_next+0xd4>
			if (trans_next > ept->size) {
    1394:	8a2b      	ldrh	r3, [r5, #16]
    1396:	4698      	mov	r8, r3
    1398:	429a      	cmp	r2, r3
    139a:	d800      	bhi.n	139e <_usb_d_dev_in_next+0x6e>
		trans_next = ept->trans_size - ept->trans_count;
    139c:	4690      	mov	r8, r2
			memcpy(ept->cache, &ept->trans_buf[ept->trans_count], trans_next);
    139e:	682b      	ldr	r3, [r5, #0]
    13a0:	469c      	mov	ip, r3
    13a2:	4461      	add	r1, ip
    13a4:	4642      	mov	r2, r8
    13a6:	68e8      	ldr	r0, [r5, #12]
    13a8:	4b3f      	ldr	r3, [pc, #252]	; (14a8 <_usb_d_dev_in_next+0x178>)
    13aa:	4798      	blx	r3
			_usbd_ep_set_buf(epn, 1, (uint32_t)ept->cache);
    13ac:	68e9      	ldr	r1, [r5, #12]
	bank->ADDR.reg          = addr;
    13ae:	0162      	lsls	r2, r4, #5
    13b0:	4b3a      	ldr	r3, [pc, #232]	; (149c <_usb_d_dev_in_next+0x16c>)
    13b2:	189b      	adds	r3, r3, r2
    13b4:	6119      	str	r1, [r3, #16]
	bank->PCKSIZE.bit.BYTE_COUNT = size;
    13b6:	0163      	lsls	r3, r4, #5
    13b8:	4a38      	ldr	r2, [pc, #224]	; (149c <_usb_d_dev_in_next+0x16c>)
    13ba:	18d2      	adds	r2, r2, r3
    13bc:	6951      	ldr	r1, [r2, #20]
    13be:	4643      	mov	r3, r8
    13c0:	049b      	lsls	r3, r3, #18
    13c2:	0c9b      	lsrs	r3, r3, #18
    13c4:	0b89      	lsrs	r1, r1, #14
    13c6:	0389      	lsls	r1, r1, #14
    13c8:	430b      	orrs	r3, r1
    13ca:	6153      	str	r3, [r2, #20]
	bank->PCKSIZE.bit.MULTI_PACKET_SIZE = count;
    13cc:	6951      	ldr	r1, [r2, #20]
    13ce:	4b37      	ldr	r3, [pc, #220]	; (14ac <_usb_d_dev_in_next+0x17c>)
    13d0:	400b      	ands	r3, r1
    13d2:	6153      	str	r3, [r2, #20]
	if (!isr) {
    13d4:	2e00      	cmp	r6, #0
    13d6:	d107      	bne.n	13e8 <_usb_d_dev_in_next+0xb8>
		if (is_ctrl) {
    13d8:	2f01      	cmp	r7, #1
    13da:	d05d      	beq.n	1498 <_usb_d_dev_in_next+0x168>
			inten = USB_D_BANK1_INT_FLAGS;
    13dc:	224a      	movs	r2, #74	; 0x4a
	((UsbDevice *)hw)->DeviceEndpoint[submodule_index].EPINTENSET.reg = mask;
    13de:	0163      	lsls	r3, r4, #5
    13e0:	4933      	ldr	r1, [pc, #204]	; (14b0 <_usb_d_dev_in_next+0x180>)
    13e2:	468c      	mov	ip, r1
    13e4:	4463      	add	r3, ip
    13e6:	701a      	strb	r2, [r3, #0]
	((UsbDevice *)hw)->DeviceEndpoint[submodule_index].EPSTATUSSET.reg = mask;
    13e8:	3408      	adds	r4, #8
    13ea:	0164      	lsls	r4, r4, #5
    13ec:	4b2d      	ldr	r3, [pc, #180]	; (14a4 <_usb_d_dev_in_next+0x174>)
    13ee:	469c      	mov	ip, r3
    13f0:	4464      	add	r4, ip
    13f2:	2380      	movs	r3, #128	; 0x80
    13f4:	7163      	strb	r3, [r4, #5]
}
    13f6:	bc04      	pop	{r2}
    13f8:	4690      	mov	r8, r2
    13fa:	bdf0      	pop	{r4, r5, r6, r7, pc}
	uint16_t           trans_count = isr ? bank[1].PCKSIZE.bit.BYTE_COUNT : 0;
    13fc:	2100      	movs	r1, #0
    13fe:	e7a7      	b.n	1350 <_usb_d_dev_in_next+0x20>
	uint16_t           last_pkt = trans_count & ((ept->size == 1023) ? ept->size : (ept->size - 1));
    1400:	b21b      	sxth	r3, r3
    1402:	e7ab      	b.n	135c <_usb_d_dev_in_next+0x2c>
			if (trans_next > USB_D_DEV_TRANS_MAX) {
    1404:	2380      	movs	r3, #128	; 0x80
    1406:	019b      	lsls	r3, r3, #6
    1408:	429a      	cmp	r2, r3
    140a:	d807      	bhi.n	141c <_usb_d_dev_in_next+0xec>
		trans_next = ept->trans_size - ept->trans_count;
    140c:	4690      	mov	r8, r2
			_usbd_ep_set_buf(epn, 1, (uint32_t)&ept->trans_buf[ept->trans_count]);
    140e:	682b      	ldr	r3, [r5, #0]
    1410:	1859      	adds	r1, r3, r1
	bank->ADDR.reg          = addr;
    1412:	0162      	lsls	r2, r4, #5
    1414:	4b21      	ldr	r3, [pc, #132]	; (149c <_usb_d_dev_in_next+0x16c>)
    1416:	189b      	adds	r3, r3, r2
    1418:	6119      	str	r1, [r3, #16]
    141a:	e7cc      	b.n	13b6 <_usb_d_dev_in_next+0x86>
				trans_next = USB_D_DEV_TRANS_MAX;
    141c:	2380      	movs	r3, #128	; 0x80
    141e:	019b      	lsls	r3, r3, #6
    1420:	4698      	mov	r8, r3
    1422:	e7f4      	b.n	140e <_usb_d_dev_in_next+0xde>
	} else if (ept->flags.bits.need_zlp) {
    1424:	7cea      	ldrb	r2, [r5, #19]
    1426:	06d2      	lsls	r2, r2, #27
    1428:	d50f      	bpl.n	144a <_usb_d_dev_in_next+0x11a>
		ept->flags.bits.need_zlp = 0;
    142a:	7ceb      	ldrb	r3, [r5, #19]
    142c:	2210      	movs	r2, #16
    142e:	4393      	bics	r3, r2
    1430:	74eb      	strb	r3, [r5, #19]
	bank->PCKSIZE.bit.BYTE_COUNT = size;
    1432:	0162      	lsls	r2, r4, #5
    1434:	4b19      	ldr	r3, [pc, #100]	; (149c <_usb_d_dev_in_next+0x16c>)
    1436:	189b      	adds	r3, r3, r2
    1438:	695a      	ldr	r2, [r3, #20]
    143a:	0b92      	lsrs	r2, r2, #14
    143c:	0391      	lsls	r1, r2, #14
    143e:	6159      	str	r1, [r3, #20]
	bank->PCKSIZE.bit.MULTI_PACKET_SIZE = count;
    1440:	6959      	ldr	r1, [r3, #20]
    1442:	4a1a      	ldr	r2, [pc, #104]	; (14ac <_usb_d_dev_in_next+0x17c>)
    1444:	400a      	ands	r2, r1
    1446:	615a      	str	r2, [r3, #20]
    1448:	e7c4      	b.n	13d4 <_usb_d_dev_in_next+0xa4>
	if (is_ctrl) {
    144a:	2f01      	cmp	r7, #1
    144c:	d00d      	beq.n	146a <_usb_d_dev_in_next+0x13a>
	((UsbDevice *)hw)->DeviceEndpoint[submodule_index].EPINTENCLR.reg = mask;
    144e:	0164      	lsls	r4, r4, #5
    1450:	4a18      	ldr	r2, [pc, #96]	; (14b4 <_usb_d_dev_in_next+0x184>)
    1452:	4694      	mov	ip, r2
    1454:	4464      	add	r4, ip
    1456:	224a      	movs	r2, #74	; 0x4a
    1458:	7022      	strb	r2, [r4, #0]
	if (last_pkt == ept->size) {
    145a:	8a2a      	ldrh	r2, [r5, #16]
    145c:	4293      	cmp	r3, r2
    145e:	d00b      	beq.n	1478 <_usb_d_dev_in_next+0x148>
	_usb_d_dev_trans_done(ept, USB_TRANS_DONE);
    1460:	2100      	movs	r1, #0
    1462:	0028      	movs	r0, r5
    1464:	4b14      	ldr	r3, [pc, #80]	; (14b8 <_usb_d_dev_in_next+0x188>)
    1466:	4798      	blx	r3
	return;
    1468:	e7c5      	b.n	13f6 <_usb_d_dev_in_next+0xc6>
    146a:	0164      	lsls	r4, r4, #5
    146c:	4a11      	ldr	r2, [pc, #68]	; (14b4 <_usb_d_dev_in_next+0x184>)
    146e:	4694      	mov	ip, r2
    1470:	4464      	add	r4, ip
    1472:	224b      	movs	r2, #75	; 0x4b
    1474:	7022      	strb	r2, [r4, #0]
    1476:	e7f0      	b.n	145a <_usb_d_dev_in_next+0x12a>
		ept->flags.bits.is_busy = 0;
    1478:	7ceb      	ldrb	r3, [r5, #19]
    147a:	2240      	movs	r2, #64	; 0x40
    147c:	4393      	bics	r3, r2
    147e:	74eb      	strb	r3, [r5, #19]
		if (dev_inst.ep_callbacks.more(ept->ep, ept->trans_count)) {
    1480:	4b06      	ldr	r3, [pc, #24]	; (149c <_usb_d_dev_in_next+0x16c>)
    1482:	6edb      	ldr	r3, [r3, #108]	; 0x6c
    1484:	7ca8      	ldrb	r0, [r5, #18]
    1486:	68a9      	ldr	r1, [r5, #8]
    1488:	4798      	blx	r3
    148a:	2800      	cmp	r0, #0
    148c:	d1b3      	bne.n	13f6 <_usb_d_dev_in_next+0xc6>
		ept->flags.bits.is_busy = 1;
    148e:	7ceb      	ldrb	r3, [r5, #19]
    1490:	2240      	movs	r2, #64	; 0x40
    1492:	4313      	orrs	r3, r2
    1494:	74eb      	strb	r3, [r5, #19]
    1496:	e7e3      	b.n	1460 <_usb_d_dev_in_next+0x130>
			inten = USB_D_BANK1_INT_FLAGS | USB_DEVICE_EPINTFLAG_TRFAIL0;
    1498:	224e      	movs	r2, #78	; 0x4e
    149a:	e7a0      	b.n	13de <_usb_d_dev_in_next+0xae>
    149c:	200000a0 	.word	0x200000a0
    14a0:	000003ff 	.word	0x000003ff
    14a4:	41005000 	.word	0x41005000
    14a8:	00001e1d 	.word	0x00001e1d
    14ac:	f0003fff 	.word	0xf0003fff
    14b0:	41005109 	.word	0x41005109
    14b4:	41005108 	.word	0x41005108
    14b8:	00001129 	.word	0x00001129

000014bc <_usb_d_dev_out_next>:
{
    14bc:	b5f8      	push	{r3, r4, r5, r6, r7, lr}
    14be:	46de      	mov	lr, fp
    14c0:	4657      	mov	r7, sl
    14c2:	464e      	mov	r6, r9
    14c4:	4645      	mov	r5, r8
    14c6:	b5e0      	push	{r5, r6, r7, lr}
    14c8:	0004      	movs	r4, r0
    14ca:	000f      	movs	r7, r1
	uint8_t            epn        = USB_EP_GET_N(ept->ep);
    14cc:	7c83      	ldrb	r3, [r0, #18]
    14ce:	250f      	movs	r5, #15
    14d0:	401d      	ands	r5, r3
	uint16_t           trans_size = isr ? bank->PCKSIZE.bit.MULTI_PACKET_SIZE : 0;
    14d2:	2900      	cmp	r1, #0
    14d4:	d059      	beq.n	158a <_usb_d_dev_out_next+0xce>
    14d6:	016a      	lsls	r2, r5, #5
    14d8:	4b71      	ldr	r3, [pc, #452]	; (16a0 <_usb_d_dev_out_next+0x1e4>)
    14da:	189b      	adds	r3, r3, r2
    14dc:	685b      	ldr	r3, [r3, #4]
    14de:	011b      	lsls	r3, r3, #4
    14e0:	0c9b      	lsrs	r3, r3, #18
    14e2:	469a      	mov	sl, r3
	uint16_t           last_trans = isr ? bank->PCKSIZE.bit.BYTE_COUNT : 0;
    14e4:	2f00      	cmp	r7, #0
    14e6:	d053      	beq.n	1590 <_usb_d_dev_out_next+0xd4>
    14e8:	016a      	lsls	r2, r5, #5
    14ea:	4b6d      	ldr	r3, [pc, #436]	; (16a0 <_usb_d_dev_out_next+0x1e4>)
    14ec:	189b      	adds	r3, r3, r2
    14ee:	685b      	ldr	r3, [r3, #4]
    14f0:	049b      	lsls	r3, r3, #18
    14f2:	0c9b      	lsrs	r3, r3, #18
    14f4:	4698      	mov	r8, r3
	uint16_t           size_mask  = (ept->size == 1023) ? 1023 : (ept->size - 1);
    14f6:	8a26      	ldrh	r6, [r4, #16]
    14f8:	4b6a      	ldr	r3, [pc, #424]	; (16a4 <_usb_d_dev_out_next+0x1e8>)
    14fa:	429e      	cmp	r6, r3
    14fc:	d001      	beq.n	1502 <_usb_d_dev_out_next+0x46>
    14fe:	3e01      	subs	r6, #1
    1500:	b2b6      	uxth	r6, r6
	uint16_t           last_pkt   = last_trans & size_mask;
    1502:	4643      	mov	r3, r8
    1504:	4033      	ands	r3, r6
    1506:	469b      	mov	fp, r3
	bool               is_ctrl = _usb_d_dev_ep_is_ctrl(ept);
    1508:	7ce3      	ldrb	r3, [r4, #19]
    150a:	2207      	movs	r2, #7
    150c:	401a      	ands	r2, r3
    150e:	4691      	mov	r9, r2
	if (isr) {
    1510:	2f00      	cmp	r7, #0
    1512:	d007      	beq.n	1524 <_usb_d_dev_out_next+0x68>
	((UsbDevice *)hw)->DeviceEndpoint[submodule_index].EPINTFLAG.reg = mask;
    1514:	002b      	movs	r3, r5
    1516:	3308      	adds	r3, #8
    1518:	015b      	lsls	r3, r3, #5
    151a:	4a63      	ldr	r2, [pc, #396]	; (16a8 <_usb_d_dev_out_next+0x1ec>)
    151c:	4694      	mov	ip, r2
    151e:	4463      	add	r3, ip
    1520:	2201      	movs	r2, #1
    1522:	71da      	strb	r2, [r3, #7]
	if (ept->flags.bits.use_cache && ept->trans_size) {
    1524:	7ce3      	ldrb	r3, [r4, #19]
    1526:	069b      	lsls	r3, r3, #26
    1528:	d511      	bpl.n	154e <_usb_d_dev_out_next+0x92>
    152a:	6862      	ldr	r2, [r4, #4]
    152c:	2a00      	cmp	r2, #0
    152e:	d00e      	beq.n	154e <_usb_d_dev_out_next+0x92>
		uint16_t buf_remain = ept->trans_size - ept->trans_count;
    1530:	b292      	uxth	r2, r2
    1532:	8923      	ldrh	r3, [r4, #8]
    1534:	1ad2      	subs	r2, r2, r3
    1536:	b292      	uxth	r2, r2
		memcpy(&ept->trans_buf[ept->trans_count], ept->cache, (buf_remain > last_pkt) ? last_pkt : buf_remain);
    1538:	6823      	ldr	r3, [r4, #0]
    153a:	68a1      	ldr	r1, [r4, #8]
    153c:	468c      	mov	ip, r1
    153e:	4463      	add	r3, ip
    1540:	0018      	movs	r0, r3
    1542:	68e1      	ldr	r1, [r4, #12]
    1544:	4593      	cmp	fp, r2
    1546:	d200      	bcs.n	154a <_usb_d_dev_out_next+0x8e>
    1548:	465a      	mov	r2, fp
    154a:	4b58      	ldr	r3, [pc, #352]	; (16ac <_usb_d_dev_out_next+0x1f0>)
    154c:	4798      	blx	r3
	if (ept->trans_size == 0 && ept->flags.bits.need_zlp) {
    154e:	6863      	ldr	r3, [r4, #4]
    1550:	2b00      	cmp	r3, #0
    1552:	d120      	bne.n	1596 <_usb_d_dev_out_next+0xda>
    1554:	7ce2      	ldrb	r2, [r4, #19]
    1556:	06d2      	lsls	r2, r2, #27
    1558:	d51d      	bpl.n	1596 <_usb_d_dev_out_next+0xda>
		ept->flags.bits.need_zlp  = 0;
    155a:	7ce3      	ldrb	r3, [r4, #19]
		ept->flags.bits.use_cache = 1;
    155c:	2210      	movs	r2, #16
    155e:	4393      	bics	r3, r2
    1560:	2220      	movs	r2, #32
    1562:	4313      	orrs	r3, r2
    1564:	74e3      	strb	r3, [r4, #19]
	bank->ADDR.reg          = addr;
    1566:	494e      	ldr	r1, [pc, #312]	; (16a0 <_usb_d_dev_out_next+0x1e4>)
    1568:	016a      	lsls	r2, r5, #5
    156a:	68e3      	ldr	r3, [r4, #12]
    156c:	5053      	str	r3, [r2, r1]
		_usbd_ep_set_out_trans(epn, 0, ept->size, 0);
    156e:	8a23      	ldrh	r3, [r4, #16]
	bank->PCKSIZE.bit.MULTI_PACKET_SIZE = size;
    1570:	188a      	adds	r2, r1, r2
    1572:	6851      	ldr	r1, [r2, #4]
    1574:	049b      	lsls	r3, r3, #18
    1576:	091b      	lsrs	r3, r3, #4
    1578:	484d      	ldr	r0, [pc, #308]	; (16b0 <_usb_d_dev_out_next+0x1f4>)
    157a:	4001      	ands	r1, r0
    157c:	430b      	orrs	r3, r1
    157e:	6053      	str	r3, [r2, #4]
	bank->PCKSIZE.bit.BYTE_COUNT = count;
    1580:	6853      	ldr	r3, [r2, #4]
    1582:	0b9b      	lsrs	r3, r3, #14
    1584:	0399      	lsls	r1, r3, #14
    1586:	6051      	str	r1, [r2, #4]
    1588:	e047      	b.n	161a <_usb_d_dev_out_next+0x15e>
	uint16_t           trans_size = isr ? bank->PCKSIZE.bit.MULTI_PACKET_SIZE : 0;
    158a:	2300      	movs	r3, #0
    158c:	469a      	mov	sl, r3
    158e:	e7a9      	b.n	14e4 <_usb_d_dev_out_next+0x28>
	uint16_t           last_trans = isr ? bank->PCKSIZE.bit.BYTE_COUNT : 0;
    1590:	2300      	movs	r3, #0
    1592:	4698      	mov	r8, r3
    1594:	e7af      	b.n	14f6 <_usb_d_dev_out_next+0x3a>
	} else if (isr && last_pkt < ept->size) {
    1596:	2f00      	cmp	r7, #0
    1598:	d01d      	beq.n	15d6 <_usb_d_dev_out_next+0x11a>
    159a:	8a22      	ldrh	r2, [r4, #16]
    159c:	4593      	cmp	fp, r2
    159e:	d21a      	bcs.n	15d6 <_usb_d_dev_out_next+0x11a>
		ept->flags.bits.need_zlp = 0;
    15a0:	7ce3      	ldrb	r3, [r4, #19]
    15a2:	2210      	movs	r2, #16
    15a4:	4393      	bics	r3, r2
    15a6:	74e3      	strb	r3, [r4, #19]
		ept->trans_count += last_trans;
    15a8:	68a3      	ldr	r3, [r4, #8]
    15aa:	4443      	add	r3, r8
    15ac:	60a3      	str	r3, [r4, #8]
	if (is_ctrl) {
    15ae:	464b      	mov	r3, r9
    15b0:	2b01      	cmp	r3, #1
    15b2:	d066      	beq.n	1682 <_usb_d_dev_out_next+0x1c6>
	((UsbDevice *)hw)->DeviceEndpoint[submodule_index].EPINTENCLR.reg = mask;
    15b4:	016b      	lsls	r3, r5, #5
    15b6:	4a3f      	ldr	r2, [pc, #252]	; (16b4 <_usb_d_dev_out_next+0x1f8>)
    15b8:	4694      	mov	ip, r2
    15ba:	4463      	add	r3, ip
    15bc:	2225      	movs	r2, #37	; 0x25
    15be:	701a      	strb	r2, [r3, #0]
	if (0 == epn) {
    15c0:	2d00      	cmp	r5, #0
    15c2:	d103      	bne.n	15cc <_usb_d_dev_out_next+0x110>
	bank->ADDR.reg          = addr;
    15c4:	016d      	lsls	r5, r5, #5
    15c6:	4b36      	ldr	r3, [pc, #216]	; (16a0 <_usb_d_dev_out_next+0x1e4>)
    15c8:	68e2      	ldr	r2, [r4, #12]
    15ca:	50ea      	str	r2, [r5, r3]
	_usb_d_dev_trans_done(ept, USB_TRANS_DONE);
    15cc:	2100      	movs	r1, #0
    15ce:	0020      	movs	r0, r4
    15d0:	4b39      	ldr	r3, [pc, #228]	; (16b8 <_usb_d_dev_out_next+0x1fc>)
    15d2:	4798      	blx	r3
	return;
    15d4:	e033      	b.n	163e <_usb_d_dev_out_next+0x182>
		ept->trans_count += trans_size;
    15d6:	68a2      	ldr	r2, [r4, #8]
    15d8:	4452      	add	r2, sl
    15da:	60a2      	str	r2, [r4, #8]
		if (ept->trans_count < ept->trans_size) {
    15dc:	4293      	cmp	r3, r2
    15de:	d9e6      	bls.n	15ae <_usb_d_dev_out_next+0xf2>
			trans_next = ept->trans_size - ept->trans_count;
    15e0:	b29b      	uxth	r3, r3
    15e2:	b291      	uxth	r1, r2
    15e4:	1a5b      	subs	r3, r3, r1
    15e6:	b29b      	uxth	r3, r3
			if (ept->flags.bits.use_cache) {
    15e8:	7ce1      	ldrb	r1, [r4, #19]
    15ea:	0689      	lsls	r1, r1, #26
    15ec:	d52d      	bpl.n	164a <_usb_d_dev_out_next+0x18e>
				if (trans_next > ept->size) {
    15ee:	8a21      	ldrh	r1, [r4, #16]
    15f0:	428b      	cmp	r3, r1
    15f2:	d800      	bhi.n	15f6 <_usb_d_dev_out_next+0x13a>
			trans_next = ept->trans_size - ept->trans_count;
    15f4:	0019      	movs	r1, r3
				_usbd_ep_set_buf(epn, 0, (uint32_t)ept->cache);
    15f6:	68e0      	ldr	r0, [r4, #12]
	bank->ADDR.reg          = addr;
    15f8:	016b      	lsls	r3, r5, #5
    15fa:	4a29      	ldr	r2, [pc, #164]	; (16a0 <_usb_d_dev_out_next+0x1e4>)
    15fc:	5098      	str	r0, [r3, r2]
	bank->PCKSIZE.bit.MULTI_PACKET_SIZE = size;
    15fe:	016b      	lsls	r3, r5, #5
    1600:	4827      	ldr	r0, [pc, #156]	; (16a0 <_usb_d_dev_out_next+0x1e4>)
    1602:	18c0      	adds	r0, r0, r3
    1604:	6842      	ldr	r2, [r0, #4]
    1606:	048b      	lsls	r3, r1, #18
    1608:	091b      	lsrs	r3, r3, #4
    160a:	4929      	ldr	r1, [pc, #164]	; (16b0 <_usb_d_dev_out_next+0x1f4>)
    160c:	400a      	ands	r2, r1
    160e:	4313      	orrs	r3, r2
    1610:	6043      	str	r3, [r0, #4]
	bank->PCKSIZE.bit.BYTE_COUNT = count;
    1612:	6843      	ldr	r3, [r0, #4]
    1614:	0b9b      	lsrs	r3, r3, #14
    1616:	039a      	lsls	r2, r3, #14
    1618:	6042      	str	r2, [r0, #4]
	if (!isr) {
    161a:	2f00      	cmp	r7, #0
    161c:	d108      	bne.n	1630 <_usb_d_dev_out_next+0x174>
		if (is_ctrl) {
    161e:	464b      	mov	r3, r9
    1620:	2b01      	cmp	r3, #1
    1622:	d035      	beq.n	1690 <_usb_d_dev_out_next+0x1d4>
			inten = USB_D_BANK0_INT_FLAGS;
    1624:	2225      	movs	r2, #37	; 0x25
	((UsbDevice *)hw)->DeviceEndpoint[submodule_index].EPINTENSET.reg = mask;
    1626:	016b      	lsls	r3, r5, #5
    1628:	4924      	ldr	r1, [pc, #144]	; (16bc <_usb_d_dev_out_next+0x200>)
    162a:	468c      	mov	ip, r1
    162c:	4463      	add	r3, ip
    162e:	701a      	strb	r2, [r3, #0]
	((UsbDevice *)hw)->DeviceEndpoint[submodule_index].EPSTATUSCLR.reg = mask;
    1630:	3508      	adds	r5, #8
    1632:	016d      	lsls	r5, r5, #5
    1634:	4b1c      	ldr	r3, [pc, #112]	; (16a8 <_usb_d_dev_out_next+0x1ec>)
    1636:	469c      	mov	ip, r3
    1638:	4465      	add	r5, ip
    163a:	2340      	movs	r3, #64	; 0x40
    163c:	712b      	strb	r3, [r5, #4]
}
    163e:	bc3c      	pop	{r2, r3, r4, r5}
    1640:	4690      	mov	r8, r2
    1642:	4699      	mov	r9, r3
    1644:	46a2      	mov	sl, r4
    1646:	46ab      	mov	fp, r5
    1648:	bdf8      	pop	{r3, r4, r5, r6, r7, pc}
				if (trans_next > ept->size) {
    164a:	8a21      	ldrh	r1, [r4, #16]
    164c:	428b      	cmp	r3, r1
    164e:	d90b      	bls.n	1668 <_usb_d_dev_out_next+0x1ac>
					if (trans_next > USB_D_DEV_TRANS_MAX) {
    1650:	2180      	movs	r1, #128	; 0x80
    1652:	0189      	lsls	r1, r1, #6
    1654:	428b      	cmp	r3, r1
    1656:	d80f      	bhi.n	1678 <_usb_d_dev_out_next+0x1bc>
    1658:	43b3      	bics	r3, r6
    165a:	0019      	movs	r1, r3
				_usbd_ep_set_buf(epn, 0, (uint32_t)&ept->trans_buf[ept->trans_count]);
    165c:	6823      	ldr	r3, [r4, #0]
    165e:	189a      	adds	r2, r3, r2
	bank->ADDR.reg          = addr;
    1660:	016b      	lsls	r3, r5, #5
    1662:	480f      	ldr	r0, [pc, #60]	; (16a0 <_usb_d_dev_out_next+0x1e4>)
    1664:	501a      	str	r2, [r3, r0]
    1666:	e7ca      	b.n	15fe <_usb_d_dev_out_next+0x142>
				} else if (trans_next < ept->size) {
    1668:	428b      	cmp	r3, r1
    166a:	d208      	bcs.n	167e <_usb_d_dev_out_next+0x1c2>
					ept->flags.bits.use_cache = 1;
    166c:	7ce1      	ldrb	r1, [r4, #19]
    166e:	2020      	movs	r0, #32
    1670:	4301      	orrs	r1, r0
    1672:	74e1      	strb	r1, [r4, #19]
			trans_next = ept->trans_size - ept->trans_count;
    1674:	0019      	movs	r1, r3
    1676:	e7f1      	b.n	165c <_usb_d_dev_out_next+0x1a0>
						trans_next = USB_D_DEV_TRANS_MAX;
    1678:	2180      	movs	r1, #128	; 0x80
    167a:	0189      	lsls	r1, r1, #6
    167c:	e7ee      	b.n	165c <_usb_d_dev_out_next+0x1a0>
			trans_next = ept->trans_size - ept->trans_count;
    167e:	0019      	movs	r1, r3
    1680:	e7ec      	b.n	165c <_usb_d_dev_out_next+0x1a0>
	((UsbDevice *)hw)->DeviceEndpoint[submodule_index].EPINTENCLR.reg = mask;
    1682:	016b      	lsls	r3, r5, #5
    1684:	4a0b      	ldr	r2, [pc, #44]	; (16b4 <_usb_d_dev_out_next+0x1f8>)
    1686:	4694      	mov	ip, r2
    1688:	4463      	add	r3, ip
    168a:	222d      	movs	r2, #45	; 0x2d
    168c:	701a      	strb	r2, [r3, #0]
    168e:	e797      	b.n	15c0 <_usb_d_dev_out_next+0x104>
	bank->STATUS_BK.reg     = 0;
    1690:	016a      	lsls	r2, r5, #5
    1692:	4b03      	ldr	r3, [pc, #12]	; (16a0 <_usb_d_dev_out_next+0x1e4>)
    1694:	189b      	adds	r3, r3, r2
    1696:	2200      	movs	r2, #0
    1698:	769a      	strb	r2, [r3, #26]
			inten = USB_D_BANK0_INT_FLAGS | USB_DEVICE_EPINTFLAG_TRFAIL1;
    169a:	322d      	adds	r2, #45	; 0x2d
    169c:	e7c3      	b.n	1626 <_usb_d_dev_out_next+0x16a>
    169e:	46c0      	nop			; (mov r8, r8)
    16a0:	200000a0 	.word	0x200000a0
    16a4:	000003ff 	.word	0x000003ff
    16a8:	41005000 	.word	0x41005000
    16ac:	00001e1d 	.word	0x00001e1d
    16b0:	f0003fff 	.word	0xf0003fff
    16b4:	41005108 	.word	0x41005108
    16b8:	00001129 	.word	0x00001129
    16bc:	41005109 	.word	0x41005109

000016c0 <_usb_d_dev_handler>:
{
    16c0:	b570      	push	{r4, r5, r6, lr}
	uint16_t epint = hw->DEVICE.EPINTSMRY.reg;
    16c2:	4b89      	ldr	r3, [pc, #548]	; (18e8 <_usb_d_dev_handler+0x228>)
    16c4:	8c1d      	ldrh	r5, [r3, #32]
    16c6:	b2ad      	uxth	r5, r5
	if (0 == epint) {
    16c8:	2d00      	cmp	r5, #0
    16ca:	d001      	beq.n	16d0 <_usb_d_dev_handler+0x10>
	bool     rc    = true;
    16cc:	2400      	movs	r4, #0
    16ce:	e0bf      	b.n	1850 <_usb_d_dev_handler+0x190>
	return tmp;
}

static inline hri_usbdevice_intflag_reg_t hri_usbdevice_read_INTFLAG_reg(const void *const hw)
{
	return ((Usb *)hw)->DEVICE.INTFLAG.reg;
    16d0:	8b99      	ldrh	r1, [r3, #28]
	return tmp;
}

static inline hri_usbdevice_intenset_reg_t hri_usbdevice_read_INTEN_reg(const void *const hw)
{
	return ((Usb *)hw)->DEVICE.INTENSET.reg;
    16d2:	8b1b      	ldrh	r3, [r3, #24]
	flags &= hri_usbdevice_read_INTEN_reg(USB);
    16d4:	400b      	ands	r3, r1
	if (flags & USB_DEVICE_INTFLAG_SOF) {
    16d6:	075a      	lsls	r2, r3, #29
    16d8:	d40d      	bmi.n	16f6 <_usb_d_dev_handler+0x36>
	if (flags & USB_DEVICE_INTFLAG_LPMSUSP) {
    16da:	059a      	lsls	r2, r3, #22
    16dc:	d415      	bmi.n	170a <_usb_d_dev_handler+0x4a>
	} else if (flags & USB_DEVICE_INTFLAG_RAMACER) {
    16de:	061a      	lsls	r2, r3, #24
    16e0:	d437      	bmi.n	1752 <_usb_d_dev_handler+0x92>
	} else if (flags & USB_D_WAKEUP_INT_FLAGS) {
    16e2:	2270      	movs	r2, #112	; 0x70
    16e4:	421a      	tst	r2, r3
    16e6:	d13e      	bne.n	1766 <_usb_d_dev_handler+0xa6>
	} else if (flags & USB_DEVICE_INTFLAG_EORST) {
    16e8:	071a      	lsls	r2, r3, #28
    16ea:	d457      	bmi.n	179c <_usb_d_dev_handler+0xdc>
	} else if (flags & USB_DEVICE_INTFLAG_SUSPEND) {
    16ec:	07db      	lsls	r3, r3, #31
    16ee:	d500      	bpl.n	16f2 <_usb_d_dev_handler+0x32>
    16f0:	e068      	b.n	17c4 <_usb_d_dev_handler+0x104>
		rc = false;
    16f2:	2300      	movs	r3, #0
    16f4:	e006      	b.n	1704 <_usb_d_dev_handler+0x44>
	((Usb *)hw)->DEVICE.INTFLAG.reg = mask;
    16f6:	2204      	movs	r2, #4
    16f8:	4b7b      	ldr	r3, [pc, #492]	; (18e8 <_usb_d_dev_handler+0x228>)
    16fa:	839a      	strh	r2, [r3, #28]
	dev_inst.callbacks.sof();
    16fc:	4b7b      	ldr	r3, [pc, #492]	; (18ec <_usb_d_dev_handler+0x22c>)
    16fe:	6e1b      	ldr	r3, [r3, #96]	; 0x60
    1700:	4798      	blx	r3
		return true;
    1702:	2301      	movs	r3, #1
		if (_usb_d_dev_handle_nep()) {
    1704:	2b00      	cmp	r3, #0
    1706:	d0e1      	beq.n	16cc <_usb_d_dev_handler+0xc>
}
    1708:	bd70      	pop	{r4, r5, r6, pc}
    170a:	4b77      	ldr	r3, [pc, #476]	; (18e8 <_usb_d_dev_handler+0x228>)
    170c:	4a78      	ldr	r2, [pc, #480]	; (18f0 <_usb_d_dev_handler+0x230>)
    170e:	839a      	strh	r2, [r3, #28]
	((Usb *)hw)->DEVICE.INTENCLR.reg = ~data;
}

static inline void hri_usbdevice_clear_INTEN_reg(const void *const hw, hri_usbdevice_intenset_reg_t mask)
{
	((Usb *)hw)->DEVICE.INTENCLR.reg = mask;
    1710:	829a      	strh	r2, [r3, #20]
	((Usb *)hw)->DEVICE.INTENSET.reg = mask;
    1712:	3a92      	subs	r2, #146	; 0x92
    1714:	3aff      	subs	r2, #255	; 0xff
    1716:	831a      	strh	r2, [r3, #24]
	for (i = 0; i < CONF_USB_D_MAX_EP_N; i++) {
    1718:	2300      	movs	r3, #0
    171a:	2b01      	cmp	r3, #1
    171c:	d812      	bhi.n	1744 <_usb_d_dev_handler+0x84>
		if (bank->EXTREG.bit.SUBPID == 0x3) {
    171e:	0158      	lsls	r0, r3, #5
    1720:	4a72      	ldr	r2, [pc, #456]	; (18ec <_usb_d_dev_handler+0x22c>)
    1722:	1812      	adds	r2, r2, r0
    1724:	8912      	ldrh	r2, [r2, #8]
    1726:	0712      	lsls	r2, r2, #28
    1728:	0f12      	lsrs	r2, r2, #28
    172a:	2a03      	cmp	r2, #3
    172c:	d002      	beq.n	1734 <_usb_d_dev_handler+0x74>
	for (i = 0; i < CONF_USB_D_MAX_EP_N; i++) {
    172e:	3301      	adds	r3, #1
    1730:	b2db      	uxtb	r3, r3
    1732:	e7f2      	b.n	171a <_usb_d_dev_handler+0x5a>
			lpm_variable = bank->EXTREG.bit.VARIABLE;
    1734:	4b6d      	ldr	r3, [pc, #436]	; (18ec <_usb_d_dev_handler+0x22c>)
    1736:	181b      	adds	r3, r3, r0
    1738:	8919      	ldrh	r1, [r3, #8]
    173a:	0449      	lsls	r1, r1, #17
    173c:	0d49      	lsrs	r1, r1, #21
			bank->EXTREG.reg = 0;
    173e:	2200      	movs	r2, #0
    1740:	811a      	strh	r2, [r3, #8]
    1742:	e000      	b.n	1746 <_usb_d_dev_handler+0x86>
	uint32_t lpm_variable = 0;
    1744:	2100      	movs	r1, #0
	dev_inst.callbacks.event(USB_EV_LPM_SUSPEND, lpm_variable);
    1746:	4b69      	ldr	r3, [pc, #420]	; (18ec <_usb_d_dev_handler+0x22c>)
    1748:	6e5b      	ldr	r3, [r3, #100]	; 0x64
    174a:	2003      	movs	r0, #3
    174c:	4798      	blx	r3
	bool     rc    = true;
    174e:	2301      	movs	r3, #1
    1750:	e7d8      	b.n	1704 <_usb_d_dev_handler+0x44>
	((Usb *)hw)->DEVICE.INTFLAG.reg = mask;
    1752:	2280      	movs	r2, #128	; 0x80
    1754:	4b64      	ldr	r3, [pc, #400]	; (18e8 <_usb_d_dev_handler+0x228>)
    1756:	839a      	strh	r2, [r3, #28]
	dev_inst.callbacks.event(USB_EV_ERROR, 0);
    1758:	4b64      	ldr	r3, [pc, #400]	; (18ec <_usb_d_dev_handler+0x22c>)
    175a:	6e5b      	ldr	r3, [r3, #100]	; 0x64
    175c:	2100      	movs	r1, #0
    175e:	2005      	movs	r0, #5
    1760:	4798      	blx	r3
	bool     rc    = true;
    1762:	2301      	movs	r3, #1
    1764:	e7ce      	b.n	1704 <_usb_d_dev_handler+0x44>
    1766:	4b60      	ldr	r3, [pc, #384]	; (18e8 <_usb_d_dev_handler+0x228>)
    1768:	839a      	strh	r2, [r3, #28]
	((Usb *)hw)->DEVICE.INTENCLR.reg = mask;
    176a:	829a      	strh	r2, [r3, #20]
	((Usb *)hw)->DEVICE.INTENSET.reg = mask;
    176c:	4a60      	ldr	r2, [pc, #384]	; (18f0 <_usb_d_dev_handler+0x230>)
    176e:	831a      	strh	r2, [r3, #24]
	if (!(SYSCTRL->DFLLCTRL.reg & SYSCTRL_DFLLCTRL_USBCRM)) {
    1770:	4b60      	ldr	r3, [pc, #384]	; (18f4 <_usb_d_dev_handler+0x234>)
    1772:	8c9b      	ldrh	r3, [r3, #36]	; 0x24
    1774:	069b      	lsls	r3, r3, #26
    1776:	d40c      	bmi.n	1792 <_usb_d_dev_handler+0xd2>
	tmp = ((Sysctrl *)hw)->PCLKSR.reg;
    1778:	4b5e      	ldr	r3, [pc, #376]	; (18f4 <_usb_d_dev_handler+0x234>)
    177a:	68da      	ldr	r2, [r3, #12]
	tmp &= mask;
    177c:	23d0      	movs	r3, #208	; 0xd0
    177e:	4013      	ands	r3, r2
		while (hri_sysctrl_get_PCLKSR_reg(SYSCTRL, DFLL_READY_FLAG) != DFLL_READY_FLAG)
    1780:	2bd0      	cmp	r3, #208	; 0xd0
    1782:	d1f9      	bne.n	1778 <_usb_d_dev_handler+0xb8>
	dev_inst.callbacks.event(USB_EV_WAKEUP, 0);
    1784:	4b59      	ldr	r3, [pc, #356]	; (18ec <_usb_d_dev_handler+0x22c>)
    1786:	6e5b      	ldr	r3, [r3, #100]	; 0x64
    1788:	2100      	movs	r1, #0
    178a:	2002      	movs	r0, #2
    178c:	4798      	blx	r3
	bool     rc    = true;
    178e:	2301      	movs	r3, #1
    1790:	e7b8      	b.n	1704 <_usb_d_dev_handler+0x44>
	tmp = ((Sysctrl *)hw)->PCLKSR.reg;
    1792:	4b58      	ldr	r3, [pc, #352]	; (18f4 <_usb_d_dev_handler+0x234>)
    1794:	68db      	ldr	r3, [r3, #12]
		while (hri_sysctrl_get_PCLKSR_reg(SYSCTRL, SYSCTRL_PCLKSR_DFLLRDY) != SYSCTRL_PCLKSR_DFLLRDY)
    1796:	06db      	lsls	r3, r3, #27
    1798:	d5fb      	bpl.n	1792 <_usb_d_dev_handler+0xd2>
    179a:	e7f3      	b.n	1784 <_usb_d_dev_handler+0xc4>
	((UsbDevice *)hw)->DeviceEndpoint[submodule_index].EPCFG.reg = data;
    179c:	4b52      	ldr	r3, [pc, #328]	; (18e8 <_usb_d_dev_handler+0x228>)
    179e:	2100      	movs	r1, #0
    17a0:	2280      	movs	r2, #128	; 0x80
    17a2:	0052      	lsls	r2, r2, #1
    17a4:	5499      	strb	r1, [r3, r2]
	((Usb *)hw)->DEVICE.INTFLAG.reg = mask;
    17a6:	3af8      	subs	r2, #248	; 0xf8
    17a8:	839a      	strh	r2, [r3, #28]
	((Usb *)hw)->DEVICE.INTENCLR.reg = mask;
    17aa:	3268      	adds	r2, #104	; 0x68
    17ac:	829a      	strh	r2, [r3, #20]
	((Usb *)hw)->DEVICE.INTENSET.reg = mask;
    17ae:	4a50      	ldr	r2, [pc, #320]	; (18f0 <_usb_d_dev_handler+0x230>)
    17b0:	831a      	strh	r2, [r3, #24]
	_usb_d_dev_reset_epts();
    17b2:	4b51      	ldr	r3, [pc, #324]	; (18f8 <_usb_d_dev_handler+0x238>)
    17b4:	4798      	blx	r3
	dev_inst.callbacks.event(USB_EV_RESET, 0);
    17b6:	4b4d      	ldr	r3, [pc, #308]	; (18ec <_usb_d_dev_handler+0x22c>)
    17b8:	6e5b      	ldr	r3, [r3, #100]	; 0x64
    17ba:	2100      	movs	r1, #0
    17bc:	2001      	movs	r0, #1
    17be:	4798      	blx	r3
	bool     rc    = true;
    17c0:	2301      	movs	r3, #1
    17c2:	e79f      	b.n	1704 <_usb_d_dev_handler+0x44>
	((Usb *)hw)->DEVICE.INTFLAG.reg = mask;
    17c4:	4b48      	ldr	r3, [pc, #288]	; (18e8 <_usb_d_dev_handler+0x228>)
    17c6:	4a4a      	ldr	r2, [pc, #296]	; (18f0 <_usb_d_dev_handler+0x230>)
    17c8:	839a      	strh	r2, [r3, #28]
	((Usb *)hw)->DEVICE.INTENCLR.reg = mask;
    17ca:	829a      	strh	r2, [r3, #20]
	((Usb *)hw)->DEVICE.INTENSET.reg = mask;
    17cc:	3a92      	subs	r2, #146	; 0x92
    17ce:	3aff      	subs	r2, #255	; 0xff
    17d0:	831a      	strh	r2, [r3, #24]
	dev_inst.callbacks.event(USB_EV_SUSPEND, 0);
    17d2:	4b46      	ldr	r3, [pc, #280]	; (18ec <_usb_d_dev_handler+0x22c>)
    17d4:	6e5b      	ldr	r3, [r3, #100]	; 0x64
    17d6:	2100      	movs	r1, #0
    17d8:	2004      	movs	r0, #4
    17da:	4798      	blx	r3
	bool     rc    = true;
    17dc:	2301      	movs	r3, #1
    17de:	e791      	b.n	1704 <_usb_d_dev_handler+0x44>
	if (flags & USB_DEVICE_EPINTFLAG_RXSTP) {
    17e0:	06da      	lsls	r2, r3, #27
    17e2:	d407      	bmi.n	17f4 <_usb_d_dev_handler+0x134>
	} else if (flags & USB_DEVICE_EPINTFLAG_STALL1) {
    17e4:	065a      	lsls	r2, r3, #25
    17e6:	d408      	bmi.n	17fa <_usb_d_dev_handler+0x13a>
	} else if (flags & USB_DEVICE_EPINTFLAG_STALL0) {
    17e8:	069b      	lsls	r3, r3, #26
    17ea:	d52f      	bpl.n	184c <_usb_d_dev_handler+0x18c>
		_usb_d_dev_handle_stall(ept, 0);
    17ec:	2100      	movs	r1, #0
    17ee:	4b43      	ldr	r3, [pc, #268]	; (18fc <_usb_d_dev_handler+0x23c>)
    17f0:	4798      	blx	r3
    17f2:	e02b      	b.n	184c <_usb_d_dev_handler+0x18c>
		_usb_d_dev_handle_setup(ept);
    17f4:	4b42      	ldr	r3, [pc, #264]	; (1900 <_usb_d_dev_handler+0x240>)
    17f6:	4798      	blx	r3
    17f8:	e028      	b.n	184c <_usb_d_dev_handler+0x18c>
		_usb_d_dev_handle_stall(ept, 1);
    17fa:	2101      	movs	r1, #1
    17fc:	4b3f      	ldr	r3, [pc, #252]	; (18fc <_usb_d_dev_handler+0x23c>)
    17fe:	4798      	blx	r3
    1800:	e024      	b.n	184c <_usb_d_dev_handler+0x18c>
	if (flags & USB_DEVICE_EPINTFLAG_STALL1) {
    1802:	065a      	lsls	r2, r3, #25
    1804:	d40f      	bmi.n	1826 <_usb_d_dev_handler+0x166>
	} else if (flags & USB_DEVICE_EPINTFLAG_TRFAIL1) {
    1806:	071a      	lsls	r2, r3, #28
    1808:	d411      	bmi.n	182e <_usb_d_dev_handler+0x16e>
	} else if (flags & USB_DEVICE_EPINTFLAG_TRCPT1) {
    180a:	079a      	lsls	r2, r3, #30
    180c:	d413      	bmi.n	1836 <_usb_d_dev_handler+0x176>
	} else if (_usb_d_dev_ep_is_ctrl(ept)) {
    180e:	7cc1      	ldrb	r1, [r0, #19]
    1810:	2207      	movs	r2, #7
    1812:	400a      	ands	r2, r1
    1814:	2a01      	cmp	r2, #1
    1816:	d119      	bne.n	184c <_usb_d_dev_handler+0x18c>
		if (flags & USB_DEVICE_EPINTFLAG_TRFAIL0) {
    1818:	075a      	lsls	r2, r3, #29
    181a:	d410      	bmi.n	183e <_usb_d_dev_handler+0x17e>
		} else if (flags & USB_DEVICE_EPINTFLAG_RXSTP) {
    181c:	06db      	lsls	r3, r3, #27
    181e:	d515      	bpl.n	184c <_usb_d_dev_handler+0x18c>
			_usb_d_dev_handle_setup(ept);
    1820:	4b37      	ldr	r3, [pc, #220]	; (1900 <_usb_d_dev_handler+0x240>)
    1822:	4798      	blx	r3
    1824:	e012      	b.n	184c <_usb_d_dev_handler+0x18c>
		_usb_d_dev_handle_stall(ept, 1);
    1826:	2101      	movs	r1, #1
    1828:	4b34      	ldr	r3, [pc, #208]	; (18fc <_usb_d_dev_handler+0x23c>)
    182a:	4798      	blx	r3
    182c:	e00e      	b.n	184c <_usb_d_dev_handler+0x18c>
		_usb_d_dev_handle_trfail(ept, 1);
    182e:	2101      	movs	r1, #1
    1830:	4b34      	ldr	r3, [pc, #208]	; (1904 <_usb_d_dev_handler+0x244>)
    1832:	4798      	blx	r3
    1834:	e00a      	b.n	184c <_usb_d_dev_handler+0x18c>
		_usb_d_dev_in_next(ept, true);
    1836:	2101      	movs	r1, #1
    1838:	4b33      	ldr	r3, [pc, #204]	; (1908 <_usb_d_dev_handler+0x248>)
    183a:	4798      	blx	r3
    183c:	e006      	b.n	184c <_usb_d_dev_handler+0x18c>
			_usb_d_dev_handle_trfail(ept, 0);
    183e:	2100      	movs	r1, #0
    1840:	4b30      	ldr	r3, [pc, #192]	; (1904 <_usb_d_dev_handler+0x244>)
    1842:	4798      	blx	r3
    1844:	e002      	b.n	184c <_usb_d_dev_handler+0x18c>
		_usb_d_dev_handle_stall(ept, 0);
    1846:	2100      	movs	r1, #0
    1848:	4b2c      	ldr	r3, [pc, #176]	; (18fc <_usb_d_dev_handler+0x23c>)
    184a:	4798      	blx	r3
	for (i = 0; i < USB_D_N_EP; i++) {
    184c:	3401      	adds	r4, #1
    184e:	b2e4      	uxtb	r4, r4
    1850:	2c08      	cmp	r4, #8
    1852:	d900      	bls.n	1856 <_usb_d_dev_handler+0x196>
    1854:	e758      	b.n	1708 <_usb_d_dev_handler+0x48>
		struct _usb_d_dev_ep *ept = &dev_inst.ep[i];
    1856:	4b25      	ldr	r3, [pc, #148]	; (18ec <_usb_d_dev_handler+0x22c>)
    1858:	3360      	adds	r3, #96	; 0x60
    185a:	00a2      	lsls	r2, r4, #2
    185c:	1911      	adds	r1, r2, r4
    185e:	0088      	lsls	r0, r1, #2
    1860:	0001      	movs	r1, r0
    1862:	3010      	adds	r0, #16
    1864:	1818      	adds	r0, r3, r0
    1866:	3004      	adds	r0, #4
		if (ept->ep == 0xFF) {
    1868:	185b      	adds	r3, r3, r1
    186a:	3326      	adds	r3, #38	; 0x26
    186c:	781b      	ldrb	r3, [r3, #0]
    186e:	2bff      	cmp	r3, #255	; 0xff
    1870:	d0ec      	beq.n	184c <_usb_d_dev_handler+0x18c>
	uint8_t epn = USB_EP_GET_N(ept->ep);
    1872:	7c82      	ldrb	r2, [r0, #18]
    1874:	230f      	movs	r3, #15
    1876:	4013      	ands	r3, r2
	if (!(epint & (1u << epn))) {
    1878:	2201      	movs	r2, #1
    187a:	409a      	lsls	r2, r3
    187c:	422a      	tst	r2, r5
    187e:	d0e5      	beq.n	184c <_usb_d_dev_handler+0x18c>
	flags = hw->DEVICE.DeviceEndpoint[epn].EPINTFLAG.reg;
    1880:	001a      	movs	r2, r3
    1882:	3208      	adds	r2, #8
    1884:	0152      	lsls	r2, r2, #5
    1886:	4918      	ldr	r1, [pc, #96]	; (18e8 <_usb_d_dev_handler+0x228>)
    1888:	468c      	mov	ip, r1
    188a:	4462      	add	r2, ip
    188c:	79d2      	ldrb	r2, [r2, #7]
	mask  = hw->DEVICE.DeviceEndpoint[epn].EPINTENSET.reg;
    188e:	015b      	lsls	r3, r3, #5
    1890:	491e      	ldr	r1, [pc, #120]	; (190c <_usb_d_dev_handler+0x24c>)
    1892:	468c      	mov	ip, r1
    1894:	4463      	add	r3, ip
    1896:	781b      	ldrb	r3, [r3, #0]
	flags &= mask;
    1898:	4013      	ands	r3, r2
	if (flags) {
    189a:	d0d7      	beq.n	184c <_usb_d_dev_handler+0x18c>
		if ((ept->flags.bits.eptype == 0x1) && !_usb_d_dev_ep_is_busy(ept)) {
    189c:	7cc2      	ldrb	r2, [r0, #19]
    189e:	2147      	movs	r1, #71	; 0x47
    18a0:	4011      	ands	r1, r2
    18a2:	2901      	cmp	r1, #1
    18a4:	d09c      	beq.n	17e0 <_usb_d_dev_handler+0x120>
		} else if (_usb_d_dev_ep_is_in(ept)) {
    18a6:	b252      	sxtb	r2, r2
    18a8:	2a00      	cmp	r2, #0
    18aa:	dbaa      	blt.n	1802 <_usb_d_dev_handler+0x142>
	if (flags & USB_DEVICE_EPINTFLAG_STALL0) {
    18ac:	069a      	lsls	r2, r3, #26
    18ae:	d4ca      	bmi.n	1846 <_usb_d_dev_handler+0x186>
	} else if (flags & USB_DEVICE_EPINTFLAG_TRFAIL0) {
    18b0:	075a      	lsls	r2, r3, #29
    18b2:	d40d      	bmi.n	18d0 <_usb_d_dev_handler+0x210>
	} else if (flags & USB_DEVICE_EPINTFLAG_TRCPT0) {
    18b4:	07da      	lsls	r2, r3, #31
    18b6:	d40f      	bmi.n	18d8 <_usb_d_dev_handler+0x218>
	} else if (_usb_d_dev_ep_is_ctrl(ept)) {
    18b8:	7cc1      	ldrb	r1, [r0, #19]
    18ba:	2207      	movs	r2, #7
    18bc:	400a      	ands	r2, r1
    18be:	2a01      	cmp	r2, #1
    18c0:	d1c4      	bne.n	184c <_usb_d_dev_handler+0x18c>
		if (flags & USB_DEVICE_EPINTFLAG_TRFAIL1) {
    18c2:	071a      	lsls	r2, r3, #28
    18c4:	d40c      	bmi.n	18e0 <_usb_d_dev_handler+0x220>
		} else if (flags & USB_DEVICE_EPINTFLAG_RXSTP) {
    18c6:	06db      	lsls	r3, r3, #27
    18c8:	d5c0      	bpl.n	184c <_usb_d_dev_handler+0x18c>
			_usb_d_dev_handle_setup(ept);
    18ca:	4b0d      	ldr	r3, [pc, #52]	; (1900 <_usb_d_dev_handler+0x240>)
    18cc:	4798      	blx	r3
    18ce:	e7bd      	b.n	184c <_usb_d_dev_handler+0x18c>
		_usb_d_dev_handle_trfail(ept, 0);
    18d0:	2100      	movs	r1, #0
    18d2:	4b0c      	ldr	r3, [pc, #48]	; (1904 <_usb_d_dev_handler+0x244>)
    18d4:	4798      	blx	r3
    18d6:	e7b9      	b.n	184c <_usb_d_dev_handler+0x18c>
		_usb_d_dev_out_next(ept, true);
    18d8:	2101      	movs	r1, #1
    18da:	4b0d      	ldr	r3, [pc, #52]	; (1910 <_usb_d_dev_handler+0x250>)
    18dc:	4798      	blx	r3
    18de:	e7b5      	b.n	184c <_usb_d_dev_handler+0x18c>
			_usb_d_dev_handle_trfail(ept, 1);
    18e0:	2101      	movs	r1, #1
    18e2:	4b08      	ldr	r3, [pc, #32]	; (1904 <_usb_d_dev_handler+0x244>)
    18e4:	4798      	blx	r3
    18e6:	e7b1      	b.n	184c <_usb_d_dev_handler+0x18c>
    18e8:	41005000 	.word	0x41005000
    18ec:	200000a0 	.word	0x200000a0
    18f0:	00000201 	.word	0x00000201
    18f4:	40000800 	.word	0x40000800
    18f8:	000012dd 	.word	0x000012dd
    18fc:	000010f9 	.word	0x000010f9
    1900:	0000106d 	.word	0x0000106d
    1904:	000011cd 	.word	0x000011cd
    1908:	00001331 	.word	0x00001331
    190c:	41005109 	.word	0x41005109
    1910:	000014bd 	.word	0x000014bd

00001914 <_usb_d_dev_init>:
{
    1914:	b500      	push	{lr}
    1916:	b083      	sub	sp, #12
	const uint8_t spdconf[4] = {
    1918:	2200      	movs	r2, #0
    191a:	ab01      	add	r3, sp, #4
    191c:	705a      	strb	r2, [r3, #1]
	return ((Usb *)hw)->DEVICE.SYNCBUSY.reg & reg;
    191e:	4b21      	ldr	r3, [pc, #132]	; (19a4 <_usb_d_dev_init+0x90>)
    1920:	789b      	ldrb	r3, [r3, #2]
	if (!hri_usbdevice_is_syncing(hw, USB_SYNCBUSY_SWRST)) {
    1922:	07db      	lsls	r3, r3, #31
    1924:	d41b      	bmi.n	195e <_usb_d_dev_init+0x4a>
	while (((Usb *)hw)->DEVICE.SYNCBUSY.reg & reg) {
    1926:	4b1f      	ldr	r3, [pc, #124]	; (19a4 <_usb_d_dev_init+0x90>)
    1928:	789b      	ldrb	r3, [r3, #2]
    192a:	079b      	lsls	r3, r3, #30
    192c:	d1fb      	bne.n	1926 <_usb_d_dev_init+0x12>

static inline hri_usb_ctrla_reg_t hri_usb_get_CTRLA_reg(const void *const hw, hri_usb_ctrla_reg_t mask)
{
	uint8_t tmp;
	hri_usb_wait_for_sync(hw, USB_SYNCBUSY_MASK);
	tmp = ((Usb *)hw)->HOST.CTRLA.reg;
    192e:	4b1d      	ldr	r3, [pc, #116]	; (19a4 <_usb_d_dev_init+0x90>)
    1930:	781b      	ldrb	r3, [r3, #0]
		if (hri_usbdevice_get_CTRLA_reg(hw, USB_CTRLA_ENABLE)) {
    1932:	079b      	lsls	r3, r3, #30
    1934:	d50c      	bpl.n	1950 <_usb_d_dev_init+0x3c>
	((Usb *)hw)->HOST.CTRLA.reg &= ~USB_CTRLA_ENABLE;
    1936:	4a1b      	ldr	r2, [pc, #108]	; (19a4 <_usb_d_dev_init+0x90>)
    1938:	7813      	ldrb	r3, [r2, #0]
    193a:	2102      	movs	r1, #2
    193c:	438b      	bics	r3, r1
    193e:	7013      	strb	r3, [r2, #0]
	while (((Usb *)hw)->DEVICE.SYNCBUSY.reg & reg) {
    1940:	4b18      	ldr	r3, [pc, #96]	; (19a4 <_usb_d_dev_init+0x90>)
    1942:	789b      	ldrb	r3, [r3, #2]
    1944:	079b      	lsls	r3, r3, #30
    1946:	d1fb      	bne.n	1940 <_usb_d_dev_init+0x2c>
    1948:	4b16      	ldr	r3, [pc, #88]	; (19a4 <_usb_d_dev_init+0x90>)
    194a:	789b      	ldrb	r3, [r3, #2]
    194c:	079b      	lsls	r3, r3, #30
    194e:	d4fb      	bmi.n	1948 <_usb_d_dev_init+0x34>
}

static inline void hri_usb_write_CTRLA_reg(const void *const hw, hri_usb_ctrla_reg_t data)
{
	USB_CRITICAL_SECTION_ENTER();
	((Usb *)hw)->HOST.CTRLA.reg = data;
    1950:	2201      	movs	r2, #1
    1952:	4b14      	ldr	r3, [pc, #80]	; (19a4 <_usb_d_dev_init+0x90>)
    1954:	701a      	strb	r2, [r3, #0]
	while (((Usb *)hw)->DEVICE.SYNCBUSY.reg & reg) {
    1956:	4b13      	ldr	r3, [pc, #76]	; (19a4 <_usb_d_dev_init+0x90>)
    1958:	789b      	ldrb	r3, [r3, #2]
    195a:	079b      	lsls	r3, r3, #30
    195c:	d1fb      	bne.n	1956 <_usb_d_dev_init+0x42>
    195e:	4b11      	ldr	r3, [pc, #68]	; (19a4 <_usb_d_dev_init+0x90>)
    1960:	789b      	ldrb	r3, [r3, #2]
    1962:	07db      	lsls	r3, r3, #31
    1964:	d4fb      	bmi.n	195e <_usb_d_dev_init+0x4a>
	dev_inst.callbacks.sof   = (_usb_d_dev_sof_cb_t)_dummy_func_no_return;
    1966:	4b10      	ldr	r3, [pc, #64]	; (19a8 <_usb_d_dev_init+0x94>)
    1968:	4a10      	ldr	r2, [pc, #64]	; (19ac <_usb_d_dev_init+0x98>)
    196a:	661a      	str	r2, [r3, #96]	; 0x60
	dev_inst.callbacks.event = (_usb_d_dev_event_cb_t)_dummy_func_no_return;
    196c:	665a      	str	r2, [r3, #100]	; 0x64
	dev_inst.ep_callbacks.setup = (_usb_d_dev_ep_cb_setup_t)_dummy_func_no_return;
    196e:	669a      	str	r2, [r3, #104]	; 0x68
	dev_inst.ep_callbacks.more  = (_usb_d_dev_ep_cb_more_t)_dummy_func_no_return;
    1970:	66da      	str	r2, [r3, #108]	; 0x6c
	dev_inst.ep_callbacks.done  = (_usb_d_dev_ep_cb_done_t)_dummy_func_no_return;
    1972:	671a      	str	r2, [r3, #112]	; 0x70
	_usb_d_dev_reset_epts();
    1974:	4b0e      	ldr	r3, [pc, #56]	; (19b0 <_usb_d_dev_init+0x9c>)
    1976:	4798      	blx	r3
	_usb_load_calib();
    1978:	4b0e      	ldr	r3, [pc, #56]	; (19b4 <_usb_d_dev_init+0xa0>)
    197a:	4798      	blx	r3
	((Usb *)hw)->HOST.CTRLA.reg = data;
    197c:	2204      	movs	r2, #4
    197e:	4b09      	ldr	r3, [pc, #36]	; (19a4 <_usb_d_dev_init+0x90>)
    1980:	701a      	strb	r2, [r3, #0]
	while (((Usb *)hw)->DEVICE.SYNCBUSY.reg & reg) {
    1982:	4b08      	ldr	r3, [pc, #32]	; (19a4 <_usb_d_dev_init+0x90>)
    1984:	789b      	ldrb	r3, [r3, #2]
    1986:	079b      	lsls	r3, r3, #30
    1988:	d1fb      	bne.n	1982 <_usb_d_dev_init+0x6e>
}

static inline void hri_usb_write_DESCADD_reg(const void *const hw, hri_usb_descadd_reg_t data)
{
	USB_CRITICAL_SECTION_ENTER();
	((Usb *)hw)->HOST.DESCADD.reg = data;
    198a:	4a06      	ldr	r2, [pc, #24]	; (19a4 <_usb_d_dev_init+0x90>)
    198c:	4b06      	ldr	r3, [pc, #24]	; (19a8 <_usb_d_dev_init+0x94>)
    198e:	6253      	str	r3, [r2, #36]	; 0x24
	hri_usbdevice_write_CTRLB_reg(hw, spdconf[speed] | USB_DEVICE_CTRLB_DETACH);
    1990:	ab01      	add	r3, sp, #4
    1992:	785b      	ldrb	r3, [r3, #1]
    1994:	2101      	movs	r1, #1
    1996:	430b      	orrs	r3, r1
    1998:	b2db      	uxtb	r3, r3
	((Usb *)hw)->DEVICE.CTRLB.reg = data;
    199a:	8113      	strh	r3, [r2, #8]
}
    199c:	2000      	movs	r0, #0
    199e:	b003      	add	sp, #12
    19a0:	bd00      	pop	{pc}
    19a2:	46c0      	nop			; (mov r8, r8)
    19a4:	41005000 	.word	0x41005000
    19a8:	200000a0 	.word	0x200000a0
    19ac:	00001015 	.word	0x00001015
    19b0:	000012dd 	.word	0x000012dd
    19b4:	00001019 	.word	0x00001019

000019b8 <_usb_d_dev_ep_stall>:
{
    19b8:	b5f0      	push	{r4, r5, r6, r7, lr}
	uint8_t               epn = USB_EP_GET_N(ep);
    19ba:	220f      	movs	r2, #15
    19bc:	4002      	ands	r2, r0
    19be:	b240      	sxtb	r0, r0
	bool                  dir = USB_EP_GET_DIR(ep);
    19c0:	0fc4      	lsrs	r4, r0, #31
	uint8_t ep_index = (epn == 0) ? 0 : (dir ? (epn + CONF_USB_D_MAX_EP_N) : epn);
    19c2:	2a00      	cmp	r2, #0
    19c4:	d005      	beq.n	19d2 <_usb_d_dev_ep_stall+0x1a>
    19c6:	2800      	cmp	r0, #0
    19c8:	db01      	blt.n	19ce <_usb_d_dev_ep_stall+0x16>
    19ca:	0013      	movs	r3, r2
    19cc:	e002      	b.n	19d4 <_usb_d_dev_ep_stall+0x1c>
    19ce:	1c93      	adds	r3, r2, #2
    19d0:	e000      	b.n	19d4 <_usb_d_dev_ep_stall+0x1c>
    19d2:	0013      	movs	r3, r2
	return &dev_inst.ep[ep_index];
    19d4:	001d      	movs	r5, r3
    19d6:	0098      	lsls	r0, r3, #2
    19d8:	18c0      	adds	r0, r0, r3
    19da:	0083      	lsls	r3, r0, #2
    19dc:	3310      	adds	r3, #16
    19de:	0018      	movs	r0, r3
    19e0:	4b47      	ldr	r3, [pc, #284]	; (1b00 <_usb_d_dev_ep_stall+0x148>)
    19e2:	3360      	adds	r3, #96	; 0x60
    19e4:	181b      	adds	r3, r3, r0
    19e6:	3304      	adds	r3, #4
	if (epn > CONF_USB_D_MAX_EP_N) {
    19e8:	2a02      	cmp	r2, #2
    19ea:	d900      	bls.n	19ee <_usb_d_dev_ep_stall+0x36>
    19ec:	e084      	b.n	1af8 <_usb_d_dev_ep_stall+0x140>
	if (USB_EP_STALL_SET == ctrl) {
    19ee:	2901      	cmp	r1, #1
    19f0:	d018      	beq.n	1a24 <_usb_d_dev_ep_stall+0x6c>
	} else if (USB_EP_STALL_CLR == ctrl) {
    19f2:	2900      	cmp	r1, #0
    19f4:	d03d      	beq.n	1a72 <_usb_d_dev_ep_stall+0xba>
	uint8_t epn = USB_EP_GET_N(ept->ep);
    19f6:	00aa      	lsls	r2, r5, #2
    19f8:	1952      	adds	r2, r2, r5
    19fa:	0091      	lsls	r1, r2, #2
    19fc:	4b40      	ldr	r3, [pc, #256]	; (1b00 <_usb_d_dev_ep_stall+0x148>)
    19fe:	3360      	adds	r3, #96	; 0x60
    1a00:	185b      	adds	r3, r3, r1
    1a02:	3326      	adds	r3, #38	; 0x26
    1a04:	781a      	ldrb	r2, [r3, #0]
    1a06:	230f      	movs	r3, #15
    1a08:	4013      	ands	r3, r2
	return ((UsbDevice *)hw)->DeviceEndpoint[submodule_index].EPSTATUS.reg;
    1a0a:	3308      	adds	r3, #8
    1a0c:	015b      	lsls	r3, r3, #5
    1a0e:	4a3d      	ldr	r2, [pc, #244]	; (1b04 <_usb_d_dev_ep_stall+0x14c>)
    1a10:	4694      	mov	ip, r2
    1a12:	4463      	add	r3, ip
    1a14:	7998      	ldrb	r0, [r3, #6]
	return (hri_usbendpoint_read_EPSTATUS_reg(hw, epn) & (USB_DEVICE_EPSTATUS_STALLRQ0 << bank_n));
    1a16:	2310      	movs	r3, #16
    1a18:	40a3      	lsls	r3, r4
    1a1a:	4018      	ands	r0, r3
    1a1c:	1e43      	subs	r3, r0, #1
    1a1e:	4198      	sbcs	r0, r3
    1a20:	b2c0      	uxtb	r0, r0
}
    1a22:	bdf0      	pop	{r4, r5, r6, r7, pc}
	uint8_t epn = USB_EP_GET_N(ept->ep);
    1a24:	4836      	ldr	r0, [pc, #216]	; (1b00 <_usb_d_dev_ep_stall+0x148>)
    1a26:	0003      	movs	r3, r0
    1a28:	3360      	adds	r3, #96	; 0x60
    1a2a:	00aa      	lsls	r2, r5, #2
    1a2c:	1956      	adds	r6, r2, r5
    1a2e:	00b1      	lsls	r1, r6, #2
    1a30:	185b      	adds	r3, r3, r1
    1a32:	3326      	adds	r3, #38	; 0x26
    1a34:	781b      	ldrb	r3, [r3, #0]
    1a36:	210f      	movs	r1, #15
    1a38:	400b      	ands	r3, r1
		hri_usbendpoint_set_EPSTATUS_reg(USB, epn, (USB_DEVICE_EPSTATUS_STALLRQ0 << bank_n));
    1a3a:	2610      	movs	r6, #16
    1a3c:	40a6      	lsls	r6, r4
    1a3e:	b2f6      	uxtb	r6, r6
	((UsbDevice *)hw)->DeviceEndpoint[submodule_index].EPSTATUSSET.reg = mask;
    1a40:	0019      	movs	r1, r3
    1a42:	3108      	adds	r1, #8
    1a44:	0149      	lsls	r1, r1, #5
    1a46:	4f2f      	ldr	r7, [pc, #188]	; (1b04 <_usb_d_dev_ep_stall+0x14c>)
    1a48:	46bc      	mov	ip, r7
    1a4a:	4461      	add	r1, ip
    1a4c:	714e      	strb	r6, [r1, #5]
	_usbd_ep_int_en(epn, USB_DEVICE_EPINTFLAG_STALL0 << dir);
    1a4e:	2120      	movs	r1, #32
    1a50:	40a1      	lsls	r1, r4
	hri_usbendpoint_set_EPINTEN_reg(USB, epn, flags);
    1a52:	b2cc      	uxtb	r4, r1
	((UsbDevice *)hw)->DeviceEndpoint[submodule_index].EPINTENSET.reg = mask;
    1a54:	0159      	lsls	r1, r3, #5
    1a56:	4b2c      	ldr	r3, [pc, #176]	; (1b08 <_usb_d_dev_ep_stall+0x150>)
    1a58:	469c      	mov	ip, r3
    1a5a:	4461      	add	r1, ip
    1a5c:	700c      	strb	r4, [r1, #0]
	ept->flags.bits.is_stalled = 1;
    1a5e:	1952      	adds	r2, r2, r5
    1a60:	0093      	lsls	r3, r2, #2
    1a62:	18c3      	adds	r3, r0, r3
    1a64:	3380      	adds	r3, #128	; 0x80
    1a66:	79da      	ldrb	r2, [r3, #7]
    1a68:	2108      	movs	r1, #8
    1a6a:	430a      	orrs	r2, r1
    1a6c:	71da      	strb	r2, [r3, #7]
		rc = _usb_d_dev_ep_stall_set(ept, dir);
    1a6e:	2000      	movs	r0, #0
    1a70:	e7d7      	b.n	1a22 <_usb_d_dev_ep_stall+0x6a>
	uint8_t epn        = USB_EP_GET_N(ept->ep);
    1a72:	7c9a      	ldrb	r2, [r3, #18]
    1a74:	310f      	adds	r1, #15
    1a76:	400a      	ands	r2, r1
	return ((UsbDevice *)hw)->DeviceEndpoint[submodule_index].EPSTATUS.reg;
    1a78:	0011      	movs	r1, r2
    1a7a:	3108      	adds	r1, #8
    1a7c:	0149      	lsls	r1, r1, #5
    1a7e:	4821      	ldr	r0, [pc, #132]	; (1b04 <_usb_d_dev_ep_stall+0x14c>)
    1a80:	4684      	mov	ip, r0
    1a82:	4461      	add	r1, ip
    1a84:	7988      	ldrb	r0, [r1, #6]
	return (hri_usbendpoint_read_EPSTATUS_reg(hw, epn) & (USB_DEVICE_EPSTATUS_STALLRQ0 << bank_n));
    1a86:	2110      	movs	r1, #16
    1a88:	40a1      	lsls	r1, r4
	if (!is_stalled) {
    1a8a:	4208      	tst	r0, r1
    1a8c:	d024      	beq.n	1ad8 <_usb_d_dev_ep_stall+0x120>
		hri_usbendpoint_clear_EPSTATUS_reg(USB, epn, (USB_DEVICE_EPSTATUS_STALLRQ0 << bank_n));
    1a8e:	b2c9      	uxtb	r1, r1
	((UsbDevice *)hw)->DeviceEndpoint[submodule_index].EPSTATUSCLR.reg = mask;
    1a90:	0010      	movs	r0, r2
    1a92:	3008      	adds	r0, #8
    1a94:	0140      	lsls	r0, r0, #5
    1a96:	4460      	add	r0, ip
    1a98:	7101      	strb	r1, [r0, #4]
	_usbd_ep_int_dis(epn, USB_DEVICE_EPINTFLAG_STALL0 << dir);
    1a9a:	2120      	movs	r1, #32
    1a9c:	40a1      	lsls	r1, r4
	hri_usbendpoint_clear_EPINTEN_reg(USB, epn, flags);
    1a9e:	b2ce      	uxtb	r6, r1
	((UsbDevice *)hw)->DeviceEndpoint[submodule_index].EPINTENCLR.reg = mask;
    1aa0:	0155      	lsls	r5, r2, #5
    1aa2:	4f1a      	ldr	r7, [pc, #104]	; (1b0c <_usb_d_dev_ep_stall+0x154>)
    1aa4:	46bc      	mov	ip, r7
    1aa6:	4465      	add	r5, ip
    1aa8:	702e      	strb	r6, [r5, #0]
	return ((UsbDevice *)hw)->DeviceEndpoint[submodule_index].EPINTFLAG.reg;
    1aaa:	79c0      	ldrb	r0, [r0, #7]
	if (_usbd_ep_is_stall_sent(epn, dir)) {
    1aac:	4208      	tst	r0, r1
    1aae:	d00a      	beq.n	1ac6 <_usb_d_dev_ep_stall+0x10e>
	((UsbDevice *)hw)->DeviceEndpoint[submodule_index].EPINTFLAG.reg = mask;
    1ab0:	0011      	movs	r1, r2
    1ab2:	3108      	adds	r1, #8
    1ab4:	0149      	lsls	r1, r1, #5
    1ab6:	4813      	ldr	r0, [pc, #76]	; (1b04 <_usb_d_dev_ep_stall+0x14c>)
    1ab8:	4684      	mov	ip, r0
    1aba:	4461      	add	r1, ip
    1abc:	71ce      	strb	r6, [r1, #7]
		hri_usbendpoint_clear_EPSTATUS_reg(USB, epn, (USB_DEVICE_EPSTATUS_DTGLOUT << bank_n));
    1abe:	2001      	movs	r0, #1
    1ac0:	40a0      	lsls	r0, r4
    1ac2:	b2c0      	uxtb	r0, r0
	((UsbDevice *)hw)->DeviceEndpoint[submodule_index].EPSTATUSCLR.reg = mask;
    1ac4:	7108      	strb	r0, [r1, #4]
	if (_usb_d_dev_ep_is_ctrl(ept)) {
    1ac6:	7cd8      	ldrb	r0, [r3, #19]
    1ac8:	2107      	movs	r1, #7
    1aca:	4001      	ands	r1, r0
    1acc:	2901      	cmp	r1, #1
    1ace:	d005      	beq.n	1adc <_usb_d_dev_ep_stall+0x124>
		ept->flags.bits.is_stalled = 0;
    1ad0:	7cda      	ldrb	r2, [r3, #19]
    1ad2:	2108      	movs	r1, #8
    1ad4:	438a      	bics	r2, r1
    1ad6:	74da      	strb	r2, [r3, #19]
		rc = _usb_d_dev_ep_stall_clr(ept, dir);
    1ad8:	2000      	movs	r0, #0
    1ada:	e7a2      	b.n	1a22 <_usb_d_dev_ep_stall+0x6a>
	return ((UsbDevice *)hw)->DeviceEndpoint[submodule_index].EPSTATUS.reg;
    1adc:	3208      	adds	r2, #8
    1ade:	0152      	lsls	r2, r2, #5
    1ae0:	4908      	ldr	r1, [pc, #32]	; (1b04 <_usb_d_dev_ep_stall+0x14c>)
    1ae2:	468c      	mov	ip, r1
    1ae4:	4462      	add	r2, ip
    1ae6:	7991      	ldrb	r1, [r2, #6]
		if ((hri_usbendpoint_read_EPSTATUS_reg(USB, epn) & USB_DEVICE_EPSTATUS_STALLRQ_Msk) == 0) {
    1ae8:	2230      	movs	r2, #48	; 0x30
    1aea:	4211      	tst	r1, r2
    1aec:	d1f4      	bne.n	1ad8 <_usb_d_dev_ep_stall+0x120>
			ept->flags.bits.is_stalled = 0;
    1aee:	0002      	movs	r2, r0
    1af0:	2108      	movs	r1, #8
    1af2:	438a      	bics	r2, r1
    1af4:	74da      	strb	r2, [r3, #19]
    1af6:	e7ef      	b.n	1ad8 <_usb_d_dev_ep_stall+0x120>
		return -USB_ERR_PARAM;
    1af8:	2012      	movs	r0, #18
    1afa:	4240      	negs	r0, r0
    1afc:	e791      	b.n	1a22 <_usb_d_dev_ep_stall+0x6a>
    1afe:	46c0      	nop			; (mov r8, r8)
    1b00:	200000a0 	.word	0x200000a0
    1b04:	41005000 	.word	0x41005000
    1b08:	41005109 	.word	0x41005109
    1b0c:	41005108 	.word	0x41005108

00001b10 <_usb_d_dev_ep_read_req>:

int32_t _usb_d_dev_ep_read_req(const uint8_t ep, uint8_t *req_buf)
{
    1b10:	b570      	push	{r4, r5, r6, lr}
    1b12:	000e      	movs	r6, r1
	uint8_t            epn   = USB_EP_GET_N(ep);
    1b14:	240f      	movs	r4, #15
    1b16:	4004      	ands	r4, r0
	UsbDeviceDescBank *bank  = prvt_inst.desc_table[epn].DeviceDescBank;
    1b18:	0162      	lsls	r2, r4, #5
    1b1a:	4b18      	ldr	r3, [pc, #96]	; (1b7c <_usb_d_dev_ep_read_req+0x6c>)
    1b1c:	189b      	adds	r3, r3, r2
	uint32_t           addr  = bank[0].ADDR.reg;
    1b1e:	6819      	ldr	r1, [r3, #0]
	uint16_t           bytes = bank[0].PCKSIZE.bit.BYTE_COUNT;
    1b20:	685d      	ldr	r5, [r3, #4]
    1b22:	04ad      	lsls	r5, r5, #18
    1b24:	0cad      	lsrs	r5, r5, #18

	if (epn > CONF_USB_D_MAX_EP_N || !req_buf) {
    1b26:	2c02      	cmp	r4, #2
    1b28:	d81f      	bhi.n	1b6a <_usb_d_dev_ep_read_req+0x5a>
    1b2a:	2e00      	cmp	r6, #0
    1b2c:	d020      	beq.n	1b70 <_usb_d_dev_ep_read_req+0x60>
	return ((UsbDevice *)hw)->DeviceEndpoint[submodule_index].EPCFG.reg;
    1b2e:	0023      	movs	r3, r4
    1b30:	3308      	adds	r3, #8
    1b32:	015b      	lsls	r3, r3, #5
    1b34:	4a12      	ldr	r2, [pc, #72]	; (1b80 <_usb_d_dev_ep_read_req+0x70>)
    1b36:	5c9b      	ldrb	r3, [r3, r2]
		return -USB_ERR_PARAM;
	}
	if (!_usbd_ep_is_ctrl(epn)) {
    1b38:	2b11      	cmp	r3, #17
    1b3a:	d11c      	bne.n	1b76 <_usb_d_dev_ep_read_req+0x66>
	tmp = ((UsbDevice *)hw)->DeviceEndpoint[submodule_index].EPINTFLAG.reg;
    1b3c:	0023      	movs	r3, r4
    1b3e:	3308      	adds	r3, #8
    1b40:	015b      	lsls	r3, r3, #5
    1b42:	4694      	mov	ip, r2
    1b44:	4463      	add	r3, ip
    1b46:	79db      	ldrb	r3, [r3, #7]
		return -USB_ERR_FUNC;
	}
	if (!_usbd_ep_is_setup(epn)) {
    1b48:	06db      	lsls	r3, r3, #27
    1b4a:	d401      	bmi.n	1b50 <_usb_d_dev_ep_read_req+0x40>
		return ERR_NONE;
    1b4c:	2000      	movs	r0, #0
	}
	memcpy(req_buf, (void *)addr, 8);
	_usbd_ep_ack_setup(epn);

	return bytes;
}
    1b4e:	bd70      	pop	{r4, r5, r6, pc}
	memcpy(req_buf, (void *)addr, 8);
    1b50:	2208      	movs	r2, #8
    1b52:	0030      	movs	r0, r6
    1b54:	4b0b      	ldr	r3, [pc, #44]	; (1b84 <_usb_d_dev_ep_read_req+0x74>)
    1b56:	4798      	blx	r3
	((UsbDevice *)hw)->DeviceEndpoint[submodule_index].EPINTFLAG.reg = mask;
    1b58:	3408      	adds	r4, #8
    1b5a:	0164      	lsls	r4, r4, #5
    1b5c:	4b08      	ldr	r3, [pc, #32]	; (1b80 <_usb_d_dev_ep_read_req+0x70>)
    1b5e:	469c      	mov	ip, r3
    1b60:	4464      	add	r4, ip
    1b62:	2310      	movs	r3, #16
    1b64:	71e3      	strb	r3, [r4, #7]
	return bytes;
    1b66:	0028      	movs	r0, r5
    1b68:	e7f1      	b.n	1b4e <_usb_d_dev_ep_read_req+0x3e>
		return -USB_ERR_PARAM;
    1b6a:	2012      	movs	r0, #18
    1b6c:	4240      	negs	r0, r0
    1b6e:	e7ee      	b.n	1b4e <_usb_d_dev_ep_read_req+0x3e>
    1b70:	2012      	movs	r0, #18
    1b72:	4240      	negs	r0, r0
    1b74:	e7eb      	b.n	1b4e <_usb_d_dev_ep_read_req+0x3e>
		return -USB_ERR_FUNC;
    1b76:	2013      	movs	r0, #19
    1b78:	4240      	negs	r0, r0
    1b7a:	e7e8      	b.n	1b4e <_usb_d_dev_ep_read_req+0x3e>
    1b7c:	200000a0 	.word	0x200000a0
    1b80:	41005000 	.word	0x41005000
    1b84:	00001e1d 	.word	0x00001e1d

00001b88 <_usb_d_dev_ep_trans>:

int32_t _usb_d_dev_ep_trans(const struct usb_d_transfer *trans)
{
    1b88:	b5f0      	push	{r4, r5, r6, r7, lr}
    1b8a:	46de      	mov	lr, fp
    1b8c:	4657      	mov	r7, sl
    1b8e:	464e      	mov	r6, r9
    1b90:	4645      	mov	r5, r8
    1b92:	b5e0      	push	{r5, r6, r7, lr}
    1b94:	b085      	sub	sp, #20
    1b96:	4680      	mov	r8, r0
	uint8_t               epn = USB_EP_GET_N(trans->ep);
    1b98:	7a05      	ldrb	r5, [r0, #8]
    1b9a:	220f      	movs	r2, #15
    1b9c:	402a      	ands	r2, r5
    1b9e:	b26d      	sxtb	r5, r5
	bool                  dir = USB_EP_GET_DIR(trans->ep);
    1ba0:	0feb      	lsrs	r3, r5, #31
    1ba2:	4699      	mov	r9, r3
	uint8_t ep_index = (epn == 0) ? 0 : (dir ? (epn + CONF_USB_D_MAX_EP_N) : epn);
    1ba4:	2a00      	cmp	r2, #0
    1ba6:	d005      	beq.n	1bb4 <_usb_d_dev_ep_trans+0x2c>
    1ba8:	2d00      	cmp	r5, #0
    1baa:	db01      	blt.n	1bb0 <_usb_d_dev_ep_trans+0x28>
    1bac:	0010      	movs	r0, r2
    1bae:	e002      	b.n	1bb6 <_usb_d_dev_ep_trans+0x2e>
    1bb0:	1c90      	adds	r0, r2, #2
    1bb2:	e000      	b.n	1bb6 <_usb_d_dev_ep_trans+0x2e>
    1bb4:	0010      	movs	r0, r2
	return &dev_inst.ep[ep_index];
    1bb6:	0006      	movs	r6, r0
    1bb8:	4b61      	ldr	r3, [pc, #388]	; (1d40 <_usb_d_dev_ep_trans+0x1b8>)
    1bba:	3360      	adds	r3, #96	; 0x60
    1bbc:	0081      	lsls	r1, r0, #2
    1bbe:	180f      	adds	r7, r1, r0
    1bc0:	00bc      	lsls	r4, r7, #2
    1bc2:	3410      	adds	r4, #16
    1bc4:	191c      	adds	r4, r3, r4
    1bc6:	3404      	adds	r4, #4
	struct _usb_d_dev_ep *ept = _usb_d_dev_ept(epn, dir);

	uint16_t size_mask      = (ept->size == 1023) ? 1023 : (ept->size - 1);
    1bc8:	00b8      	lsls	r0, r7, #2
    1bca:	181b      	adds	r3, r3, r0
    1bcc:	8c9b      	ldrh	r3, [r3, #36]	; 0x24
    1bce:	495d      	ldr	r1, [pc, #372]	; (1d44 <_usb_d_dev_ep_trans+0x1bc>)
    1bd0:	428b      	cmp	r3, r1
    1bd2:	d044      	beq.n	1c5e <_usb_d_dev_ep_trans+0xd6>
    1bd4:	1e5f      	subs	r7, r3, #1
    1bd6:	b2bf      	uxth	r7, r7
	bool     size_n_aligned = (trans->size & size_mask);
    1bd8:	4641      	mov	r1, r8
    1bda:	6849      	ldr	r1, [r1, #4]
    1bdc:	400f      	ands	r7, r1

	bool use_cache = false;

	volatile hal_atomic_t flags;

	if (epn > CONF_USB_D_MAX_EP_N) {
    1bde:	2a02      	cmp	r2, #2
    1be0:	d900      	bls.n	1be4 <_usb_d_dev_ep_trans+0x5c>
    1be2:	e0a3      	b.n	1d2c <_usb_d_dev_ep_trans+0x1a4>
	 * 1. Buffer not in RAM (cache all).
	 * 2. IN/OUT with unaligned buffer (cache all).
	 * 3. OUT with unaligned packet size (cache last packet).
	 * 4. OUT size < 8 (sub-case for 3).
	 */
	if (!_usb_is_addr4dma(trans->buf, trans->size) || (!_usb_is_aligned(trans->buf))
    1be4:	4642      	mov	r2, r8
    1be6:	6812      	ldr	r2, [r2, #0]
    1be8:	4857      	ldr	r0, [pc, #348]	; (1d48 <_usb_d_dev_ep_trans+0x1c0>)
    1bea:	4282      	cmp	r2, r0
    1bec:	d90c      	bls.n	1c08 <_usb_d_dev_ep_trans+0x80>
    1bee:	1888      	adds	r0, r1, r2
    1bf0:	9001      	str	r0, [sp, #4]
